:100000000C9436560C9467560C9467560C946756AD
:100010000C9467560D9472600C9467560C94675656
:100020000C946E740C9467560C9467560C94675637
:100030000C94F3660C9467560D94DB330D94682D85
:100040000C9467560D9463440C9467560C94675651
:100050000C9467560C9467560C9467560C94A273D4
:100060000C9467560D949CD60C9467560C94675666
:100070000C9467560C94C78C0C9467560C94675676
:100080000C9467560C9467560C9467560C946756FC
:100090000D9458D60C9467560C9467560C9467567A
:1000A0000C9467560C9467560D9482230C946756F3
:1000B0000C9467560D9464230C9467560D9425395F
:1000C0000C9467560C9467560C9467560D94242331
:1000D0000C9467560C9467560C9467560C946756AC
:1000E0000C946756000000000000000000000000B3
:1000F0000000000000000000000000000000000000
:100100005F5345435F4C414E470000000000000034
:1001100000000000000000000000000000000000DF
:1001200000000000000000000000000000000000CF
:1001300000000000000000000000000000000000BF
:1001400000000000000000000000000000000000AF
:103600000000437261736820646574656374656467
:103610002E000100536F6D652070726F626C656DD6
:1036200020656E636F756E74657265642C205A2D0B
:103630006C6576656C696E6720656E666F72636532
:1036400064202E2E2E0002004D6573682062656492
:10365000206C6576656C696E67206661696C65646F
:103660002E205072696E742063616E63656C6564B0
:103670002E00030048656174696E67206469736198
:10368000626C656420627920736166657479207468
:10369000696D65722E00040053544F505045442EFE
:1036A00000050050415553454420544845524D4172
:1036B0004C204552524F52000600472D636F6465FF
:1036C00020736C6963656420666F72206120646991
:1036D00066666572656E74206C6576656C2E000793
:1036E00000472D636F646520736C696365642066B1
:1036F0006F72206120646966666572656E74206C05
:103700006576656C2E20506C656173652072652D41
:10371000736C69636520746865206D6F64656C20E7
:10372000616761696E2E000800472D636F64652034
:10373000736C6963656420666F722061206E6577C3
:103740006572206669726D776172652E00090047A7
:103750002D636F646520736C6963656420666F72A6
:103760002061206E65776572206669726D7761727F
:10377000652E20506C656173652075706461746599
:1037800020746865206669726D776172652E000A23
:1037900000472D636F646520736C69636564206600
:1037A0006F72206120646966666572656E74207050
:1037B00072696E74657220747970652E000B004713
:1037C0002D636F646520736C6963656420666F7236
:1037D000206120646966666572656E742070726926
:1037E0006E74657220747970652E20506C656173FB
:1037F000652072652D736C69636520746865206D42
:103800006F64656C20616761696E2E000C005072F8
:1038100065737320746865206B6E6F6220746F200F
:1038200070726568656174206E6F7A7A6C6520616C
:103830006E6420636F6E74696E75652E000D0050A6
:103840006C656173652070726573732074686520A0
:103850006B6E6F6220746F20756E6C6F6164206692
:10386000696C616D656E74000E00616E642070722B
:1038700065737320746865206B6E6F62000F00497A
:103880006E736572742066696C616D656E7400108C
:1038900000436F6C6F72206E6F7420636F7272657D
:1038A000637400110046696C616D656E74206E6F03
:1038B00074206C6F616465640012004368616E6718
:1038C000656420636F72726563746C790013004CD9
:1038D0006F6164696E6720636F6C6F7200140043E0
:1038E00068616E6765207375636365737321001586
:1038F00000506C65617365206F70656E2069646C43
:10390000657220616E642072656D6F7665206669F0
:103910006C616D656E74206D616E75616C6C792E75
:103920000016005761732066696C616D656E7420C6
:10393000756E6C6F61642073756363657373667510
:103940006C3F001700506C6561736520757067727D
:103950006164652E0018004E6577206669726D7788
:103960006172652076657273696F6E206176616938
:103970006C61626C653A00190057616974696E6721
:1039800020666F722050494E44412070726F62650C
:1039900020636F6F6C696E67001A00506C6561730D
:1039A000652077616974001B004E6F206D6F76652E
:1039B0002E001C005761697420666F722075736554
:1039C000722E2E2E001D00537461626C6520616D95
:1039D0006269656E742074656D706572617475726C
:1039E000652032312D323643206973206E6565645F
:1039F00065642061207269676964207374616E6414
:103A00002069732072657175697265642E001E00ED
:103A1000506C656173652072756E2058595A206329
:103A2000616C6962726174696F6E20666972737429
:103A30002E001F0045787472756465720020004D79
:103A40006F7665205A0021004D6F7665205900225F
:103A5000004D6F7665205800230043726173682023
:103A6000646574656374696F6E2063616E0A626574
:103A7000207475726E6564206F6E206F6E6C792095
:103A8000696E0A4E6F726D616C206D6F6465002403
:103A9000005741524E494E473A0A437261736820BB
:103AA000646574656374696F6E0A64697361626CDE
:103AB000656420696E0A537465616C7468206D6F6B
:103AC00064650025004D6F6465206368616E6765FD
:103AD00020696E2070726F67726573732E2E2E00D0
:103AE0002600436F70792073656C6563746564208C
:103AF0006C616E67756167653F002700436F6D6D90
:103B0000756E697479206D6164650028005368657D
:103B1000657420252E37730A5A206F6666736574A4
:103B20003A20252B312E33666D6D0A2563436F6E67
:103B300074696E75650A25635265736574002900A2
:103B4000506C65617365206C6F61642066696C619F
:103B50006D656E742066697273742E002A00536559
:103B60006C6563742066696C616D656E743A002BD8
:103B70000043616E63656C002C0052756E6E696E59
:103B8000672057697A6172642077696C6C2064657C
:103B90006C6574652063757272656E742063616C08
:103BA0006962726174696F6E20726573756C74738B
:103BB00020616E642073746172742066726F6D2070
:103BC00074686520626567696E6E696E672E002D88
:103BD0000050726568656174696E67206E6F7A7AED
:103BE0006C652E20506C6561736520776169742E59
:103BF000002E00506C6561736520696E7365727488
:103C00002066696C616D656E7420696E746F2074D6
:103C100068652065787472756465722C20746865B7
:103C20006E20707265737320746865206B6E6F62AE
:103C300020746F206C6F61642069742E002F005017
:103C40006C6561736520696E736572742066696C5A
:103C5000616D656E7420696E746F2074686520668E
:103C6000697273742074756265206F66207468656C
:103C7000204D4D552C207468656E207072657373ED
:103C800020746865206B6E6F6220746F206C6F61AA
:103C9000642069742E003000546865207072696E6B
:103CA0007465722077696C6C207374617274207013
:103CB00072696E74696E672061207A69672D7A6116
:103CC00067206C696E652E20526F74617465207474
:103CD0006865206B6E6F6220756E74696C20796FF9
:103CE0007520726561636820746865206F707469FF
:103CF0006D616C206865696768742E204368656330
:103D00006B207468652070696374757265732069CF
:103D10006E207468652068616E64626F6F6B202826
:103D200043616C6962726174696F6E20636861706F
:103D3000746572292E00310053656C6563742074BC
:103D4000656D706572617475726520776869636806
:103D5000206D61746368657320796F7572206D6181
:103D600074657269616C2E00320053656C65637412
:103D700020612066696C616D656E7420666F7220CB
:103D8000746865204669727374204C61796572208D
:103D900043616C6962726174696F6E20616E642048
:103DA00073656C65637420697420696E207468653E
:103DB000206F6E2D73637265656E206D656E752E56
:103DC0000033004E6F7720492077696C6C20636167
:103DD0006C6962726174652064697374616E636595
:103DE000206265747765656E20746970206F662047
:103DF000746865206E6F7A7A6C6520616E642068E5
:103E000065617462656420737572666163652E0016
:103E100034005A2063616C6962726174696F6E204C
:103E20007265636F6D6D656E6465642E2052756E8C
:103E3000206974206E6F773F003500506C656173A8
:103E4000652072656D6F766520737465656C20738F
:103E5000686565742066726F6D206865617462655F
:103E6000642E003600497320737465656C20736896
:103E7000656574206F6E20686561746265643F00DB
:103E80003700506C6561736520636865636B206FF4
:103E900075722068616E64626F6F6B20616E642062
:103EA000666978207468652070726F626C656D2E2B
:103EB000205468656E20726573756D652074686541
:103EC0002057697A617264206279207265626F6F2F
:103ED00074696E6720746865207072696E746572AB
:103EE0002E003800416C6C20697320646F6E652E63
:103EF000204861707079207072696E74696E6721F4
:103F0000003900596F752063616E20616C776179AB
:103F10007320726573756D65207468652057697AC2
:103F20006172642066726F6D2043616C69627261B8
:103F300074696F6E202D3E2057697A6172642E007D
:103F40003A00496620796F75206861766520616462
:103F5000646974696F6E616C20737465656C20733D
:103F600068656574732C2063616C69627261746545
:103F70002074686569722070726573657473206956
:103F80006E2053657474696E6773202D2048572026
:103F90005365747570202D20537465656C207368AB
:103FA000656574732E003B00506C6561736520631A
:103FB0006C65616E206865617462656420616E6421
:103FC000207468656E207072657373207468652054
:103FD0006B6E6F622E003C00446F20796F75207706
:103FE000616E7420746F20726570656174206C61FD
:103FF0007374207374657020746F20726561646AD5
:104000007573742064697374616E6365206265748E
:104010007765656E206E6F7A7A6C6520616E6420BC
:10402000686561746265643F003D0053656C65635B
:1040300074206E6F7A7A6C65207072656865617441
:104040002074656D7065726174757265207768693A
:104050006368206D61746368657320796F75722081
:104060006D6174657269616C2E003E004973206653
:10407000696C616D656E74206C6F616465643F008E
:104080003F00546865726D616C206D6F64656C20D3
:1040900063616C2E2074616B657320617070726F48
:1040A000782E203132206D696E732E205365650A9B
:1040B00070727573612E696F2F746D2D63616C0062
:1040C00040004E6F7720492077696C6C20707265D4
:1040D00068656174206E6F7A7A6C6520666F7220F5
:1040E000504C412E004100492077696C6C2072755C
:1040F0006E207A2063616C6962726174696F6E20F0
:104100006E6F772E0042004E6F772072656D6F766E
:1041100065207468652074657374207072696E74AC
:104120002066726F6D20737465656C2073686565B9
:10413000742E004300506C656173652072656D6F6D
:104140007665207368697070696E672068656C7049
:104150006572732066697273742E0044004920777B
:10416000696C6C2072756E2078797A2063616C6955
:1041700062726174696F6E206E6F772E20497420B1
:1041800077696C6C2074616B6520757020746F208A
:104190003234206D696E732E004500466972737467
:1041A0002C20492077696C6C2072756E20746865CC
:1041B0002073656C667465737420746F2063686522
:1041C000636B206D6F737420636F6D6D6F6E206114
:1041D0007373656D626C792070726F626C656D735C
:1041E0002E00460048692C204920616D20796F75AA
:1041F00072204F726967696E616C205072757361CD
:10420000206933207072696E7465722E20576F7545
:104210006C6420796F75206C696B65206D65207406
:104220006F20677569646520796F75207468726F97
:104230007567682074686520736574757020707286
:104240006F636573733F00470048692C2049206104
:104250006D20796F7572204F726967696E616C208D
:104260005072757361206933207072696E74657263
:104270002E20492077696C6C206775696465207908
:104280006F75207468726F75676820612073686F3E
:1042900072742073657475702070726F63657373C8
:1042A0002C20696E20776869636820746865205ADD
:1042B0002D617869732077696C6C20626520636179
:1042C0006C696272617465642E205468656E2C207E
:1042D000796F752077696C6C206265207265616406
:1042E0007920746F207072696E742E004800452D1D
:1042F000636F72726563740049005A2D636F727246
:10430000656374004A00592D636F727265637400AF
:104310004B00582D636F7272656374004C005061DE
:10432000757365004D00465320416374696F6E00DC
:104330004E00436F6E742E004F00462E206A616D52
:1043400020646574656374005000462E20617574A6
:104350006F6C6F6164005100462E2072756E6F7530
:10436000740052004D4D55204D6F6465005300435D
:104370007574746572005400537465616C746800E0
:1043800055004372617368206465742E00560046C0
:10439000616E207370656564005700426564005863
:1043A0000046616E7320636865636B0059004D6F52
:1043B00064656C005A004E6F7A7A6C65005B005041
:1043C0006C6561736520756E6C6F616420746865DF
:1043D0002066696C616D656E742066697273742CF9
:1043E000207468656E2072657065617420746869F8
:1043F0007320616374696F6E2E005C0043686563AF
:104400006B73005D004E6F7A7A6C65206368616E35
:104410006765005E00416C706861626574005F00F2
:10442000536F727400600054696D650061004E6FD7
:10443000726D616C006200534420636172640063BA
:104440000053656C656374206C616E6775616765A8
:1044500000640052506920706F72740065004C69EE
:104460006E2E20636F7272656374696F6E006600F2
:1044700048572053657475700067004C6F6164691C
:104480006E67205465737400680044697361626CE0
:10449000652073746570706572730069004D6F7686
:1044A000652061786973006A0054656D706572619A
:1044B00074757265006B0050494E44412063616C15
:1044C0002E006C0052657365742058595A20636140
:1044D0006C6962722E006D005049442063616C6902
:1044E00062726174696F6E006E00426564206C6573
:1044F00076656C20636F7272656374006F004D6542
:10450000736820426564204C6576656C696E67004F
:10451000700043616C696272617465205A007100B9
:1045200043616C6962726174652058595A00720067
:1045300053656C667465737400730042656C742017
:104540007465737400740057697A61726400750051
:1045500054657374696E672066696C616D656E740D
:104560000076004C6F616420416C6C007700506CE9
:10457000656173652070756C6C206F757420666959
:104580006C616D656E7420696D6D656469617465DB
:104590006C79007800526573657400790052656E1D
:1045A000616D65007A004669727374206C6179658B
:1045B000722063616C2E007B0053656C6563740030
:1045C0007C00537465656C20736865657473007D49
:1045D00000537570706F7274007E004661696C20C4
:1045E0007374617473204D4D55007F004661696C92
:1045F0002073746174730080005374617469737400
:1046000069637300810043616C6962726174696FF0
:104610006E0082004175746F4C6F61642066696C36
:10462000616D656E740083004C6F61642066696C17
:10463000616D656E74008400556E6C6F61642066F8
:10464000696C616D656E740085004C6F61642074E7
:104650006F206E6F7A7A6C650086005072656C6FA1
:10466000616420746F204D4D550087004E6F7A7A3B
:104670006C6520642E0088004E6F205344206361D7
:1046800072640089005072696E742066726F6D20CA
:104690005344008A00436C65617220544D2065725A
:1046A000726F72008B00526573756D652070726950
:1046B0006E74008C005061757365207072696E7441
:1046C000008D00536574205265616479008E00533B
:1046D0006574206E6F74205265616479008F00509C
:1046E00072656865617400900054756E6500910094
:1046F0004C6976652061646A757374205A00920073
:1047000052657072696E74009300496E666F207313
:10471000637265656E0094004272696768746E65C5
:104720007373009500417373697374009600536945
:104730006C656E740097004F6E6365009800536F50
:10474000756E640099004C6F7564009A0046696C40
:104750002E2073656E736F72009B004368616E67F5
:10476000652066696C616D656E74009C00466C6FB7
:1047700077009D005370656564009E004D61676E13
:1047800065747320636F6D702E009F004E2F410083
:10479000A0005A2D70726F6265206E722E00A1000B
:1047A0004D65736800A20054696D656F757400A350
:1047B000004D6F646500A4004175746F00A500444E
:1047C000696D00A60042726967687400A7004C65B5
:1047D00076656C2044696D6D656400A8004C657653
:1047E000656C2042726967687400A900536574742F
:1047F000696E677300AA0059657300AB004E6F00C5
:10480000AC0053746F70207072696E7400AD004319
:104810006865636B696E672066696C6500AE00460B
:10482000696C6520696E636F6D706C6574652E00D0
:10483000AF00845265667265736800B0004D6169AF
:104840006E00B10057616974696E6720666F7220EF
:104850006E6F7A7A6C6520616E6420626564206395
:104860006F6F6C696E6700B20053656C6674657338
:1048700074204F4B00B30053656C667465737420ED
:10488000737461727400B4005072696E7420666152
:104890006E3A00B500486F74656E642066616E3ACA
:1048A00000B60043616C6962726174696E6720686A
:1048B0006F6D6500B700416C6C20636F7272656349
:1048C0007400B800436865636B696E672073656E3A
:1048D000736F727300B900436865636B696E67201C
:1048E000686F74656E6400BA00436865636B696ED7
:1048F000672062656400BB00436865636B696E672F
:10490000205A206178697300BC00436865636B6955
:104910006E672059206178697300BD004368656344
:104920006B696E672058206178697300BE00436828
:1049300065636B696E6720656E6473746F70730076
:10494000BF00436172642072656D6F76656400C05C
:10495000004261636B00C10053747269637400C2EA
:10496000005761726E00C3004E6F6E6500C4004E4A
:104970006F7A7A6C65206368616E6765643F00C515
:10498000004E6F7A7A6C6520697320686F742120FD
:104990005761697420666F7220636F6F6C646F7704
:1049A0006E2E00C6005049442063616C2E2066695B
:1049B0006E697368656400C7005049442063616C88
:1049C0002E00C8005072696E742070617573656442
:1049D00000C9005072696E742061626F7274656400
:1049E00000CA004E6F7A7A6C65206469616D6574E7
:1049F000657220646966666572732066726F6D20E9
:104A000074686520472D636F64652E00CB004E6F80
:104A10007A7A6C65206469616D6574657220646979
:104A200066666572732066726F6D207468652047D4
:104A30002D636F64652E20506C656173652063681B
:104A400065636B207468652076616C756520696E9E
:104A50002073657474696E67732E00CC00546865AA
:104A60007265206973206E6F2066696C616D656E7A
:104A700074206C6F616465642E00CD004D4B332053
:104A80006669726D776172652064657465637465CB
:104A900064206F6E204D4B3353207072696E7465C5
:104AA0007200CE00426C61636B6F7574206F63633C
:104AB00075727265642E205265636F766572207020
:104AC00072696E743F00CF00546865726D616C202E
:104AD0006D6F64656C206E6F742063616C696272C7
:104AE00061746564207965742E00D0005468657225
:104AF00065206973207374696C6C2061206E656534
:104B00006420746F206D616B65205A2063616C694D
:104B100062726174696F6E2E20506C6561736520DE
:104B2000666F6C6C6F7720746865206D616E75615F
:104B30006C2C2063686170746572204669727374AE
:104B40002073746570732C2073656374696F6E20B5
:104B500043616C6962726174696F6E20666C6F7715
:104B60002E00D1005072696E7465722068617320E6
:104B70006E6F74206265656E2063616C696272613C
:104B8000746564207965742E20506C6561736520AE
:104B9000666F6C6C6F7720746865206D616E7561EF
:104BA0006C2C20636861707465722046697273743E
:104BB0002073746570732C2073656374696F6E2045
:104BC00043616C6962726174696F6E20666C6F77A5
:104BD0002E00D20053656C66746573742077696C1F
:104BE0006C2062652072756E20746F2063616C6941
:104BF00062726174652061636375726174652073AC
:104C0000656E736F726C657373207265686F6D6922
:104C10006E672E00D3004F6C642073657474696EE8
:104C2000677320666F756E642E2044656661756CCF
:104C300074205049442C204573746570732065744A
:104C4000632E2077696C6C206265207365742E007A
:104C5000D4005761726E696E673A20626F74682083
:104C60007072696E746572207479706520616E640B
:104C7000206D6F74686572626F6172642074797000
:104C800065206368616E6765642E00D500576172A8
:104C90006E696E673A207072696E746572207479FD
:104CA0007065206368616E6765642E00D600576189
:104CB000726E696E673A206D6F74686572626F61BB
:104CC00072642074797065206368616E6765642E14
:104CD00000D700536865657400D8005265636F762D
:104CE0006572696E67207072696E7400D9005448ED
:104CF00045524D414C20414E4F4D414C5900DA0038
:104D0000526573756D696E67207072696E7400DB31
:104D10000050494E44412048656174696E6700DC6B
:104D20000043616C6962726174696F6E20646F6EBA
:104D30006500DD0043616C6962726174696E6720B1
:104D40005A00DE0042656420646F6E6500DF004239
:104D500065642048656174696E6700E000486561BC
:104D600074696E6720646F6E652E00E100486561AE
:104D700074696E6700E2004D4D55206661696C7381
:104D800000E3004D4D55206C6F6164206661696CD5
:104D90007300E4004D4D5520706F77657220666199
:104DA000696C7300E5004D6174657269616C206324
:104DB00068616E67657300E600546F74616C20660D
:104DC00061696C7572657300E7004C6173742070E3
:104DD00072696E74206661696C7572657300E800B3
:104DE000506F776572206661696C7572657300E952
:104DF0000046696C2E2072756E6F75747300EA0040
:104E0000437261736800EB00546F74616C00EC00D6
:104E10004C617374207072696E7400ED00416D62B4
:104E200069656E7400EE00566F6C7461676573009F
:104E3000EF0054656D70657261747572657300F092
:104E40000042656C742073746174757300F10053D3
:104E5000656E736F7220696E666F00F2004578743C
:104E6000727564657220696E666F00F30058595A56
:104E70002063616C2E2064657461696C7300F400BA
:104E80005072696E74657220495020416464723AB0
:104E900000F500756E6B6E6F776E00F6004D4D5528
:104EA00020636F6E6E656374656400F7004461741F
:104EB000653A00F800746F20756E6C6F616420664F
:104EC000696C616D656E7400F900746F206C6F61C0
:104ED000642066696C616D656E7400FA00507265DD
:104EE000737320746865206B6E6F6200FB005072F4
:104EF0006568656174696E6720746F2063757400FE
:104F0000FC0050726568656174696E6720746F207B
:104F1000656A65637400FD00507265686561746957
:104F20006E6720746F20756E6C6F616400FE0050B8
:104F3000726568656174696E6720746F206C6F615B
:104F40006400FF00436F6F6C646F776E0000014672
:104F5000696C616D656E7420657874727564696ED4
:104F6000672026207769746820636F7272656374A6
:104F700020636F6C6F723F000101456A65637400C6
:104F800002014175746F6C6F6164696E67206669B8
:104F90006C616D656E7420697320616374697665F8
:104FA0002C206A7573742070726573732074686541
:104FB000206B6E6F6220616E6420696E736572741F
:104FC0002066696C616D656E742E2E2E000301548F
:104FD0006F74616C2066696C616D656E74000401AC
:104FE000546F74616C207072696E742074696D65A1
:104FF00000050146696C616D656E742075736564AA
:105000000006015072696E742074696D65000701B5
:105010005072656865617420746865206E6F7A7A75
:105020006C65210008014552524F523A000901595E
:105030002064697374616E63652066726F6D206DA4
:10504000696E000A014C656674000B01526967685D
:1050500074000C014D6561737572656420736B6536
:1050600077000D01536C6967687420736B65770076
:105070000E0153657665726520736B6577000F01CD
:105080005B303B305D20706F696E74206F666673B5
:10509000657400100141646A757374696E67205A03
:1050A000001101526561722073696465205BE46DD3
:1050B0005D00120146726F6E7420736964655BE473
:1050C0006D5D001301526967687420736964655BE4
:1050D000E46D5D0014014C6566742073696465209D
:1050E0005BE46D5D0015015365742074656D70653A
:1050F0007261747572653A00160150494E44412040
:1051000063616C6962726174696F6E206661696C5B
:10511000656400170150494E44412063616C696227
:10512000726174696F6E2069732066696E69736855
:10513000656420616E64206163746976652E204920
:10514000742063616E2062652064697361626C65BE
:105150006420696E206D656E752053657474696E88
:1051600067732D3E50494E44412063616C2E0018F8
:105170000146656564696E6720746F204653656EED
:10518000736F720019014D6F76696E672073656CDD
:105190006563746F72001A01486F6D696E67001B5A
:1051A00001526574726163742066726F6D204649A6
:1051B0004E4441001C01456A656374696E67206650
:1051C000696C616D656E74001D015061726B696E72
:1051D000672073656C6563746F72001E015265749D
:1051E00075726E696E672073656C6563746F7200AB
:1051F0001F01506572666F726D696E67206375740A
:1052000000200150757368696E672066696C616D76
:10521000656E74002101507265706172696E67205D
:10522000626C61646500220153656C656374696E2C
:10523000672066696C2E20736C6F74002301556EB5
:105240006C6F6164696E672066696C616D656E7410
:1052500000240145525220544D43206661696C651B
:10526000640025014552522048656C702066696CC7
:10527000616D656E7400260145525220496E746559
:10528000726E616C0027014552522057616974208B
:10529000666F72205573657200280146696E6973E6
:1052A00068696E67206D6F76656D656E7473002931
:1052B0000141766F6964696E67206772696E640088
:1052C0002A0146656564696E6720746F206E6F7A87
:1052D0007A6C65002B0146656564696E6720746FA2
:1052E000206578747275646572002C01466565648A
:1052F000696E6720746F2046494E4441002D015568
:105300006E6C6F6164696E6720746F2070756C6C71
:105310006579002E01556E6C6F6164696E6720744B
:105320006F2046494E4441002F01446973656E6702
:105330006167696E672069646C6572003001456E53
:10534000676167696E672069646C65720031014F3F
:105350004B003201554E4B4E4F574E204552524F47
:105360005200330146494C414D454E54204348417B
:105370004E474500340146494C414D454E54204569
:105380004A4543544544003501554E4C4F41442055
:105390004D414E55414C4C5900360146572052550F
:1053A0004E54494D45204552524F520037014D4D04
:1053B0005520465720555044415445204E454544BC
:1053C000454400380151554555452046554C4C0043
:1053D0003901494E56414C494420544F4F4C003AF4
:1053E0000146494C2E20414C5245414459204C4FD6
:1053F00041444544003B01434F4D4D554E494341C7
:1054000054494F4E204552524F52003C014D4D558C
:10541000204E4F5420524553504F4E44494E470062
:105420003D014D4D55204D4355204552524F5200A0
:105430003E014D4D552053454C465445535420464E
:1054400041494C4544003F01544D43204452495684
:1054500045522053484F52544544004001544D4357
:1054600020554E444552564F4C54414745204552D5
:1054700052004101544D4320445249564552205256
:1054800045534554004201544D432044524956452A
:1054900052204552524F52004301544D43204F5623
:1054A000455248454154204552524F5200440157FD
:1054B00041524E494E4720544D4320544F4F2048AF
:1054C0004F5400450149444C45522043414E4E4FF4
:1054D00054204D4F564500460149444C4552204307
:1054E000414E4E4F5420484F4D4500470153454CC7
:1054F0004543544F522043414E4E4F54204D4F563A
:105500004500480153454C4543544F522043414EBA
:105510004E4F5420484F4D450049014C4F414420C7
:10552000544F20455854522E204641494C45440082
:105530004A01494E53504543542046494E44410088
:105540004B014653454E534F5220544F4F20454137
:10555000524C59004C0150554C4C45592043414E3A
:105560004E4F54204D4F5645004D014653454E5326
:105570004F522046494C2E20535455434B004E0168
:105580004653454E534F52204449444E54205452A2
:105590004947472E004F0146494E44412046494C59
:1055A000414D2E20535455434B00500146494E4423
:1055B00041204449444E54205452494747455200E3
:1055C00051014E6F74207370696E6E696E67005280
:1055D000015370696E6E696E6700530146616E20FB
:1055E0007465737400540153656C6674657374203C
:1055F0006661696C656400550146696C616D656E34
:10560000742073656E736F7200560153776170700A
:10561000656400570146726F6E742F6C6566742066
:1056200066616E73005801417869730059014178D1
:105630006973206C656E677468005A014C6F6F73F4
:10564000652070756C6C6579005B014C6566742033
:10565000686F74656E642066616E3F005C0146721F
:105660006F6E74207072696E742066616E3F005DAB
:1056700001456E6473746F70206E6F742068697476
:10568000005E01456E6473746F70005F014D6F744E
:105690006F72006001456E6473746F707300610116
:1056A000576972696E67206572726F72006201429B
:1056B00065642F4865617465720063014E6F7420E4
:1056C000636F6E6E65637465640064014865617440
:1056D00065722F546865726D6973746F720065012D
:1056E000506C6561736520636865636B3A006601A1
:1056F00053656C6674657374206572726F722100F5
:10570000670158595A2063616C6962726174696FEC
:105710006E20616C6C2072696768742E20536B6513
:10572000772077696C6C20626520636F72726563A5
:10573000746564206175746F6D61746963616C6C0C
:10574000792E00680158595A2063616C6962726150
:1057500074696F6E20616C6C2072696768742E20AA
:10576000582F5920617865732061726520736C69C8
:105770006768746C7920736B657765642E20476F5A
:105780006F64206A6F622100690158595A20636171
:105790006C6962726174696F6E206F6B2E20582F76
:1057A000592061786573206172652070657270653B
:1057B0006E646963756C61722E20436F6E677261EF
:1057C00074756C6174696F6E7321006A0158595A5F
:1057D0002063616C6962726174696F6E20636F6DC2
:1057E00070726F6D697365642E20526967687420EA
:1057F00066726F6E742063616C6962726174696F46
:105800006E20706F696E74206E6F742072656163B4
:105810006861626C652E006B0158595A2063616C97
:105820006962726174696F6E20636F6D70726F6D03
:10583000697365642E2046726F6E742063616C69B3
:1058400062726174696F6E20706F696E7473206E1E
:105850006F7420726561636861626C652E006C0113
:1058600058595A2063616C6962726174696F6E2065
:105870006661696C65642E2052696768742066727F
:105880006F6E742063616C6962726174696F6E20FF
:10589000706F696E74206E6F7420726561636861E9
:1058A000626C652E006D0158595A2063616C696203
:1058B000726174696F6E206661696C65642E204642
:1058C000726F6E742063616C6962726174696F6E6D
:1058D00020706F696E7473206E6F742072656163DF
:1058E0006861626C652E006E0158595A2063616CC4
:1058F0006962726174696F6E206661696C65642E9D
:1059000020506C6561736520636F6E73756C7420D5
:10591000746865206D616E75616C2E006F01585959
:105920005A2063616C6962726174696F6E2066618E
:10593000696C65642E204265642063616C696272E3
:105940006174696F6E20706F696E74207761732067
:105950006E6F7420666F756E642E007001506C65FA
:1059600061736520706C61636520737465656C207C
:105970007368656574206F6E206865617462656424
:105980002E00710144697374616E636520626574F1
:105990007765656E20746970206F66207468652075
:1059A0006E6F7A7A6C6520616E642074686520621F
:1059B0006564207375726661636520686173206E2B
:1059C0006F74206265656E20736574207965742E2E
:1059D00020506C6561736520666F6C6C6F77207406
:1059E0006865206D616E75616C2C206368617074F0
:1059F00065722046697273742073746570732C200D
:105A000073656374696F6E204669727374206C618C
:105A10007965722063616C6962726174696F6E2E60
:105A2000007201506C616365206120736865657464
:105A3000206F6620706170657220756E64657220DB
:105A4000746865206E6F7A7A6C6520647572696E11
:105A500067207468652063616C6962726174696F44
:105A60006E206F66206669727374203420706F69CF
:105A70006E74732E20496620746865206E6F7A7A82
:105A80006C65206361746368657320746865207059
:105A9000617065722C20706F776572206F6666206A
:105AA000746865207072696E74657220696D6D65C9
:105AB00064696174656C792E00730153656172636A
:105AC00068696E67206265642063616C69627261F7
:105AD00074696F6E20706F696E740074014D65613A
:105AE000737572696E67207265666572656E63654F
:105AF00020686569676874206F662063616C6962FD
:105B0000726174696F6E20706F696E7400750150F8
:105B10006C6561736520636C65616E2074686520D7
:105B20006E6F7A7A6C6520666F722063616C696251
:105B3000726174696F6E2E20436C69636B207768A5
:105B4000656E20646F6E652E0076014175746F205E
:105B5000686F6D650077014375742066696C616DCF
:105B6000656E74007801456A6563742066726F6DB6
:105B7000204D4D550079014C6F6164696E67206658
:105B8000696C616D656E74007A014D4D55205265EA
:105B90007472793A20526573746F72696E672074FB
:105BA000656D70657261747572652E2E2E007B01B5
:105BB000536F7274696E672066696C6573007C014F
:105BC000536F6D652066696C65732077696C6C2016
:105BD0006E6F7420626520736F727465642E204D41
:105BE00061782E204E6F2E206F662066696C65737B
:105BF00020696E203120666F6C64657220666F725A
:105C000020736F7274696E67206973203130302E93
:105C1000007D014F6666007E014F6E007F01556E6C
:105C20006578706563746564206572726F72206F49
:105C3000636375727265642E0080014D36303020CA
:105C400046696C616D656E74204368616E67652E90
:105C5000204C6F61642061206E65772066696C61FD
:105C60006D656E74206F7220656A65637420746858
:105C700065206F6C64206F6E652E00810152656D2A
:105C80006F76652074686520656A65637465642055
:105C900066696C616D656E742066726F6D207468E4
:105CA000652066726F6E74206F6620746865204D83
:105CB0004D552E00820146696C616D656E742064DD
:105CC0006574656374656420756E6578706563746A
:105CD00065646C792E20456E73757265206E6F2039
:105CE00066696C616D656E74206973206C6F6164A8
:105CF00065642E20436865636B2074686520736556
:105D00006E736F727320616E6420776972696E675B
:105D10002E008301496E7465726E616C2072756E1F
:105D200074696D65206572726F722E2054727920CD
:105D3000726573657474696E6720746865204D4D73
:105D400055206F72207570646174696E6720746885
:105D500065206669726D776172652E0084014D4D14
:105D6000552046572076657273696F6E20697320DF
:105D7000696E636F6D70617469626C6520776974B8
:105D800068207072696E7465722046572E55706473
:105D900061746520746F2076657273696F6E20334D
:105DA0002E302E332E0085014D4D55204669726DE3
:105DB0007761726520696E7465726E616C206572C0
:105DC000726F722C20706C656173652072657365EB
:105DD0007420746865204D4D552E00860152657102
:105DE0007565737465642066696C616D656E742099
:105DF000746F6F6C206973206E6F742061766169B7
:105E00006C61626C65206F6E2074686973206861D4
:105E10007264776172652E20436865636B207468D5
:105E20006520472D636F646520666F7220746F6F05
:105E30006C20696E646578206F7574206F662072BF
:105E4000616E6765202854302D5434292E00870157
:105E500043616E6E6F7420706572666F726D207430
:105E6000686520616374696F6E2C2066696C616D72
:105E7000656E7420697320616C7265616479206C51
:105E80006F616465642E20556E6C6F616420697467
:105E90002066697273742E0088014D4D55206E6F17
:105EA0007420726573706F6E64696E6720636F72C1
:105EB000726563746C792E20436865636B20746827
:105EC0006520776972696E6720616E6420636F6E0A
:105ED0006E6563746F72732E0089014D4D55206E8F
:105EE0006F7420726573706F6E64696E672E2043E5
:105EF0006865636B2074686520776972696E6720D6
:105F0000616E6420636F6E6E6563746F72732E00D2
:105F10008A014D6F72652064657461696C73206FCE
:105F20006E6C696E652E008B015468652049646C47
:105F300065722063616E6E6F7420686F6D6520708E
:105F4000726F7065726C792E20436865636B206692
:105F50006F7220616E797468696E6720626C6F631E
:105F60006B696E6720697473206D6F76656D656E01
:105F7000742E008C0143616E2774206D6F7665204E
:105F800053656C6563746F72206F722049646C6531
:105F9000722E008D015468652053656C6563746FC3
:105FA000722063616E6E6F7420686F6D6520707211
:105FB0006F7065726C792E20436865636B20666F25
:105FC0007220616E797468696E6720626C6F636BB2
:105FD000696E6720697473206D6F76656D656E7488
:105FE0002E008E014C6F6164696E6720746F2065AE
:105FF00078747275646572206661696C65642E20C0
:10600000496E7370656374207468652066696C619D
:106010006D656E74207469702073686170652E20E0
:10602000526566696E65207468652073656E736F6E
:10603000722063616C6962726174696F6E2C206991
:1060400066206E65656465642E008F0153656C651E
:1060500063746F722063616E2774206D6F766520A4
:1060600064756520746F2046494E44412064657410
:10607000656374696E6720612066696C616D656E29
:10608000742E204D616B652073757265206E6F20D4
:1060900066696C616D656E7420697320696E20534A
:1060A000656C6563746F7220616E642046494E446E
:1060B0004120776F726B732070726F7065726C79AC
:1060C0002E00900146696C616D656E742073656E7B
:1060D000736F722074726967676572656420746F8C
:1060E0006F206561726C79207768696C65206C6FD0
:1060F0006164696E6720746F206578747275646579
:10610000722E20436865636B207468657265206930
:10611000736E277420616E797468696E672073747A
:1061200075636B20696E2050544645207475626516
:106130002E20436865636B20746861742073656EFC
:10614000736F722072656164732070726F70657214
:106150006C792E00910150756C6C6579206D6F74AF
:106160006F72207374616C6C65642E20456E73755C
:106170007265207468652070756C6C657920636148
:106180006E206D6F766520616E6420636865636B59
:106190002074686520776972696E672E00920146E7
:1061A000696C616D656E742073656E736F722064C7
:1061B00069646E277420737769746368206F6666FC
:1061C000207768696C6520756E6C6F6164696E67B5
:1061D0002066696C616D656E742E20456E737572F4
:1061E000652066696C616D656E742063616E206DFB
:1061F0006F766520616E64207468652073656E73C8
:106200006F7220776F726B732E00930146696C6119
:106210006D656E742073656E736F72206469646E51
:1062200027742074726967676572207768696C6586
:10623000206C6F6164696E67207468652066696CA4
:10624000616D656E742E20456E737572652074687D
:10625000652073656E736F722069732063616C696A
:1062600062726174656420616E6420746865206682
:10627000696C616D656E7420726561636865642028
:1062800069742E00940146494E4441206469646E4D
:10629000277420737769746368206F666620776857
:1062A000696C6520756E6C6F6164696E67206669E4
:1062B0006C616D656E742E2054727920756E6C6FF2
:1062C0006164696E67206D616E75616C6C792E20FA
:1062D000456E737572652066696C616D656E7420BC
:1062E00063616E206D6F766520616E642046494E55
:1062F000444120776F726B732E00950146494E44DE
:1063000041206469646E27742074726967676572DE
:10631000207768696C65206C6F6164696E672074B2
:1063200068652066696C616D656E742E20456E73BC
:10633000757265207468652066696C616D656E7440
:106340002063616E206D6F766520616E6420464922
:106350004E444120776F726B732E0096014469732F
:1063600061626C6500970153746F700098014C6F07
:106370006164009901556E6C6F6164009A01526509
:106380007365744D4D55009B015265747279009C84
:1063900001426564206C6576656C696E6720666194
:1063A000696C65642E2053656E736F722064696436
:1063B0006E277420747269676765722E2044656267
:1063C000726973206F6E206E6F7A7A6C653F20570A
:1063D000616974696E6720666F7220726573657497
:1063E0002E009D0153656E73697469766974790036
:1063F0009E01446F6E6500656E717565696E6720FC
:106400002200446F6E65207072696E74696E672039
:1064100066696C65004E6F204C696E65204E756D27
:10642000626572207769746820636865636B737551
:106430006D2C204C617374204C696E653A20004EBF
:106440006F20436865636B73756D2077697468208E
:106450006C696E65206E756D6265722C204C61737F
:1064600074204C696E653A2000636865636B7375D0
:106470006D206D69736D617463682C204C61737459
:10648000204C696E653A20004C696E65204E756D32
:10649000626572206973206E6F74204C6173742082
:1064A0004C696E65204E756D6265722B312C204CE7
:1064B000617374204C696E653A2000256C7520620A
:1064C00079746573207772697474656E20746F20B7
:1064D0002553206174206164647265737320307881
:1064E0002530346C780A00442564202D20526561E3
:1064F000642F57726974652025530A003F3F00528C
:106500006F6D616E61004872766174736B69004DE6
:10651000616779617200536C6F76656E63696E6155
:10652000004E6F72736B005376656E736B61004E35
:10653000656465726C616E647300506F6C736B6937
:10654000004974616C69616E6F004672616E6361CF
:10655000697300457370616E6F6C00446575747388
:1065600063680043657374696E6100456E676C69AA
:1065700073680020436F756E7420583A20004530D0
:106580003A25642052504D2050524E313A25642015
:1065900052504D204530403A25752050524E3140E2
:1065A0003A25750A00526573656E640025533A20DA
:1065B000256C640A25530A002F2F616374696F6E7E
:1065C0003A6E6F74696669636174696F6E202553F2
:1065D0000A0046696C616D656E742072756E6F7528
:1065E0007420646574656374656421005072696E1B
:1065F0007465722073746F707065642064756520B3
:10660000746F206572726F72732E2053757065728D
:10661000766973696F6E2072657175697265642E33
:106620000064756D7020636C65617265640A006E4C
:106630006F2064756D7020617661696C61626C6554
:106640000A00443231202D2072656164206372613A
:1066500073682064756D700A006E6F2064756D70CC
:1066600020617661696C61626C650A0064756D70A9
:1066700020636F6D706C6574656420696E20256C95
:10668000756D730A0058464C4153480045455052B9
:106690004F4D005352414D00442D31202D20456E69
:1066A000646C657373206C6F6F700A00416374696A
:1066B00076652045787472756465723A20300049B9
:1066C0006E76616C696420657874727564657200B9
:1066D000746D63323133305F7072696E745F6375ED
:1066E0007272656E747328290A094809520A58099A
:1066F00025640925640A590925640925640A5A098B
:1067000025640925640A450925640925640A00539E
:1067100044207072696E74696E67206279746520B6
:1067200000556E6B6E6F776E20636F6D6D616E647A
:106730003A2022004D32303020496E76616C696417
:1067400020657874727564657220007A5F6D617877
:106750003A20007A5F6D696E3A2000795F6D61784A
:106760003A2000795F6D696E3A2000785F6D61783C
:106770003A2000545249474745524544006F7065DE
:106780006E00785F6D696E3A20005265706F7274AA
:10679000696E6720656E6473746F702073746174C2
:1067A0007573004D3131322063616C6C65642E204D
:1067B000456D657267656E63792053746F702E0046
:1067C0002F2F616374696F6E3A75766C6F5F7265B7
:1067D000636F766572795F7265616479002F2F61EE
:1067E0006374696F6E3A75766C6F5F6175746F5F15
:1067F0007265636F766572795F7265616479002591
:10680000533A256C7520636D0A25533A256C752023
:106810006D696E0A0053494C454E54004E4F524D1F
:10682000414C002553204D4F44453A20506572633A
:10683000656E7420646F6E653A20256868643B203D
:106840007072696E742074696D652072656D61691E
:106850006E696E6720696E206D696E733A202564DB
:106860003B204368616E676520696E206D696E73B9
:106870003A2025640A005072696E7465725374611F
:1068800074653A2025640A00456E642066696C656B
:10689000206C69737400426567696E2066696C6577
:1068A000206C69737400556E6B6E6F776E20256374
:1068B00020636F64653A2025730A000A50494E44EC
:1068C000412074656D70657261747572653A20253A
:1068D0002E3166205A20736869667420286D6D29F0
:1068E0003A20252E3366000A537465703A202564D9
:1068F0002F360A000A537465703A2025642F36201B
:1069000028736B6970706564290A50494E444120B0
:1069100074656D70657261747572653A20256420C6
:106920005A20736869667420286D6D293A300A0010
:106930000A5A45524F3A20252E33660A0073746175
:1069400072742074656D70657261747572653A2039
:10695000252E31660A0025642020252E326600256A
:106960005320583A20252E356620593A20252E35B9
:1069700066205A3A20252E35660A00536C656570EC
:106980002E2E2E0045303A25642052504D0A50528A
:106990004E303A25642052504D0A00473930004DA0
:1069A00031303700423A20253364202020202058FF
:1069B000643A2536640A533A202533642020202087
:1069C0002059643A2536640046494E4441005049F6
:1069D0004E44410057697A61726420656E64207389
:1069E000746174653A2025640A0053706F6F6C4AB5
:1069F0006F696E004669726D776172650048426525
:106A000064206F6E206C6F616400466C6173684136
:106A1000697200546865726D616C204D6F64656CBD
:106A20002063616C2E004572723A5052494E5420D8
:106A300046414E204552524F52004572723A484FDD
:106A400054454E442046414E204552524F52002F4D
:106A50002F616374696F6E3A726573756D6564005A
:106A60002F2F616374696F6E3A726573756D65007F
:106A70002F2F616374696F6E3A7265616479002FBC
:106A80002F616374696F6E3A6E6F745F72656164D3
:106A900079002F2F616374696F6E3A63616E63656D
:106AA0006C004D38340041786973206C656E6774F2
:106AB0006820646966666572656E63653A252E3383
:106AC000660A004D6561737572656420617869734B
:106AD000206C656E6774683A252E33660A004F4B4A
:106AE000004C434420737461747573206368616E55
:106AF00067656400534420636172642072656C654D
:106B0000617365640046616B652073657269616CD1
:106B1000206E756D62657200452D636F6F6C206D20
:106B20006F6465002F2F616374696F6E3A737461CF
:106B3000727400473931004D373032004D38330020
:106B40004732382057004D35303000457874657233
:106B50006E616C2053504920666C6173680A584618
:106B60004C415348206973206E6F74207265732DF9
:106B70000A706F6E64696E672E204C616E67756176
:106B800067650A73776974636820756E61766169F9
:106B90006C61626C652E0058464C415348206E6F04
:106BA0007420726573706F6E64696E672E0046574D
:106BB0002063726173682064657465637465642121
:106BC00020596F752063616E20636F6E74696E75F6
:106BD00065207072696E74696E672E2044656275F7
:106BE00067206461746120617661696C61626C65C3
:106BF00020666F7220616E616C797369732E204319
:106C00006F6E7461637420737570706F727420742A
:106C10006F207375626D69742064657461696C734B
:106C20002E002F2F616374696F6E3A64756D705F0B
:106C3000617661696C61626C65004372617368447E
:106C400065746563742044495341424C4544004394
:106C50007261736844657465637420454E41424CAB
:106C6000454421002020506C616E6E65724275664D
:106C700066657242797465733A20002046726565D4
:106C8000204D656D6F72793A2000207C204175742B
:106C9000686F723A2000204C6173742055706461F3
:106CA0007465643A200020536F66747761726520C2
:106CB000526573657400205761746368646F672060
:106CC0005265736574002042726F776E206F757421
:106CD000205265736574002045787465726E616C2E
:106CE00020526573657400506F776572557000654A
:106CF00072726F722077726974696E6720746F2088
:106D000066696C6500446F6E6520736176696E67B5
:106D10002066696C652E006F6B0046696C616D655D
:106D20006E7400504F5745522050414E4943204405
:106D3000455445435445440055564C4F202D20653D
:106D40006E642025640A0055564C4F5F54494E59D5
:106D5000202D20656E642025640A00776F726C64B4
:106D600020636F6F7264696E617465733A202825C1
:106D70002E33662C20252E33662C20252E336629B3
:106D80000A004D3232302053256400446F6E652076
:106D900072656164696E6720454550524F4D0A0027
:106DA00054656D7065726174757265205265737497
:106DB0006F7265640A0047312045252D2E33662009
:106DC000463237303000544D4320445249564552E4
:106DD000204F56455254454D5000486F6C64206317
:106DE000757272656E74207472756E636174656419
:106DF00020746F2052756E2063757272656E740018
:106E000025632533642F256481005A25362E32668A
:106E10002563005A2020202D2D2D20008625336447
:106E20002525002D2D2D2525002533642525002021
:106E30005344002020200020484F008725337568E8
:106E400020256325630087253032753A2530327559
:106E500025632563002F2F616374696F6E3A70613B
:106E600075736564002F2F616374696F6E3A70618A
:106E70007573650044756D70206D656D6F72790076
:106E800068656C702E707275736133642E636F6DFC
:106E900000666F72756D2E707275736133642E6348
:106EA0006F6D00707275736133642E636F6D004D8A
:106EB0003730310025533A0A2531382E32666D209D
:106EC0000A25533A0A2531306C6464202530326437
:106ED0006820253032646D0025533A0A2531382E5A
:106EE00032666D200A25533A0A2531306C646820D9
:106EF000253032646D2025303264730025362E3201
:106F0000666D6D0025530A25530A25533A0A255309
:106F10003A0025332E32668100252D31342E31344E
:106F2000533A0A25530A252D31342E3134533A254C
:106F3000332E3266810A252D31342E3134533A25D1
:106F4000332E3266810020203000202031004D6534
:106F500061737572656420736B6577733A2025667B
:106F60002025660A0046697474696E672066616947
:106F70006C6564203D3E2063616C69627261746976
:106F80006F6E206661696C65642E0A0043616C69EE
:106F900062726174696F6E20737563636573732EBB
:106FA0000A00416C6C20342063616C696272617408
:106FB000696F6E20706F696E747320666F756E6492
:106FC0002E0A00312F3400312F3400312F39005078
:106FD00072757361206933204D4B332D52204F4B16
:106FE0002E0053442063617264206F6B006F7065E4
:106FF0006E526F6F74206661696C656400766F6CA9
:10700000756D652E696E6974206661696C656400D2
:10701000534420696E6974206661696C006F706505
:107020006E206661696C65642C2046696C653A2047
:107030000043616E6E6F7420656E746572207375A7
:10704000626469723A20004D363030004D323400AF
:107050004D323320257300312F3900880020746FA2
:107060006F206C6F6E6720657874727573696F6ED0
:107070002070726576656E7465640020636F6C6461
:1070800020657874727573696F6E207072657665AD
:107090006E746564004D6F76652061626F72746511
:1070A0006400084AD73B3BCE016E84BCBFFDC12FB4
:1070B0003D6C74319ABD56833DDA3D00C77F11BEE9
:1070C000D9E4BB4C3E916BAAAABE000000803F05EC
:1070D000A84CCDB2D44EB93836A9020C50B991861D
:1070E00088083CA6AAAA2ABE000000803F07634287
:1070F00036B79BD8A71A39685618AEBAAB558C1D4F
:107100003CB7CC5763BD6DEDFD753EF6177231BFD0
:10711000000000803F08000000BE922449123EABF0
:10712000AAAA2ABECDCCCC4C3E00000080BEABAAA1
:10713000AAAA3E00000000BF000000803F0000003F
:107140000000084178D3BB4387D1133D190E3CC3DF
:10715000BD4282AD2B3E68EC8276BED98FE1A93E5E
:107160004C80EFFFBE01C4FF7F3F00000000000025
:107170000C948AEF0C9422FB0C9471EA0D94C808CD
:107180000D94621D0C9453E20C94ACE00D94D1224A
:107190000C947BCF0C949EEA0C9436740C94F6F00D
:1071A0000C94E1E00C9499D20C94EDD00D9426A7A8
:1071B0000C94CBF50D948D0A0C94B6D50D94C4198E
:1071C0000C94C6EA0C9408F10C9494D10C94A8EA9F
:1071D0000C944DFB0C94AFE30D94352C0C9413746C
:1071E0000C94E0CD0D943E510C946BFA0D943AAD95
:1071F0000C9473700C946BDA0C94AECE0C94D8CDC6
:107200000D946FA00D94910A0D9448170D944F1989
:107210000C94DAD00D9427520C94A3D40D9472528E
:107220000C94F4CD0C941BFA0C946DDC0C9486D465
:107230000C94B3CD0D9472A00C943FE20C94A8CEA4
:107240000C9429EF0C94E1FA0C94E6E20C94D2CD64
:107250000D94912C0C94B2EA0C94CECD0C94AEE229
:107260000C949CD00D94591D0D9405180D9429A7CC
:107270000D94DA3F0C9443EA0C94EDFA0C9494EAE2
:107280000C9434EA0C9485EA0C94B9E10C949FD4E4
:107290000C94DCCD0D949B210D94CE080C94E375D9
:1072A0000C9457EA0C94BCEA0C9495D40D9406A067
:1072B0000D9460170C94ADF80C94C5CD0D942B1A59
:1072C0000C9468D00D94C1510C948DD10C94AAE10A
:1072D0000C9481D40C944BDA0D944F110C9406D875
:1072E0000C9407FB0C9405E40D94C42C0C9425D548
:1072F0000C9453F50D94ED510D942CA70D949C0C0A
:107300000C946DE20C945EE20D94051B0D949E1599
:107310000C94BFF00C9449D00D9409AD0D94220B40
:107320000C94A4E10D9475A00C94E1D40C944DEA56
:107330000C94A1E10C942ED50D94D1180D945651B6
:107340000C94A7FA0C940A740D9465170D9428AD4B
:107350000D9462520D946A520C942FDB0C941BD046
:107360000C94F8CD0D947A520C9482CF0D9454174E
:107370000D945A520C9472D00D9448220C94C3D0A0
:107380000D9454100C947CD00D942A520C940EE061
:107390000D94EA0F0D94C7A60D94A2150C9414E059
:1073A0000C94E6730C94B9CD0D9432520D94790B74
:1073B0000C9418FB0D94B3170D94BED40D94471D77
:1073C0000C9489CF0C9479D90D94482C0D942019E4
:1073D0000C94E3CF0D9425AD0C94C1CD0C94CCE46A
:1073E0000C94A6D00C949DFA0C9488D00D948C1F0C
:1073F0000D9432300D9480160D9485510C944CF1FF
:107400000C94B8D00D9490A00C942CEA0D94200A02
:107410000C948BD40C94F5F80D9421520D94CC0D52
:107420000C94A7E10D94F3510C9430FB0C9447F0AD
:107430000D9424520C940FD00D9437110C942FE21C
:107440000D94AEA60C94B0D10D94D52C0D94BA40E9
:107450000C94ADE10C942ED00D94AB1F0D94E30B66
:107460000D94701A0D9435AD0D94C3AC0D944A5221
:107470000C9492D00C94C1730D941EA00D94525292
:107480000C947CD40C945ED00C9491FA0C9405CEA0
:107490000D9469100C9428E00C94DB730D943A520F
:1074A0000C9454D00C9490D40D9409A70D94FA9F89
:1074B0000C94CB760C949AD40D9484A00D9463A074
:1074C0000C944CF20C94B6E00C9448740D948851D2
:1074D0000D94F0510D942CAD0C94E6CD0C946AE112
:1074E0000D946D170C94B5E50C94F4730C9439FB62
:1074F0000D94B7D20D9442520C94F3CD0C94B0E19C
:107500000C94F5630D94CF1D0C9424F90D94501D2B
:107510000D948B280C947BEA0C945AE10C94BDCD0D
:107520000C9437E20C94C8CD0D9478A00D9470188B
:107530000C9467EA0D947E510D94810D0C943DD00E
:107540000C9439EA0C94EACD0D949D100C9468D3F8
:107550000C9400CE0D94901D0C945FEA0C941EFBCD
:107560000C946DCF0D947B510D94E70B0C9447E276
:107570000C9496CE0D94F12C0C94FCCD0C942BD342
:107580000D946A740D94BC1F0C941EE00C9474CF7F
:107590000D94BC290C94EECD0D945D2A6E616E00A5
:1075A000696E660000407A10F35A00A0724E180906
:1075B0000010A5D4E80000E87648170000E40B545A
:1075C000020000CA9A3B000000E1F5050000809629
:1075D0009800000040420F000000A086010000005B
:1075E000102700000000E803000000006400000015
:1075F00000000A00000000000100000000002C76DE
:10760000D888DC674F0823DFC1DFAE59E1B1B796F8
:10761000E5E3E453C63AE651997696E8E6C2842655
:10762000EB898C9B62ED407C6FFCEFBC9C9F40F231
:10763000BAA56FA5F490055A2AF75C936B6CF967AD
:107640006DC11BFCE0E40D47FEF520E6B500D0ED72
:10765000902E0300943577050080841E08000020DA
:107660004E0A000000C80C333333330F986E128378
:107670001141EF8D2114893BE65516CFFEE6DB184C
:10768000D1844B381BF77C1D901DA4BBE424203211
:1076900084725E228100C9F124ECA1E53D2722001D
:1076A000002045535000204E535000204F464600C6
:1076B000204F4E005056303100205B4D505D200071
:1076C000256920686F757273202569206D696E7554
:1076D0007465730052582074696D656F7574004D40
:1076E000333130004D313132004D3131300046758B
:1076F0006C6C205258204275666665720053657442
:1077000074696E67732053746F72656400544D3AE8
:107710002073746F7265642063616C696272617456
:10772000696F6E20696E76616C69642C2072657376
:10773000657474696E670053746F72656420736555
:107740007474696E677320726574726965766564B6
:107750000048617264636F646564204465666175A6
:107760006C742053657474696E6773204C6F616428
:10777000656400563200000000C8420000C84200A4
:1077800000C84300008C4300004843000048430009
:107790000040410000F042E8030000E8030000C898
:1077A0000000008813000000409C4400409C4400FE
:1077B00000000000000000204E00000000204100FA
:1077C000002041CDCCCC3E000090400000000000E5
:1077D00000000000000000CDCCCC3E0000C8419C61
:1077E00053493F80F946438F42FC42E65A343F4CAE
:1077F00062B045000000000040400000344200003C
:1078000000000000000000000041000000E03F0018
:1078100000C8420000C842000040410000F042C0E1
:10782000030000C0030000C800000088130000101F
:1078300010102000409C440000803F0000003F19D1
:1078400014000000437573746F6D004E796C6F6E99
:10785000504100536174696E20200054657874753E
:107860007200536D6F6F746800486F74656E6420AA
:1078700066616E207370656564206973206C6F7734
:107880006572207468616E206578706563746564E4
:10789000005072696E742066616E20737065656455
:1078A000206973206C6F776572207468616E206543
:1078B0007870656374656400312E3000312E3500B8
:1078C000554E4B4E4F574E004C413130433A204CB1
:1078D000696E65617220416476616E6365206D6FCB
:1078E00064653A20004C413130433A2041646A7566
:1078F0007374656420452D4A65726B3A20005D38CB
:107900004D6D3E0FA8AF00480069960000DF60256E
:10791000555887680427F2E0005E3403CC1960F301
:107920003C0EF88F00DB08029492003E1C079A87F9
:1079300000E524008528527E06001BE4007E7812B4
:1079400070787061F812788F884178427078706131
:10795000782570787061F850788F88D1F0252707E6
:107960008761F025278F88412C0D27AA50D1BC07AD
:1079700007871161BE788F881141785270787061E5
:10798000F852788F88412012788870632052788866
:1079900070634852788887430311179970641812EE
:1079A00078F870654412F8F8F045184278F8706578
:1079B000182578F87065185278F87065185078F8BE
:1079C00070650C078F872365A20F8F8F11450012FA
:1079D00006227069001207222749002506227069D5
:1079E00000250722274900120622276C026236A2D0
:1079F000706C40456C44704C03622222706C43886A
:107A00008888F04C7812BC88806E7852BC88806E72
:107A100038127888706F78127888874F3842788863
:107A2000706F38257888706F3A0079AC786F3D07B1
:107A30009AAC786F7850788887EF39497888706F7A
:107A40000852BC8880729852F88F98522012787031
:107A5000F07348127863875320527870F07348525D
:107A6000786387531007870F247312786387245332
:107A700060699A988BE22304E4443074104E4443C6
:107A800024747C12888960753C50888870557825EC
:107A9000288960757949088960753C128870707909
:107AA0000C12885222594412F124F07A4452F124E3
:107AB000F07A8C52F0368F5A4420F124F07A00404C
:107AC0001454CDCCCC3D0AD7233C17B7D13877CC52
:107AD0002B329595E6241FB14F0A0000204100008B
:107AE000C84200401C4620BCBE4CCA1B0E5AAEC544
:107AF0009D744E414E494E46627573793A207061CD
:107B00007573656420666F7220696E7075740062AB
:107B10007573793A2070617573656420666F7220A1
:107B20007573657200627573793A2070726F636560
:107B30007373696E670000007F4300805443000048
:107B4000524300000000000080C09A99193E0000D6
:107B50000000000080C09A99193E0000A04000007B
:107B6000A0400000004025336420737465703D25FB
:107B70003264206D73636E743D2534640A00000026
:107B80007F43008058439AD95143FFFFFF20413A79
:107B90000020503A002042403A0020403A00202F76
:107BA000002054303A00202F0020423A00202F00BD
:107BB000543A00255345786365737369766520628E
:107BC0006564206C6576656C696E6720636F7272A0
:107BD000656374696F6E3A202569206D6963726F01
:107BE0006E730A00426564206C6576656C696E6729
:107BF000206661696C65642E20546F6F206D75631B
:107C00006820766172696174696F6E2066726F6D4B
:107C100020656570726F6D206D65736800426564E4
:107C2000206C6576656C696E67206661696C656459
:107C30002E2053656E736F72207472696767657268
:107C4000656420746F6F20736F6F6E002020004D8D
:107C50006561737572656420706F696E74733A0044
:107C60005A20736561726368206865696768743A51
:107C700020352E3066004E756D20582C593A20372D
:107C80002C37004D65736820626564206C657665ED
:107C90006C696E67206E6F74206163746976652EFF
:107CA0000020453A00205A3A0020593A0020453A2F
:107CB00000205A3A0020593A00583A00202D3E2020
:107CC0000053706F6F6C4A6F696E3A20002C200071
:107CD000496E616374697669747920536875746458
:107CE0006F776E004B494C4C45442E005072696EC4
:107CF0007465722068616C7465642E206B696C6CAD
:107D000028292063616C6C656421005A206C6976B7
:107D1000652061646A757374206F7574206F6620C6
:107D200072616E67652E2053657474696E67207486
:107D30006F20302E20436C69636B20746F20636F5B
:107D40006E74696E75652E005A206C6976652061C7
:107D5000646A757374206F7574206F662072616E2B
:107D600067652E2053657474696E6720746F2030C8
:107D70000020453A3020423A00543A004731205A18
:107D8000252D2E33662046252D2E336600496E762E
:107D9000616C6964205420636F64652E00447570C3
:107DA0006C696361746520542D636F646520696735
:107DB0006E6F7265642E00416476616E6365204B60
:107DC0003D004B206F7574206F6620616C6C6F777F
:107DD00065642072616E676521004D4B33004D4B29
:107DE000334D4D5533005C762C012533642F2533FC
:107DF000640025336400200A200A200A200025534D
:107E0000537461746973746963733A0A255320204B
:107E10004D37382053256C752054256C750A002584
:107E2000534172632053657474696E67733A2050CE
:107E30003A4D6178206C656E677468286D6D2920F5
:107E4000533A4D696E206C656E67746820286D6DBD
:107E500029204E3A436F7272656374696F6E7320A6
:107E6000523A4D696E207365676D656E7473204676
:107E70003A5365676D656E74732F7365632E0A25BB
:107E80005320204D3231342050252E326620532588
:107E90002E3266204E256420522564204625640A31
:107EA00000255346696C616D656E7420736574744A
:107EB000696E67733A2044697361626C65640A0095
:107EC000255346696C616D656E74207365747469C1
:107ED0006E67733A0A25532020204D3230302044FB
:107EE000252E32660A002553526574726163743A16
:107EF00020533D4C656E67746820286D6D292046BF
:107F00003A537065656420286D6D2F6D29205A3AAB
:107F1000205A4C69667420286D6D290A255320204B
:107F2000204D3230372053252E32662046252E3202
:107F300066205A252E32660A25535265636F766590
:107F4000723A20533D4578747261206C656E677497
:107F50006820286D6D2920463A5370656564202895
:107F60006D6D2F6D290A25532020204D3230382089
:107F700053252E32662046252E32660A255341753A
:107F8000746F2D526574726163743A20533D3020D2
:107F9000746F2064697361626C652C203120746F8A
:107FA00020696E746572707265742065787472757C
:107FB00064652D6F6E6C79206D6F766573206173CB
:107FC000207265747261637473206F7220726563CE
:107FD0006F7665726965730A25532020204D323013
:107FE00039205325640A00255350494420686561AF
:107FF000746265642073657474696E67733A0A25E8
:10800000532020204D3330342050252E3266204915
:10801000252E32662044252E32660A00255350490B
:10802000442073657474696E67733A0A255320207F
:10803000204D3330312050252E32662049252E32F6
:10804000662044252E32660A0025535374657073EA
:108050002070657220756E69743A0A255320204D90
:1080600039322058252E32662059252E3266205A64
:10807000252E32662045252E32660A255355537427
:108080006570207265736F6C7574696F6E3A200A43
:108090002553204D33353020582564205925642040
:1080A0005A2564204525640A25534D6178696D750C
:1080B0006D20666565647261746573202D206E6F36
:1080C000726D616C20286D6D2F73293A0A2553203B
:1080D000204D3230332058252E32662059252E323D
:1080E00066205A252E32662045252E32660A2553F3
:1080F0004D6178696D756D20666565647261746542
:1081000073202D20737465616C746820286D6D2F49
:1081100073293A0A255320204D3230332058252E1A
:1081200032662059252E3266205A252E3266204589
:10813000252E32660A25534D6178696D756D206173
:108140006363656C65726174696F6E202D206E6F5C
:10815000726D616C20286D6D2F7332293A0A255398
:1081600020204D3230312058256C752059256C75F2
:10817000205A256C752045256C750A25534D61786C
:10818000696D756D20616363656C65726174696F9B
:108190006E202D20737465616C746820286D6D2FBE
:1081A0007332293A0A255320204D32303120582588
:1081B0006C752059256C75205A256C752045256CE9
:1081C000750A2553416363656C65726174696F6EEE
:1081D0003A20503D7072696E742C20523D72657465
:1081E000726163742C20543D74726176656C0A254B
:1081F0005320204D3230342050252E326620522517
:108200002E32662054252E32660A2553416476614B
:108210006E636564207661726961626C65733A2091
:10822000533D4D696E2066656564726174652028F2
:108230006D6D2F73292C20543D4D696E2074726131
:1082400076656C20666565647261746520286D6D65
:108250002F73292C20423D6D696E696D756D2073F9
:1082600065676D656E742074696D65202875732966
:108270002C20583D6D6178696D756D205859206AC4
:1082800065726B20286D6D2F73292C20205A3D6D4F
:108290006178696D756D205A206A65726B20286D52
:1082A0006D2F73292C2020453D6D6178696D756DAA
:1082B0002045206A65726B20286D6D2F73290A2571
:1082C0005320204D3230352053252E326620542540
:1082D0002E32662042256C752058252E3266205994
:1082E000252E3266205A252E32662045252E3266EE
:1082F0000A2553486F6D65206F6666736574202884
:108300006D6D293A0A255320204D323036205825EC
:108310002E32662059252E3266205A252E32660AC4
:1083200000544D3A20525B25755D20657374696D6C
:108330006174652E00544D3A202553205220256447
:108340004300544D3A2025532043206573742E007A
:10835000544D3A20636F6F6C20646F776E203C251C
:10836000644300726566696E6500696E697469616F
:108370006C00544D3A2063616C6962722E20666114
:10838000696C65642100544D3A2063616C696272C6
:108390006174696F6E20737461727400544D3A2079
:1083A00043616C2E204E4F542049444C450043619C
:1083B000703A25533A25630A0050525553415F4D98
:1083C0004D553200455854454E4445445F4D32307A
:1083D000004155544F5245504F52545F504F5349EE
:1083E00054494F4E004155544F5245504F52545FDF
:1083F00046414E53004155544F5245504F52545FE1
:1084000054454D500000332E31342E310044656CFC
:108410006574696F6E206661696C65642C204669BD
:108420006C653A200046696C652064656C6574650E
:10843000643A004E6F74205344207072696E746900
:108440006E67005072696E742073617665640053C4
:1084500044207072696E74207061757365640025C4
:1084600033642F253364004F4B0042414400524196
:108470004D426F2046414E200043524153485F43D6
:10848000414E43454C0043524153485F5245434F90
:108490005645520043524153485F5245434F56455B
:1084A0005200222832290025533A2025530A002C55
:1084B000204D39303720452069676E6F7265640042
:1084C0006E6F2076616C696420636F6D6D616E64A0
:1084D000007A65726F72697A656400666163746FB1
:1084E000727920726573746F72656400696E646579
:1084F000782C2074656D702C2075737465702C2039
:10850000756D0050494E44412063616C2073746165
:108510007475733A2000503A005761697420666F91
:10852000722050494E444120746172676574207412
:10853000656D70657261747572653A002041002046
:108540005000204200204C00205200205A00204EB3
:108550004F5420494E495449414C495A45440053CF
:10856000686565742000205A2056414C5545204FBF
:108570005554204F462052414E474500496E766182
:108580006C69642073686565742049442E20416CD1
:108590006C6F7765643A20302E2E004155544F00A1
:1085A0004C414E472053454C20464F5243454400D2
:1085B0004D323536204225642044256420532564FD
:1085C000205425750A0020643A0020693A00207082
:1085D0003A0020643A0020693A0020703A00256988
:1085E00025250A00256925250A0022283129002F82
:1085F0002F00002045585452554445525F434F5573
:108600004E543A3100204D414348494E455F54593C
:1086100050453A00312E3000206261736564206F4E
:108620006E204D61726C696E204649524D57415221
:10863000455F55524C3A68747470733A2F2F6769CE
:10864000746875622E636F6D2F7072757361336419
:108650002F50727573612D4669726D776172652056
:1086600050524F544F434F4C5F56455253494F4E13
:108670003A00373733313032346564005F003832C6
:108680003739002B004649524D574152455F4E4104
:108690004D453A50727573612D4669726D776172FE
:1086A0006520004D3131332053006F6B20006E2F59
:1086B00061003F546F736869626120466C61736842
:1086C000416972204765744950206661696C656430
:1086D0000A00000125311D0C4024301C0B45232FBE
:1086E0001B0A17FF0406222B1A0336373538256973
:1086F000206D696E2C2025692073656300496E76B4
:10870000616C6964204D20636F64653A2025730AAB
:108710000050494E44412070726F62652063616C65
:108720006962726174696F6E207374617274004E55
:108730006F2050494E444120746865726D697374AE
:108740006F7200736574006E6F7A7A6C65004D42CB
:108750004C004652004C7A004C616E6700315F3726
:10876000356D6D5F4D4B332D45494E53795F31303B
:10877000612D4533445245564F0052657600332EE5
:1087800031342E312D383237390046697200534E5C
:1087900020696E76616C696400534E005245534502
:1087A00054004D4D555245530075766C6F0046414F
:1087B0004E0046414E50494E54535400505255536A
:1087C00041005345545F43484F505F005345545F49
:1087D000535445505F005345545F574156455F0021
:1087E000544D435F0043524153485F43414E43451C
:1087F0004C0043524153485F5245434F5645520047
:1088000043524153485F4445544543544544004313
:10881000524153485F004D31303453300047315896
:1088200031305931383046343030300047315A31E8
:10883000304631333030004D313430533000473121
:10884000452D302E3037354632313030004D323004
:108850003453313030300047315A354637323030BA
:10886000004731452D312E35463231303000473109
:108870005A302E32004731583230322E3545384684
:1088800031343030004731592D32463130303000EC
:108890004731583234304532354632323030004775
:1088A000315A302E3346313030300047315835356B
:1088B0004538463230303000473158354532394638
:1088C000313830300047315835354532394631304E
:1088D000373300473932453000473238004D3130A8
:1088E00039004D31393000473830004D3435004DB6
:1088F0003435205A00473736004D3730312050305C
:108900000057697A6172642073746174653A202536
:10891000640A004D393134004D39313500457870E5
:108920006572696D656E74616C00302E3830003090
:108930002E363000302E343000302E323500526565
:10894000736574204D4D55004D4D55004D34340028
:10895000302E383000302E363000302E343000309B
:108960002E323500473238205859004D2038340017
:10897000852E2E00593A202575202D3E202E2E2E94
:1089800000583A202575202D3E202E2E2E0025330E
:10899000642F30002533642F30002563204158496F
:1089A00053205347313D25640A00486F74656E6457
:1089B00000426564005A00590058002D2D2D2D2DC0
:1089C0002D2D2D2D2D2D2D2D2D2D2D2D2D2D2D0004
:1089D000435A5058496E76616C6964536572696197
:1089E0006C4E72009B699F693E8837882C881D8871
:1089F000376B1688A26A473159252E346645252ED5
:108A000034660047315A252E3266004731583530DA
:108A10005931353500D3889B693C6B618857884D47
:108A200088473158252E346645252E346600473157
:108A3000463130383000C588B888AB889F88D388E5
:108A40009088858875886E885425640047315A302F
:108A50002E34004731592D334631303030009F6974
:108A6000E288DD88D988D3884D38342058590047AA
:108A7000312058313235205A3230302046313030B2
:108A800030004D33313020412046310047312058ED
:108A90003132352059313035205A31204638303086
:108AA0003000496E76616C696420504944206361EE
:108AB0006C2E20726573756C74732E204E6F74204B
:108AC00073746F72656420746F20454550524F4D2A
:108AD0002E004D3330312050252E32662049252E70
:108AE00032662044252E3266004D33303320453027
:108AF00020532533750052430044455600424554E7
:108B00004100414C50484100000021002400270052
:108B10002A002D003000330001010000040107018C
:108B20000A0100002200250028002B002E00310041
:108B3000340002010000050108010B0100002000C3
:108B40002300260029002C002F0032000001000025
:108B500003010601090105050505070508080808C0
:108B6000020202020A0A08080404040401010101C5
:108B700001010101030303030303030304070707C0
:108B80000C0C0C0C0C0C0C0C020202020606060665
:108B9000060606060B0B0B0B0B0B0B0B07070A0A43
:108BA0000A0A0A0A0505050404040808010210203F
:108BB0002008081020401020408002010201080413
:108BC00002010102040810204080804020100804A7
:108BD0000201800402018040201008040201080400
:108BE0000201010204081020408001020408102044
:108BF000408010080408801020400440801020406D
:108C0000048000000A0B02090C0D0E080703040182
:108C10000000000000000000000000000000000054
:108C20000000000000000000000000000000121121
:108C30001000000000000000000000000000000024
:108C40000000000000000000000000000000000024
:108C50000000000000000000332E31342E31000AE5
:108C6000204F726967696E616C2050727573612064
:108C700069330A2020205072757361205265736534
:108C8000617263680A2532302E323053004C616EB7
:108C900067756167652075706461746500435A503B
:108CA00058003B530053706F6F6C4A6F696E2069B8
:108CB0007320006164635F696E697400200A200A92
:108CC000200A2000416C6C2044617461005365727D
:108CD00076696365207072657000536869707069A9
:108CE0006E67207072657000537461746973746983
:108CF0006373004C616E677561676500455241534F
:108D0000494E4720616C6C20646174610046616368
:108D1000746F727920524553455400505255534157
:108D20003344465700494E54340003000E000100FE
:108D3000400003000200000004007072757361338C
:108D40006400323032352D30342D32322032323A16
:108D500030333A35330020332E31342E312D383232
:108D600037395F37373331303234656400737461BB
:108D7000727400534E207570646174652066616979
:108D80006C656400534E20757064617465640043C3
:108D90005A50580043524153485F44455445435448
:108DA000454458590043524153485F444554454354
:108DB000544544590043524153485F444554454348
:108DC00054454458004D323900252D392E39535B16
:108DD00000544D20657374696D6174696F6E206411
:108DE0006964206E6F7420636F6E766572676500CC
:108DF000544D20697465723A257520763A252E32D5
:108E00006620653A252E33660A00200A200A2000D3
:108E100000004842000058419A998D413333534035
:108E20004D4D55323A004D494E54454D5020424526
:108E300044206669786564004D494E54454D502084
:108E4000484F54454E4420666978656400726563F6
:108E50006F7665725F6D616368696E655F7374617B
:108E600074655F61667465725F706F7765725F705D
:108E7000616E69632C20696E697469616C200050B1
:108E8000525553412075766C6F00473420533000A3
:108E90004D313130204E256C75004D323620532532
:108EA0006C75004D31303620532575004731204612
:108EB0002564004D3832004739322045252D2E33A8
:108EC00066004D3230342050252D2E31662052253B
:108ED0002D2E31662054252D2E3166004731205A23
:108EE000252D2E3366005052555341204D424C20C3
:108EF00056310047312058252D2E33662059252D17
:108F00002E3366204633303030002C206665656491
:108F10006D756C7469706C793A0046656564726150
:108F200074653A0047312045352046313230004DD6
:108F300031303920532564004D31343020532564BD
:108F4000004D3130342053256400473238205820FA
:108F500059004731205A252E3366204638303000DC
:108F600000002110422063308440A550C660E770A5
:108F7000088129914AA16BB18CC1ADD1CEE1EFF14D
:108F80003112100273325222B5529442F772D662F5
:108F9000399318837BB35AA3BDD39CC3FFF3DEE39D
:108FA0006224433420040114E664C774A444855445
:108FB0006AA54BB528850995EEE5CFF5ACC58DD5ED
:108FC0005336722611163006D776F6669556B44695
:108FD0005BB77AA719973887DFF7FEE79DD7BCC73D
:108FE000C448E5588668A7784008611802282338E5
:108FF000CCC9EDD98EE9AFF9488969990AA92BB98D
:10900000F55AD44AB77A966A711A500A333A122A34
:10901000FDDBDCCBBFFB9EEB799B588B3BBB1AABDC
:10902000A66C877CE44CC55C222C033C600C411C84
:10903000AEED8FFDECCDCDDD2AAD0BBD688D499D2C
:10904000977EB66ED55EF44E133E322E511E700ED4
:109050009FFFBEEFDDDFFCCF1BBF3AAF599F788F7C
:109060008891A981CAB1EBA10CD12DC14EF16FE15C
:109070008010A100C230E320045025404670676094
:10908000B9839893FBA3DAB33DC31CD37FE35EF3AC
:10909000B1029012F322D2323542145277625672E4
:1090A000EAB5CBA5A89589856EF54FE52CD50DC5FC
:1090B000E234C324A0148104667447642454054434
:1090C000DBA7FAB79987B8975FE77EF71DC73CD74C
:1090D000D326F2369106B016576676761546345684
:1090E0004CD96DC90EF92FE9C899E9898AB9ABA99C
:1090F0004458654806782768C018E1088238A328D4
:109100007DCB5CDB3FEB1EFBF98BD89BBBAB9ABBEB
:10911000754A545A376A167AF10AD01AB32A923A23
:109120002EFD0FED6CDD4DCDAABD8BADE89DC98D3B
:10913000267C076C645C454CA23C832CE01CC10C73
:109140001FEF3EFF5DCF7CDF9BAFBABFD98FF89F8B
:10915000176E367E554E745E932EB23ED10EF01EC3
:109160007C3C3E3F2F2A225C0024F4D43050C38E36
:1091700020C2A24017828B7011127A910D816CD996
:109180000AA861E108C7586607615143061E4B5D96
:1091900005C145A7041A411104093D9803713931ED
:1091A000034036DB0265339102D4305402802E1D19
:1091B00002632CEE01752AC501B028A00110278199
:1091C000018F2564012B244B01E0223401AC211FC7
:1091D000018D200D01801FFC00841EED00971DDF16
:1091E00000B81CD200E61BC600201BBC00641AB2EB
:1091F00000B219A8000A19A0006A189900D11791A5
:109200000040178B00B516840031167E00B3157927
:10921000003A157300C7146F0058146A00EE136605
:10922000008813630025135E00C7125B006C1257A1
:109230000015125400C111510070114F0021114B43
:1092400000D61049008D104700461044000210421D
:1092500000C00F4000800F3E00420F3C00060F3B55
:1092600000CB0E3800930E37005C0E3500270E340D
:1092700000F30D3200C10D3100900D3000600D2E55
:1092800000320D2D00050D2C00D90C2B00AE0C2941
:1092900000850C29005C0C2700350C27000E0C26DD
:1092A00000E80B2400C40B2400A00B23007D0B233B
:1092B000005A0B2100390B2100180B2000F80A1F5F
:1092C00000D90A1E00BB0A1E009D0A1D00800A1D4F
:1092D00000630A1C00470A1B002C0A1B00110A1A13
:1092E00000F7091A00DD091900C4091900AB0919B2
:1092F00000920917007B091800630917004C091632
:109300000036091600200916000A091500F508158F
:1093100000E0081400CC081400B8081400A40814D5
:1093200000900813007D0812006B08130058081203
:109330000046081200340811002308110012081119
:109340000001081100F0071000E0071000D007101E
:1093500000C0071000B0070F00A107100091070E12
:109360000083070F0074070F0065070E0057070EF4
:109370000049070E003B070D002E070E0020070DC9
:109380000013070D0006070D00F9060C00ED060D91
:1093900000E0060C00D4060C00C8060C00BC060C4D
:1093A00000B0060C00A4060B0099060C008D060BFD
:1093B0000082060B0077060B006C060B0061060AA4
:1093C0000057060B004C060A0042060A0038060A3F
:1093D000002E060A0024060A001A060A00100609D2
:1093E0000007060A00FD050900F4050900EB050960
:1093F00000E2050900D9050900D0050900C70509E3
:1094000000BE050900B5050800AD050800A5050961
:10941000009C050800940508008C050800840508D8
:10942000007C050800740508006C05070065050848
:10943000005D050700560508004E050700470507B3
:10944000004005080038050700310507002A050718
:1094500000230507001C050600160507000F050779
:10946000000805060002050700FB040600F50407D6
:1094700000EE040600E8040600E2040700DB040630
:1094800000D5040600CF040600C9040600C3040684
:1094900000BD040600B7040600B1040500AC0406D4
:1094A00000A6040600A00405009B04060095040520
:1094B00000900406008A0405008504050080040667
:1094C000007A04050075040500700405006B0405AE
:1094D0000066040500610405005C040500570405EE
:1094E00000520405004D040500480405004304052E
:1094F000003E0404003A040500350405003004046D
:10950000002C04050027040400230405001E0404A5
:10951000001A04040016040500110404000D0404DC
:1095200000090405000404040000040400FC030412
:1095300000F8030400F4030400F0030400EC030447
:1095400000E8030400E4030400E0030400DC030477
:1095500000D8030400D4030400D0030400CC0304A7
:1095600000C8030300C503030024F404D9201BC46E
:109570000C5C0E9804C4095F0265077101F405F9DB
:1095800000FB04B30048048700C103690058035579
:109590000003034500BE023A008402310053022A50
:1095A000002902250004022000E4011C00C8011962
:1095B00000AF01170098011400840113007101101D
:1095C000006101100051010E0043010D0036010B36
:1095D000002B010B0020010B00150109000C0109F3
:1095E0000003010800FB000800F3000800EB00077F
:1095F00000E4000600DE000600D8000600D20006E7
:1096000000CC000500C7000500C2000500BD000435
:1096100000B9000400B5000400B1000400AD00046E
:1096200000A9000400A5000300A20003009F00049D
:10963000009B0003009800030095000200930003C4
:1096400000900003008D0002008B000300880002E0
:10965000008600020084000300810002007F0002F7
:10966000007D0002007B000200790002007700010B
:109670000076000200740002007200010071000216
:10968000006F0002006D0001006C0002006A000122
:10969000006900020067000100660001006500012A
:1096A000006400020062000100610001006000012E
:1096B000005F0002005D0001005C0001005B000132
:1096C000005A000100590001005800010057000134
:1096D0000056000100550001005400010053000035
:1096E0000053000100520001005100010050000130
:1096F000004F0001004E0000004E0001004D00012F
:10970000004C0001004B0000004B0001004A00012A
:109710000049000100480000004800010047000126
:109720000046000000460001004500000045000121
:10973000004400010043000000430001004200001B
:109740000042000100410000004100010040000112
:10975000003F0000003F0001003E0000003E00010D
:10976000003D0000003D0001003C0000003C000006
:10977000003C0001003B0000003B0001003A0000FB
:10978000003A0001003900000039000100380000F3
:1097900000380000003800010037000000370001E9
:1097A00000360000003600000036000100350000E1
:1097B00000350000003500010034000000340000D6
:1097C00000340001003300000033000000330001CA
:1097D00000320000003200000032000100310000C1
:1097E00000310000003100010030000000300000B6
:1097F00000300001002F0000002F0000002F0000AB
:10980000002F0001002E0000002E0000002E00019D
:10981000002D0000002D0000002D0000002D000193
:10982000002C0000002C0000002C0000002C000187
:10983000002B0000002B0000002B0000002B00017B
:10984000002A0000002A0000002A0000002A00016F
:109850000029000000290000002900000029000064
:109860000029000100280000002800000028000056
:109870000028000000280001002700000027000049
:10988000002700000027000000270001002600003C
:10989000002600000026000000260000002600012F
:1098A0000025000000250000002500000025000024
:1098B0000025000000250001002400000024000015
:1098C0000024000000240000002400010023000008
:1098D00000230000002300000023000000230000FC
:1098E00000230000002300010022000000220000ED
:1098F00000220000002200000022000000220001DF
:1099000000210000002100000021000000210000D3
:1099100000210000002100000021000100200000C3
:1099200000200000002000000020000000200000B7
:10993000002000000020000000200001001F0000A7
:10994000001F0000001F0000001F0000001F00009B
:10995000001F0000001F0001001E0000001E00008C
:10996000001E0000001E0000005049442041757494
:109970006F74756E652066696E6973686564212011
:1099800050757420746865206C617374204B702C62
:10999000204B6920616E64204B6420636F6E73748A
:1099A000616E74732066726F6D2061626F766520E0
:1099B000696E746F20436F6E666967757261746952
:1099C0006F6E2E6800504944204175746F74756E37
:1099D00065206661696C6564212074696D656F75C9
:1099E000740020403A00543A00423A005049442062
:1099F0004175746F74756E65206661696C6564216C
:109A00002054656D706572617475726520746F6F36
:109A1000206869676800204B643A2000204B693A4F
:109A20002000204B703A200020436C6173736963FF
:109A30002050494420002054753A2000204B753AAC
:109A40002000206D61783A2000206D696E3A200078
:109A500020643A200020626961733A200050494432
:109A6000204175746F74756E652073746172740033
:109A7000504944204175746F74756E652066616944
:109A80006C65642E2042616420657874727564652B
:109A900072206E756D6265722E00544D4C202564E7
:109AA00020256420257820256C7820256C780A00F4
:109AB0004D494E54454D50004D494E54454D502052
:109AC000424544004D494E54454D5020414D4200C1
:109AD0004D415854454D50004D415854454D50202E
:109AE000424544004D415854454D5020414D42009F
:109AF000544D3A206572726F7220636C65617265B5
:109B00006400544D3A206572726F722074726967F6
:109B100067657265642100544D3A206572726F72F8
:109B2000207C25667C3E25660A0070012C01900190
:109B30002701B0012201C0011D01F001180110022E
:109B4000130130020E016002090190020401C002FB
:109B5000FF000003FA004003F5008003F000D0038B
:109B6000EB002004E6007004E100E004DC004005A6
:109B7000D700C005D2004006CD00D006C80080073F
:109B8000C3003008BE00F008B900C009B400B00A34
:109B9000AF00B00BAA00D00CA500000EA000500F23
:109BA0009B00C01096005012910000148C00C0154C
:109BB0008700B0178200B0197D00D01B7800001E0E
:109BC000730040206E0090226900F024640040275A
:109BD0005F0090295A00E02B5500102E50002030D5
:109BE0004B0010324600E033410090353C00103706
:109BF000370070383200A0392D00B03A2800A03B61
:109C00002300603C1E00103D1900903D1400103EE2
:109C10000F00703E0A00C03E0500003F0000901398
:109C20007D00B0157800F0177300601A6E00F01C0C
:109C30006900A01F640050225F0020255A00E02721
:109C40005500902A5000202D4B00A02F4600F031E7
:109C5000410010343C00F0353700A0373200203985
:109C60002D00603A2800703B2300603C1E00203D20
:109C70001900C03D1400403E0F00A03E0A00F03E17
:109C80000500403F0000703FFBFF903FF6FFB03FF4
:109C9000F1FFC03FECFFD03FE7FFE03FE2FFF03FC6
:109CA000DDFFF03FD8FF20484F54454E4420544834
:109CB00045524D414C2052554E4157415900204884
:109CC00045415442454420544845524D414C205250
:109CD000554E4157415900544845524D414C205230
:109CE000554E415741590042454420544845524D34
:109CF000414C2052554E415741590020544845523D
:109D00004D414C2052554E41574159202850524503
:109D10004845415420484F54454E4429002054485A
:109D200045524D414C2052554E41574159202850E3
:109D30005245484541542048454154424544290034
:109D400050524548454154204552524F52004245D9
:109D5000442050524548454154204552524F5200EC
:109D60002074726967676572656421004865617473
:109D7000657273207377697463686564206F6666C3
:109D80002E20003A20004572723A200000FF0102A6
:109D9000010002FFFFFE0001FE01FF00506C656143
:109DA0007365207265737461727400544D3A206952
:109DB0006E76616C696420706172616D6574657244
:109DC000732C2063616E6E6F7420656E61626C65CA
:109DD00000255320204D3331302050252E3266206F
:109DE00055252E34662056252E32662043252E32E8
:109DF000662044252E3466204C2575205325752079
:109E00004225752045252E32662057252E326620A4
:109E100054252E32660A00255320204D3331302040
:109E20004925752052252E32660A00546865726DE8
:109E3000616C204D6F64656C2073657474696E6726
:109E4000733A006666CA413333BF410000B441CD66
:109E5000CC9C4100009841666692419A998D41CD13
:109E6000CC88416666864100008441666682410076
:109E700000804166667E4133337B419A9979416621
:109E8000667641452D6D6F746F72206375727265D1
:109E90006E74207363616C696E6720656E61626CBD
:109EA000656400010808010A0A0114140112127401
:109EB0006D63323133305F686F6D655F656E7465F9
:109EC0007228617865735F6D61736B3D3078253002
:109ED0003278290A00746D63323133305F686F6DF8
:109EE000655F6578697420746D63323133305F73F8
:109EF000675F686F6D696E675F617865735F6D61DD
:109F0000736B3D3078253032780A00726573756C5A
:109F1000742076616C75653A2025640A0020693DDD
:109F200025326420636E743D2532642076616C3D79
:109F30002532640A00636C7573746572733A00208D
:109F4000693D25326420737465703D2532640A00D2
:109F5000736F727465642073616D706C65733A0021
:109F60005553415254322072782046756C6C212131
:109F700021003A2000252D31322E313253252D6417
:109F80002F36002533642F252D336400203A20001E
:109F900025335300252D3773004E642025342E328F
:109FA000662000252D31352E313553252D35640A97
:109FB000252D31352E313553252D35640A00255395
:109FC0000A20252D31362E313653252D33640A20B3
:109FD000252D31362E313653252D33640025530A75
:109FE00020252D31362E313653252D33640A202578
:109FF0002D31362E313653252D33640A20252D314F
:10A00000362E313653252D33640025530A20252D55
:10A0100031362E313653252D33640A20252D313625
:10A020002E313653252D33640A20252D372E3753F4
:10A030005820252D336420205920252D33640020FD
:10A04000257325336481200A00205057523A20207E
:10A050002020202025342E3166560A204245443ADD
:10A0600020202020202025342E3166560025530A3A
:10A0700020582025640A20592025640025752E25A6
:10A08000752E25752E25750020002000466C617305
:10A090006841697220495020416464723A004D4D14
:10A0A0005520202020202020204E2F410025642EE6
:10A0B00025642E2564002046573A00323032352D73
:10A0C00030342D3232004533445245564F00454915
:10A0D0004E53795F31306100315F37356D6D5F4DC3
:10A0E0004B330020486173683A37373331303234AC
:10A0F000656400205265706F3A70727573613364E5
:10A100000020332E31342E312D3832373900466954
:10A11000726D776172653A003E00464C4558202DBD
:10A1200020203234302F353000464C4558202D2029
:10A13000203234300050502020202D202032353461
:10A140002F3130300050502020202D202032353447
:10A150000048495053202D20203232302F313030EA
:10A160000048495053202D202032323000414253C4
:10A1700020202D20203235352F3130300041425300
:10A1800020202D20203235350050412020202D2048
:10A19000203237352F39300050412020202D20200B
:10A1A0003237350050564220202D20203231352FB5
:10A1B00037350050564220202D20203231350050B6
:10A1C000432020202D20203237352F3131300050D0
:10A1D000432020202D2020323735004153412020BC
:10A1E0002D20203236302F31303500415341202090
:10A1F0002D20203236300050455420202D20203292
:10A2000033302F38350050455420202D2020323354
:10A210003000504C4120202D20203231352F363057
:10A2200000504C4120202D202032313500252D3189
:10A23000322E313253252B382E3166004578747218
:10A24000756465723A0025632531372E32666D6D6F
:10A2500000583A00593A005A3A002563252D313307
:10A260002E313353252B352E3366002533750050A0
:10A27000494E44412063616C6962726174696F6E1A
:10A28000206661696C65642E20436F6E74696E751B
:10A29000652077697468207072657373696E6720D2
:10A2A000746865206B6E6F622E0050494E444120E9
:10A2B00063616C6962726174696F6E20646F6E6550
:10A2C0002E20436F6E74696E7565207769746820FF
:10A2D0007072657373696E6720746865206B6E6F4A
:10A2E000622E001000C90210012C014001220170F1
:10A2F000011801B0010E01F00104015002FA00B092
:10A3000002F0003003E600D003DC009004D20070BD
:10A3100005C800A006BE000008B400B009AA00D01D
:10A320000BA000600E960060118C000015820020CA
:10A33000197800C01D6E00A0226400B0275A00905A
:10A340002C500000314600E0343C001038320090C0
:10A350003A2800603C1E00A03D1400803E0A002008
:10A360003F00004D6561737572652063656E7465AD
:10A370007220200078797A63616C5F6D6561737516
:10A3800072655F656E7465720A0078797A63616CD4
:10A390005F73706972616C382063783D2564206357
:10A3A000793D2564207A303D256420647A3D25641A
:10A3B000207261646975733D25642061643D256484
:10A3C0000A0078797A63616C5F7365617263685AB9
:10A3D000206E6F207369676E616C0A20783D256C72
:10A3E0006420793D256C64207A3D256C640A002048
:10A3F0004F4E2D5349474E414C20617420783D25E6
:10A400006420793D2564207A3D25642061643D25E2
:10A41000640A0078797A63616C5F7365617263685E
:10A420005A20783D256C6420793D256C64207A3D66
:10A43000256C640A002530327800205B25662025D3
:10A44000665D206D6D207061747465726E20636549
:10A450006E7465720A00205B25662025665D5B25AB
:10A46000665D206D6D20646976657267656E6365F3
:10A470000A000000F000F801FC03FE07FE07FE07DB
:10A48000FE07FC03F801F000000000000000F000EF
:10A49000F801FC03FC03FC03FC03F801F0000000DE
:10A4A000000078797A63616C5F6D656173757265C0
:10A4B0005F6C656176650A00203C20005741524E72
:10A4C000494E473A2046726F6E7420706F696E7401
:10A4D000206E6F7420726561636861626C652E2006
:10A4E0005920636F6F7264696E6174653A00000091
:10A4F0000040410000C04000005C430000C040003C
:10A50000005C4300004643000040410000464325F4
:10A51000642F3400497465726174696F6E3A20006B
:10A5200043616C6962726174696F6E206661696C07
:10A5300065642120436865636B20746865206178D9
:10A54000657320616E642072756E20616761696E4B
:10A550002E0078797A63616C5F73706972616C3216
:10A560002063783D25642063793D2564207A303D61
:10A57000256420647A3D2564207261646975733DA9
:10A5800025642061643D25640A000A00436F756EEE
:10A5900074646F776E3A202564200025640A0053A6
:10A5A00063616E20636F756E74646F776E3A20001E
:10A5B0005061747465726E2063656E746572205BA1
:10A5C00025662025665D2C206D61746368202566F4
:10A5D00025250A00205B25662C2025665D5B256607
:10A5E0005D2066696E616C20636972636C650A0048
:10A5F000746D63323133305F676F746F5F7374658E
:10A6000070202564202564202564202564200A000C
:10A61000E02D903E8988B24111369C3E7777C1414A
:10A6200029CBB03EEFEEDA41BA49CC3EEFEEFC4129
:10A6300061C3F33EEFEE16429CA2133FCDCC3642EF
:10A640008AB0113FABAA56428863DD3DABAA5642A1
:10A65000B8AF433F555572421826533F33B3824239
:10A66000302A593FEF6E8642000070C10000C84298
:10A670000000C4C10000A0410000E0C00000204173
:10A68000000060C00000C0400000A0412222F24053
:10A690000000A0C19A99A14000000CC25555054286
:10A6A00052657365745265747279417474656D7026
:10A6B000747300436F6F6C696E672074696D6572A7
:10A6C0002073746F707065640048656174657220F2
:10A6D000636F6F6C646F776E00436F6F6C696E674A
:10A6E0002054696D656F757420737461727465644C
:10A6F00000536176696E6720616E64207061726BD1
:10A70000696E670048656174657220636F6F6C6481
:10A710006F776E2070656E64696E67005265737541
:10A720006D696E672058595A004D4D5532746F6FE0
:10A730006C3D004D4D55323A0057726974696E6731
:10A7400020746F2066696C653A200046696C65204C
:10A75000616C7265616479206F70656E6564004D2F
:10A76000533C5328531353FD52EA52D452C052AFB4
:10A7700052995228533C5385527652625251523C60
:10A7800052755B265214520152F051DB51C851B43C
:10A79000519F51965184516F514D36303020415563
:10A7A000544F0046494E44412066696C616D656EA8
:10A7B000742072756E6F75742100436F6D6D756EC8
:10A7C00069636174696F6E2074696D656F7574007B
:10A7D00050726F746F636F6C204572726F720003FA
:10A7E000000356657273696F6E206D69736D6174D5
:10A7F000636800436F6D6D616E64204572726F72A5
:10A8000000436F6D6D616E642072656A6563746587
:10A8100064004D4D5520427574746F6E20707573D1
:10A82000686564005265747279427574746F6E5015
:10A8300072657373656400AA5595557E55695554C4
:10A84000554055305519550255EB54D754C354ADA6
:10A8500054AD54AD549854985498548554855485A7
:10A86000547254725472545B545B545B5446544655
:10A8700054465430543054305420540B54F553DF64
:10A8800053D053C353AC53995387537453625352A9
:10A8900053427574746F6E00436865636B557365DE
:10A8A00072496E7075742D62746E4C4D5220004664
:10A8B000493A202046533A202020203E2020822062
:10A8C00020208100486F74656E642074656D70652A
:10A8D00072617475726520726561636865640052A7
:10A8E0006573756D696E672054656D7000436F6F99
:10A8F0006C646F776E20666C616720636C65617253
:10A9000065640020573A0020453A00543A004E6FE3
:10A910002030784646207265636569766564005329
:10A92000656E64696E6720307846460046696C65DE
:10A930002073656C6563746564002053697A653AB9
:10A94000200046696C65206F70656E65643A200072
:10A950004E6F772066726573682066696C653A2071
:10A96000004E6F7720646F696E672066696C653A88
:10A9700020002220706F73002220706172656E7457
:10A980003A2200535542524F5554494E45204341B7
:10A990004C4C207461726765743A22007472796954
:10A9A0006E6720746F2063616C6C207375622D6715
:10A9B000636F64652066696C6573207769746820CD
:10A9C000746F6F206D616E79206C6576656C732E87
:10A9D00000062833D036C23E013F154132423B4388
:10A9E000F2443B45F24622473B48F2493B4AF05885
:10A9F00098590C5A085B0C5C086110679B6E2271B9
:10AA0000077208FF095A0D000EF019145E08206441
:10AA10002B6D322FFF2022257322002025236C78F6
:10AA2000004449525F45584954004449525F454EDD
:10AA30005445523A20257320222573220A0061755D
:10AA4000746F25692E6700041A44656372656D652D
:10AA50006E745265747279417474656D70747300AC
:10AA6000081B1C0B14525354436F6D6D54696D6574
:10AA70006F7574002C206C61737420627974657337
:10AA80003A200022206661696C65643A204275664E
:10AA90006665722066756C6C21004572726F723A41
:10AAA000002200456E717565696E6720746F2074B1
:10AAB00068652066726F6E743A2022004D4D5532E3
:10AAC0003A006563686F3A003E53302A63362E00C1
:10AAD0004D4D552069732000252E3130532000251F
:10AAE000346400457872656D65207370616E206F07
:10AAF0006620746865205A2076616C756573210044
:10AB000025642F39004D4D55323A00253364001825
:10AB1000010419020AFA6284620A629D615461C2E8
:10AB2000604A60E25F935F735F275F735F105F103F
:10AB30005F105F105F105F105F105F105F105F109D
:10AB40005F105F105F105F105F105F105F105F108D
:10AB50005F105F105F105F105FD95E985E4E5EDB26
:10AB60005DA65D5C5D125DB45C7B5C395C1C5C0168
:10AB7000010101010101027101710132323203034D
:10AB80000303030303030303030303030303030395
:10AB90000393932438039303010256036500660070
:10ABA0006700680069006A006B006C007300740045
:10ABB0007D007E00C900D300DD00CA00D400DE00A5
:10ABC0002D01370141012E01380142012F013901C8
:10ABD000430130013A01440131013B014501320199
:10ABE00091019201F501F601F701F801F901FA016D
:10ABF000FB01FC0184038763F0637C6373636C6314
:10AC0000784FE74665635B63252E3230530A7072D6
:10AC10007573612E696F2F3034256875002055706B
:10AC200067726164696E672078666C6173680A2078
:10AC3000446F206E6F7420646973636F6E6E65631A
:10AC4000742100773235783230636C5F63666D0A49
:10AC500000773235783230636C5F656E7465720AE6
:10AC60000073746172740A00C03AF56311241FBE48
:10AC7000CFEFD1E2DEBFCDBF00E00CBF13E0A0E01C
:10AC8000B2E0E0E4F6EC03E00BBF02C007900D92E7
:10AC9000A432B107D9F728E1A4E2B3E001C01D92C4
:10ACA000A032B207E1F716E5C5E3D6E500E006C03D
:10ACB00021970109802FFE010F9464DDC433D10771
:10ACC00080E00807A9F70E946EFB0D940EE30C9438
:10ACD000EB662F923F924F925F926F927F928F928C
:10ACE0009F92AF92BF92CF92DF92EF92FF920F931B
:10ACF0001F93CF93DF93CDB7DEB72F970FB6F8949E
:10AD0000DEBF0FBECDBF6C011B015A01FC011782D3
:10AD1000168283819E012F5F3F4F490181FDD2C082
:10AD20008FEF9FEFEEC2F12C512C00E0003238F48F
:10AD30008B3209F190F48032F9F0833209F107FD8A
:10AD400034C020ED280F2A3020F506FF1BC0FAE0A2
:10AD5000FF9E200D1124F22E05C08D3279F0803334
:10AD600071F70160F10193FD859193FF81911F01BE
:10AD70008111DCCF1AC002600460F4CF0860F2CF0A
:10AD80000061F0CF3AE0539E200D1124522E006254
:10AD9000E9CF8E3221F406FDB1C20064E3CF8C36D8
:10ADA00011F40068DFCF8836E9F29BEB980F9330FF
:10ADB00008F05FC00061805E06FD02C046E0F42E30
:10ADC000102F1F73853609F05BC0106417FF61C038
:10ADD0008F2D9BE39F1508F48BE344244394480E86
:10ADE00027E03501F4E06F0E711CF501608171817F
:10ADF00082819381042DA4010F940DD95C01F98106
:10AE0000FC87F0FF03C00DE2F3FF07C00BE211FD6A
:10AE100004C0012F047012FD00E22C852C70E22E7C
:10AE200009F46BC00111D8C2F3E0E12CF515A0F4D0
:10AE300083E0E52CE81A13FD08C0B60180E290E03B
:10AE40000F94BCDAEA94E110F8CF002329F0B601A0
:10AE5000802F90E00F94BCDA3C852CE9A22E25E7E8
:10AE6000B22E33FD04C090EAA92E95E7B92E1071D9
:10AE700022C09BE9980F933008F047C10F7E9CCF0A
:10AE8000863611F41068A2CFFF2009F49FCFFA9400
:10AE90009DCFE7E02F2DEF1518F427E037E0F32ED4
:10AEA000412C9FCF11118052B60190E00F94BCDA73
:10AEB0008FEFA81AB80AF50184918111F3CFE11040
:10AEC00084C25301F6019381F10193FD859193FFB3
:10AED00081911F01882309F411C2853241F493FD49
:10AEE000859193FF81911F01853209F01CCFB60136
:10AEF00090E00F94BCDA3501E4CF17FF6FC04A0C25
:10AF0000FC85F4FF04C08A81813309F44A94141447
:10AF10000CF086C028E0241510F488E0482E85E067
:10AF200090E017FF06C0C501B7FE02C090E080E0C8
:10AF3000019601110196FF2031F02F2D30E02F5F97
:10AF40003F4F820F931F5816190619F014F0E52C85
:10AF5000E81A812F897011F4E11067C0002329F0ED
:10AF6000B601802F90E00F94BCDA13FD02C0E1100F
:10AF700063C017FF7CC08501B7FE02C010E000E08F
:10AF8000C501841991092C016F2D70E0EE27FF2770
:10AF9000E61BF70BFF87EE870F3F100729F4B6017A
:10AFA0008EE290E00F94BCDAA016B1060CF44BC010
:10AFB000401651060CF047C0F501E01BF10BE80DFF
:10AFC000F91D8181015011092E853F850217130754
:10AFD000E4F1B60190E00F94BCDADECF16FD9FCF0E
:10AFE000EF2DF0E0EA15FB0534F03CEFA3163FEF40
:10AFF000B3060CF010683296E80DF91D01C0FA9402
:10B00000FF2019F082918033D1F317FF88CF4424B9
:10B0100043944F0CFA141B0431F02CF0FA187FCF34
:10B02000442443947CCFF12C7ACFB60180E290E0A7
:10B030000F94BCDAEA9490CFB60180E390E00F94CD
:10B04000BCDAEA9494CF80E3BDCFA016B10641F4F8
:10B050009A81963350F4953319F43C8534FF05C03A
:10B06000B60190E00F94BCDA2ACF81E3F9CF8A8150
:10B07000813319F09C859F7E9C87B60190E00F94E8
:10B08000BCDAFF20A9F0B6018EE290E00F94BCDAA2
:10B09000F394F394E2E001E00E0FE80DF92DF11DB9
:10B0A0008081B60190E00F94BCDAE02F0F11F3CF4E
:10B0B00085E690E014FF02C085E490E0B6010F94AD
:10B0C000BCDAB7FC06C0A114B104C1F4EC85E4FFFE
:10B0D00015C0B194A194B1088DE2B60190E00F942F
:10B0E000BCDA80E32AE0A216B10454F4B60190E081
:10B0F0000F94BCDAB601C501C096B4CF8BE2EDCF98
:10B100008F5FFAE0AF1AB108EDCF8336C9F083370D
:10B1100071F1833509F05BC03501F2E06F0E711CEF
:10B12000F501A080B1806F2D70E006FD02C06FEFC9
:10B130007FEFC5010F9450DA9D878C8700680DC0A2
:10B14000350132E0630E711CF5018081898321E0B5
:10B1500030E03D872C8754010F7703FD06C02C8516
:10B160003D855216130609F0A8F4E52C2BC03501D5
:10B1700032E0630E711CF501A080B1806F2D70E08C
:10B1800006FD02C06FEF7FEFC5010F9475DA9D8752
:10B190008C87E2CFB60180E290E00F94BCDA5A943B
:10B1A000DECFF50107FD859107FF81915F01B601B3
:10B1B00090E00F94BCDAE110EA948C859D850197AC
:10B1C0009D878C87EC85FD85EF2B59F778CE8436EB
:10B1D00019F0893609F074C0350107FF66C0F4E044
:10B1E0006F0E711CF5016081718182819381102F36
:10B1F0001F7697FF08C090958095709561957F4F59
:10B200008F4F9F4F10682AE030E0A4010F94E3DBDA
:10B21000A82EA818BA2C012F16FF0AC00E7FAF1453
:10B2200038F414FF04C012FD02C0012F0E7EBF2CA3
:10B2300004FFA3C0FE01EA0DF11D8081803309F0F7
:10B2400095C0097EF02FF870EF2E03FDA5C000FF1A
:10B250009FC0FA2CB51410F4F50CFB1804FFA2C023
:10B26000B60180E390E00F94BCDA02FF09C088E7E2
:10B2700090E001FF02C088E590E0B6010F94BCDACF
:10B28000AF1408F49BC0AA940A2D10E00F5F1F4F63
:10B29000080D191DF80182918F01B60190E00F94FD
:10B2A000BCDA80169106B1F70ACEF2E06F0E711C7F
:10B2B000F50160817181072E000C880B990B97CFE7
:10B2C000102F8537A9F41F7E2AE030E0350117FFE3
:10B2D00044C0F4E06F0E711CF501608171818281C0
:10B2E0009381A4010F94E3DBA82EA8181F7792CFB7
:10B2F000197F8F3679F1F0F4883539F1F6018681BE
:10B3000097812F960FB6F894DEBF0FBECDBFDF91A9
:10B31000CF911F910F91FF90EF90DF90CF90BF9052
:10B32000AF909F908F907F906F905F904F903F90E5
:10B330002F900895803739F0883701F714FD146095
:10B3400020E130E0C3CF1061F9CF04FD166020E1A9
:10B3500032E0BCCF28E030E0B9CFF2E06F0E711CD4
:10B36000F5016081718190E080E0BBCF02FD02C0F9
:10B37000B39468CFB394B39465CF802F867809F4E3
:10B3800061CFF6CFB60180E290E00F94BCDAB394BF
:10B39000B514C0F3E12C62CFE52CEB18B51408F41A
:10B3A0005DCFF8CF802F867809F46ACF8BE201FF5A
:10B3B00080E207FD8DE2B60190E060CFB60180E348
:10B3C00090E00F94BCDAFA945BCFB60180E290E093
:10B3D0000F94BCDAEA9473CD24E0E12C251508F033
:10B3E00036CD84E026CD20E030E040E85FEB609190
:10B3F00083027091840280918502909186020F945D
:10B4000071DE882321F1E0919212F0919312EB55B5
:10B41000FF4E80818B7F8230D1F480E1E3E8F2E05F
:10B42000A2E9B6E001900D928A95E1F780E090E004
:10B43000A0E8BFEB8093830290938402A0938502DF
:10B44000B09386028091690590916A05089581E024
:10B4500090E00895CF92DF92EF92FF920F931F93A7
:10B46000CF93DF9390E0EC01CC0FDD1FCC0FDD1FFD
:10B47000FE01E25BF4482591359145915491FE011E
:10B48000EA5EF14FC080D180E280F3808E010E56DB
:10B49000194FC701B6010F947CDDF80160837183F9
:10B4A00082839383FE01EE5BF448259135914591AB
:10B4B00054918E010F5D1D4FC701B6010F947CDDC5
:10B4C000F8016083718382839383FE01EA5CF44810
:10B4D0002591359145915491CB5EDD4FC701B60161
:10B4E0000F947CDD688379838A839B83DF91CF917E
:10B4F0001F910F91FF90EF90DF90CF90089580E122
:10B50000E4E7F6E0A2E9B6E001900D928A95E1F752
:10B510000895E1ECFAE7833021F0E82FF0E0E254FF
:10B52000F548849108954091A3105091A41090E0A3
:10B5300080E041155105B1F12091921230919312A2
:10B5400090E080E0F901EB55FF4EA081A23021F49C
:10B5500061817281860F971F4150510919F1F901DC
:10B56000E855FF4EA1919F01255A3041A111FACF14
:10B57000F901EB55FF4E2D3EA1E03A0730F4A191C1
:10B58000A111E0CF2F5F3F4FF6CF2D3EE1E03E0708
:10B59000C9F6E5EAF0E19F01255A3041A191AA23BD
:10B5A000D1F3D0CF0895982F9F7083FF0DC0809165
:10B5B0007B00886080937B0080917C00887F9770FF
:10B5C000892B80937C00089580917B00877FF2CF48
:10B5D00080919503909196034AE050E070E060E01E
:10B5E00001960F94DFD7862F08958091950390914F
:10B5F00096034AE050E070E060E001960F94DFD7D8
:10B60000CB01089580919503909196034AE050E014
:10B6100070E060E001960D94DFD780919B049091DB
:10B620009C0490939A048093990487E19DE69F93EC
:10B630008F9380917A0390917B03A0917C03B091CA
:10B640007D030196A11DB11DBF93AF939F938F936F
:10B6500085EA95E69F938F938CEA95E69F938F9367
:10B660000F9416DB8DB79EB70A960FB6F8949EBF5F
:10B670000FBE8DBF08950F931F93CF93DF93EC01FF
:10B68000C60FD71F8C179D0779F08C010F5F1F4FD6
:10B690000F9454DC8F3F31F081E0DF91CF911F9107
:10B6A0000F910895C801EECF80E0F7CF682F880F83
:10B6B000770B809192129091931288559F4E0F9420
:10B6C000ABE29C01909396038093950381E0232B3A
:10B6D00009F480E008950F931F93CF93DF938C01BB
:10B6E000862FEA010E94565B882319F10E94F55AC1
:10B6F0009C0197FF03C0319521953109253631050D
:10B700009CF09F938F938AE99AEA9F938F9383EBA0
:10B710009BE79F938F930F9416DB0F900F900F90E2
:10B720000F900F900F9080E0DF91CF911F910F91BC
:10B730000895F80180818823B1F3CE01DF91CF9184
:10B740001F910F910D9454DC60E086E69FE00F940A
:10B7500078DC60E088E69FE00F9478DC60E085E6C6
:10B760009FE00F9478DC60E084E69FE00F9478DC43
:10B7700060E082ED9EE00F9478DC60E08FEC9EE06C
:10B780000D9478DC80369105F8F440919212509136
:10B7900093122091A0103091A1104217530739F451
:10B7A0006091A3107091A410161617066CF0B901E1
:10B7B000680F791FFB01E359FF4F2417350730F459
:10B7C00081E04E175F0708F480E00895EE3EF140F7
:10B7D000F8F06C5F7F4F6E3E714018F449365105AA
:10B7E000B8F483599F4F4817590770F34DEE51E055
:10B7F000421B530B70E060E0C9018B559F4E0F94C4
:10B8000086E28FB7F8941092A1101092A0108FBF0B
:10B8100081E008952F923F924F925F926F927F92B4
:10B820008F929F92AF92BF92CF92DF92EF92FF9250
:10B830000F931F93CF93DF93CDB7DEB7CC58D24091
:10B840000FB6F894DEBF0FBECDBFCB58DD4F688377
:10B8500079838A839B83C557D240FE01E754FE4F0C
:10B8600088E2DF011D928A95E9F7E85BF1401F014C
:10B8700080E991E0DF01FC011D923197E9F7C75A99
:10B88000DD4F19821882C955D2409E012F513E4F7B
:10B89000C159DD4F39832883CF56D2408E01075AD4
:10B8A0001D4FCE018F5C9D4FC359DD4F9983888317
:10B8B000CD56D2403C01490140EBA42E4FE0B42EBE
:10B8C00053E2C52ED12CF12CE12CB6010D2C000C2D
:10B8D000880B990B0F94E2D6D4016D937D938D93D1
:10B8E0009D934D01F801619171918F01072E000C1C
:10B8F000880B990B0F94E2D6D3016D937D938D93B2
:10B900009D933D01BFEFEB1AFB0AE6E0EE16F10452
:10B9100009F038C3CB58DD4F288139814A815B81DA
:10B92000C557D240C159DD4FA881B981CF56D24009
:10B930006D917D918D919C910F9405E0412C512C3E
:10B94000320118160CF402C3C359DD4F0881198166
:10B95000CD56D2400C5E1F4FC159DD4FE880F980B3
:10B96000CF56D240B4E1EB0EF11C6E01EFEDCE1AD2
:10B97000EDEFDE0A9E012B553E4FCF58DD4F398348
:10B980002883C157D240D8014D905D906D907C9036
:10B99000F7016081718182819381D7015E914E911F
:10B9A0003E912E917D010F947BDD4B015C01F801EE
:10B9B00052914291329122918F01C301B2010F94B1
:10B9C0007BDDA50194010F947BDED6019E938E93BF
:10B9D0007E936E936D01CF58DD4FE881F981C15799
:10B9E000D240B292A29292928292CF58DD4FF983C6
:10B9F000E883C157D240C359DD4F28813981CD56E4
:10BA0000D2400217130709F0BECF4E013FE6831A5A
:10BA10003EEF930A5E0183EFA81A8DEFB80A610129
:10BA20008101EE24E394F12CD4014D905D906D9052
:10BA30007D904D012D913D914D915C91C301B201DD
:10BA40000F947CDD9B01AC010F947CDDF80164A7B1
:10BA500075A786A797A7F1E0EF16F10461F0D8016A
:10BA600098964D925D926D927C929B97F8014482DC
:10BA7000558266827782FFEFEF1AFF0AF501208177
:10BA800031814281538184E0A80EB11C64817581AB
:10BA9000868197810F947BDD20E030E040EC50E41C
:10BAA0000F9421D7D601DC966D937D938D939C9353
:10BAB000DF97045D1F4FB8E2CB0ED11CE5E0EE1618
:10BAC000F10409F0B1CF7E01FDE2EF0EF11C28E296
:10BAD000A22EB12C00EB1FEF24E0220E311CD70167
:10BAE0002D913D914D915C91139798966D917D911B
:10BAF0008D919C919B970F947BDE2B013C01610102
:10BB0000C01AD10A88248394912CF601E00FF11F0A
:10BB1000EA0DFB1D2081318142815381C301B201B5
:10BB20000F9421D79B01AC01F60160817181828164
:10BB300093810F947BDDD6016D937D938D939D93BF
:10BB40006D01BFEF8B1A9B0AE6E08E169104E9F6B1
:10BB50003CE2E30EF11C0852110988E2A80EB11C68
:10BB600008339FEF190709F0BACF1E01F5EB2F0E2E
:10BB7000311C6E0121EBC20ED11C7E0137E3E31AAA
:10BB80003EEFF30A04E010E04801B12CA12C412C57
:10BB9000512C3201F601EA0DFB1DD701AA0DBB1D88
:10BBA0002D913D914D915C91608171818281938154
:10BBB0000F9421D79B01AC01C301B2010F947CDD2E
:10BBC0002B013C018FEF881A980A94E0A90EB11C52
:10BBD000A5E08A169104F1F6A3019201F1016081BA
:10BBE0007181828193810F947BDDD6012D913D91EE
:10BBF0004D915C910F947BDEF701608371838283AA
:10BC0000938301501109F8E22F1A31082CE2C21A6D
:10BC1000D10834E0E31AF1080115110509F0B4CF99
:10BC2000CB50DE4F88819981AA81BB81C55FD1400D
:10BC3000CF57DD4F88839983AA83BB83C158D240F5
:10BC40001E0197E4291A9EEF390A10E000E0C1595D
:10BC5000DD4FA881B981CF56D240CD90DD90ED90D7
:10BC6000FD90C159DD4FB983A883CF56D240CB5840
:10BC7000DD4F288139814A815B81C557D240C70198
:10BC8000B6010F9471DE1816B4F0CB58DD4F288141
:10BC900039814A815B81C557D240C159DD4FE88166
:10BCA000F981CF56D24060817181828193810F9456
:10BCB00005E087FF18C00430110509F030C1CB58EA
:10BCC000DD4F288139814A815B81C557D240CF57EA
:10BCD000DD4F688179818A819B81C158D2400F9460
:10BCE00071DE87FF1CC1D10114968D909D90AD909F
:10BCF000BC9017978D919D910D90BC91A02DCF5820
:10BD0000DD4F88839983AA83BB83C157D240F80152
:10BD1000EE0FFF1FEE0FFF1F21E931E02C0F3D1F3B
:10BD2000E20FF31F4080518062807380C359DD4F62
:10BD3000A881B981CD56D2408D919D910D90BC9135
:10BD4000A02DC358DD4F88839983AA83BB83CD5729
:10BD5000D240A7019601CB58DD4F688179818A8155
:10BD60009B81C557D2400F947BDD6B017C0120E0A5
:10BD700030E040E450E40F94ECE0CB57DD4F6883B3
:10BD800079838A839B83C558D240C358DD4F28816D
:10BD900039814A815B81CD57D240C359DD4FE8815B
:10BDA000F981CD56D24064817581868197810F9447
:10BDB0007BDDA30192010F947BDEC758DD4F6883C2
:10BDC00079838A839B83C957D240A3019201C3011F
:10BDD000B2010F947CDDCF58DD4F288139814A8133
:10BDE0005B81C157D2400F9421D7C757DD4F68837D
:10BDF00079838A839B83C958D240A3019201C501EC
:10BE0000B4010F9421D79B01AC01C757DD4F688166
:10BE100079818A819B81C958D2400F947CDD20E0D2
:10BE200030E040EC50E40F947BDE9B01AC01C7583E
:10BE3000DD4F688179818A819B81C957D2400F94F7
:10BE40007BDDA70196010F9421D7C758DD4F68838A
:10BE500079838A839B83C957D240CF58DD4F28818D
:10BE600039814A815B81C157D240C501B4010F9429
:10BE70007BDD4B015C0120E030E040EC50E4C3018D
:10BE8000B2010F9421D79B01AC01C501B4010F94FD
:10BE90007BDECB57DD4F288139814A815B81C558D4
:10BEA000D2400F9421D74B015C0120E030E040E00C
:10BEB0005FE3CF58DD4F688179818A819B81C157CB
:10BEC000D2400F9421D72B013C01A7019601C70155
:10BED000B6010F9421D79B01AC01C301B2010F94AD
:10BEE00021D79B01AC01C501B4010F947CDD9B01FE
:10BEF000AC01C758DD4F688179818A819B81C95720
:10BF0000D2400F947CDDC358DD4F288139814A81AE
:10BF10005B81CD57D2400F947CDD2B013C010F5F3C
:10BF20001F4FF4E02F0E311CC359DD4F288139819A
:10BF3000CD56D2402C5F3F4FC359DD4F3983288304
:10BF4000CD56D2400530110509F081CEC301B201B2
:10BF5000C457DD4F0FB6F894DEBF0FBECDBFDF91E3
:10BF6000CF911F910F91FF90EF90DF90CF90BF90F6
:10BF7000AF909F908F907F906F905F904F903F9089
:10BF80002F900895C5010F9462DCD8018D939C9386
:10BF9000B5E0CB0ED11CE2E0AE0EB11C96CC0F93F7
:10BFA0001F93CF932091BA13213079F58C0180E54E
:10BFB0000E94565B882349F10E94E85AC82F8530B9
:10BFC00020F5013C82E0180749F0023C124069F07C
:10BFD0008C2FCF911F910F910D948DAD60E08C2F20
:10BFE000CF911F910F910D94D0AD8EEC9EE00F94E8
:10BFF00054DC882351F00F94BC88882331F08C2FB7
:10C00000CF911F910F910D944DAECF911F910F9134
:10C010000895CF93C82F0F94ED43F894C0938C06E6
:10C020000F94DC640E94AFF0880F82700F94652734
:10C030000F9447447894CF9108958F929F92AF9236
:10C04000BF92CF92DF92EF92FF920F931F93CF9305
:10C05000DF9300919503109196030F5F1F4F6801C6
:10C060008FEFC81AD80AD801DC918D2F90E00F9479
:10C07000E5D97C01892B01F5DD3201F56801B2E0DB
:10C08000CB0ED11CF801D181C1E08601015011090C
:10C0900043E050E065EF7AE7C8010F941BDA892B83
:10C0A000C1F460E070E080E89FEFC111DBC060E0A8
:10C0B00070E080E89FE7D6C08601D1CFDB3239F44B
:10C0C0006801F2E0CF0ED11CD8011196DC91C0E0DE
:10C0D000DCCF43E050E062EF7AE7C8010F941BDA4F
:10C0E000892B09F4CCC0F60110E000E020E030E03C
:10C0F000A9016F01D053DA3060F5BC2E6894B1F815
:10C100008C2F8870C2FF09C0811102C00F5F1F4FC2
:10C110003196D601DC91CB2DECCF882311F0015064
:10C120001109A5E0B0E00F94E9DC9B01AC01220FFE
:10C13000331F441F551F2D0F311D411D511D28391F
:10C14000B9E93B074B07B9E15B0710F3C660BC2EAA
:10C15000DFCFDE3F31F4C3FD33C0BC2E6894B3F8AB
:10C16000D7CFD53369F580818D3231F4C061BF01FD
:10C170006E5F7F4F818105C0BF018B32C9F36F5F56
:10C180007F4F80538A30E0F4FB01B0E8EB16BCE04F
:10C19000FB065CF4B701660F771F660F771FE60E8C
:10C1A000F71EEE0CFF1CE80EF11C819180538A30C3
:10C1B00060F3C4FF03C0F194E194F1080E0D1F1D5C
:10C1C000CA01B9010F94E0D6C370C33009F4905886
:10C1D0004B015C0120E030E0A9010F9471DE88235F
:10C1E00009F43EC0CEEEDAE717FF05C011950195C0
:10C1F0001109C6EDDAE76E01E8E1CE1AD10880E256
:10C20000E82EF12C0DC0FE012591359145915491F8
:10C210000E191F09C501B4010F9421D74B015C0110
:10C22000D501C4010E151F0574F72497F594E79402
:10C23000CC16DD06A9F78A2F880F8B2F881F8F3F1A
:10C2400049F020E030E0A901C501B4010F9471DE8E
:10C25000811106C082E290E0909315188093141823
:10C26000C501B401DF91CF911F910F91FF90EF9025
:10C27000DF90CF90BF90AF909F908F90089560E037
:10C2800070E080EC9FE7EECF2F923F924F925F924B
:10C290006F927F928F929F92AF92BF92CF92DF92D6
:10C2A000EF92FF920F931F93CF93DF9300D0CDB700
:10C2B000DEB78DEDC82E82E0D82E84E796E09B8312
:10C2C0008A8392E9E92E96E0F92E3324339400E034
:10C2D000F60181916F010E94565B282E882309F494
:10C2E000A6C01091E50313210E941D602B013C01A3
:10C2F000EA81FB814082518262827382033009F0BD
:10C3000046C0F1E0F983111101C0198280909302B7
:10C3100090909402A0909502B090960220E030E0B8
:10C3200040E85FE3C501B4010F9471DE882359F141
:10C33000111115C020919E0630919F064091A006D4
:10C340005091A106C301B2010F947BDD609380067A
:10C350007093810680938206909383062982A501BB
:10C36000940160918006709181068091820690917F
:10C3700083060F9421D76093800670938106809383
:10C38000820690938306E981E11103C022C0112344
:10C3900099F0F7012081318142815381EA81FB814B
:10C3A00060817181828193810F947CDDEA81FB81C0
:10C3B00060837183828393830F5F330C8A819B81B7
:10C3C00004969B838A8394E0E90EF11C043009F003
:10C3D0007FCF86E40E94565B882399F00E941D60FF
:10C3E0006B017C0120E030E0A9010F9405E01816F4
:10C3F00044F4C092B802D092B902E092BA02F0922C
:10C40000BB020F900F900F90DF91CF911F910F9172
:10C41000FF90EF90DF90CF90BF90AF909F908F9064
:10C420007F906F905F904F903F902F900895F7010D
:10C4300080819181A281B381EA81FB818083918394
:10C44000A283B383B9CF2F923F924F925F926F92A4
:10C450007F928F929F92AF92BF92CF92DF92EF9294
:10C46000FF920F931F93CF93DF93CDB7DEB76597FE
:10C470000FB6F894DEBF0FBECDBF698B7A8B8B8B66
:10C480009C8B49015A01302ECD8A2D2C81E080935E
:10C49000BE02DF922D892F931F92EF9287EE94E6D2
:10C4A0009F938F930F9416DB81E40E94565B0F904D
:10C4B0000F900F900F900F900F908823A1F0809114
:10C4C000950390919603FC012181283709F069C0FA
:10C4D00040E150E070E060E002960F94DFD7698B96
:10C4E0007A8B8B8B9C8B83E40E94565B882309F4A8
:10C4F00065C00E94025B2B013C01C988DA88EB8889
:10C50000FC888C149D04AE04BF0410F47501640112
:10C51000D301C2018C0D9D1DAE1DBF1D881699064D
:10C52000AA06BB0628F08C159D05AE05BF0530F4A4
:10C53000240135014C185D086E087F0888E50E94CB
:10C54000565B882309F491C020919503309196039E
:10C550002F5F3F4FFE01319610E000E04F01D901FF
:10C560008C912F5F3F4F882309F43FC000311105A4
:10C57000E1F18032A1F38A30C1F190ED980F9A3049
:10C5800010F58295807F9D012E5F3F4F11969C9103
:10C5900040ED490F4A30F8F4842B81930F5F1F4F11
:10C5A000DECF0E941D600F94EDDE9B01770F440BE0
:10C5B000550B298B3A8B4B8B5C8B95CF44244A943B
:10C5C000542C32019ACF9FE9980F963058F48295F7
:10C5D000807F8057D8CF4FE9490F463018F49755E0
:10C5E000892BDBCF1195019511092801012E000C33
:10C5F00066087708DA8AC98AB12CA12C0A151B05AE
:10C60000F1F0332039F031E0331671F04FEFA41A16
:10C61000B40AF4CFF401EA0DFB1D8081E989FA899F
:10C62000EA0DFB1D8083F2CFF401EA0DFB1D608152
:10C6300089899A898A0D9B1D0F949CDCE7CFFF9214
:10C64000EF92DF92CF922F925D895F937F926F92EC
:10C650005F924F928BEB94E69F938F930F9416DB30
:10C660000FB6F894DEBF0FBECDBF032DA30192011C
:10C67000C701B6010F94648765960FB6F894DEBFC4
:10C680000FBECDBFDF91CF911F910F91FF90EF9023
:10C69000DF90CF90BF90AF909F908F907F906F90E2
:10C6A0005F904F903F902F90089560911C1870916B
:10C6B0001D1890E08A3020F0895A9F4F0D94BCDA03
:10C6C000C096FCCF84FF18C08D9A85FF17C0A49A2E
:10C6D0002FB786FF15C0F89490910201906890934F
:10C6E00002012FBF87FF11C0A39A8F9A85E08A9518
:10C6F000F1F700008F9808958D98E7CFA498E8CFC0
:10C70000F894909102019F77EACFA398EECF0F9310
:10C710001F93CF93DF93C82FD62F8A0160FF15C0D8
:10C720005D9A8AE18A95F1F700C08C2F0E946263BE
:10C73000D1FD04C08C2F82950E946263C801DF91F5
:10C74000CF911F910F910C9461E95D98EACFCF9240
:10C75000DF92EF92FF92CF93DF93EC016A017B01AE
:10C760000F945CDC6F3F7F4F8F4F9F4F59F4B701A1
:10C77000A601CE01DF91CF91FF90EF90DF90CF9097
:10C780000D94AADCDF91CF91FF90EF90DF90CF90D6
:10C79000089580E1E2E9F6E0A3E7B2E001900D92AE
:10C7A0008A95E1F78091390290913A029093720351
:10C7B000809371038091B60D9091B70D9093AD0564
:10C7C0008093AC05809172068093AE058091E5035D
:10C7D00083FB882780F9809364058091E703809329
:10C7E000AB0581E08093A2060895CF93DF9380E2AA
:10C7F00097E10E94B1768EE595E1892B51F0C0E377
:10C80000D6E1A397CE010E94B17685E1CE35D80757
:10C81000C1F78BE395E10E94B17686E195E1DF9166
:10C82000CF910C94B176CF93DF93C2E9D6E020E0AC
:10C8300030E048EC51E46C857D858E859F850F94B2
:10C840007CDD6C877D878E879F8763E373E383E559
:10C8500090E4DF91CF910D9481C060E085EA9FE084
:10C860000F9478DC60E08FE79CE00F9478DC80E048
:10C8700090E0A0E8BFEB8093830290938402A093A2
:10C880008502B093860282E080936A021092A90D1D
:10C8900008958091AC059091AD052091B60D309131
:10C8A000B70D2817390771F09093B70D8093B60D27
:10C8B00081E08093E3030F94512A0F941C8382E05C
:10C8C0008093E30308958091A90D882341F080911E
:10C8D000390290913A029093720380937103089504
:10C8E0008091A1059091A205009729F12091A80DB2
:10C8F000211121C02091A70D21111DC0FC01E85A72
:10C90000FF4F20E1A3E8B2E001900D922A95E1F7F4
:10C91000FC01E659FF4F2081318130935F05209360
:10C920005E0588599F4FFC018081918190936A0533
:10C9300080936905089580E090E0A0E8BFEB8093C4
:10C94000830290938402A0938502B0938602609143
:10C95000B8027091B9028091BA029091BB020F9413
:10C96000F4DE70935F0560935E0510926A05109285
:10C9700069050895CF92DF92EF92FF928091901413
:10C980008823D9F18091820390918303A09184033D
:10C99000B09185038093600590936105A093620533
:10C9A000B09363050F946A64C0906005D0906105F0
:10C9B000E0906205F0906305C81AD90AE108F10811
:10C9C000C0926005D0926105E0926205F092630525
:10C9D0000E94935AC81AD90AE108F108C09260056A
:10C9E000D0926105E0926205F092630510926A02AE
:10C9F000FF90EF90DF90CF90089580910E058823EF
:10CA0000B1F180917A0390917B03A0917C03B09166
:10CA10007D038093600590936105A0936205B093B8
:10CA200063050F946A6440916005509161056091BF
:10CA3000620570916305481B510961097109809174
:10CA4000A3109091A410092E000CAA0BBB0B481B3D
:10CA5000590B6A0B7B0B4093600550936105609303
:10CA600062057093630581E080936A02C1CF82E022
:10CA7000FBCFCF92DF92EF92FF92C090560ED090F4
:10CA8000570EE090580EF090590E8091550E882365
:10CA900009F44EC020E030E0A901C701B6010F94AF
:10CAA00005E018160CF044C02BED3FE049E450E4DB
:10CAB000C701B6010F9421D7A70196010F9421D782
:10CAC00020E030E040E85EE30F9421D79B01AC0109
:10CAD00060E070E080E89FE30F947BDE6B017C01F7
:10CAE0006091BC027091BD0264367105A1F0072E01
:10CAF000000C880B990B0F94E2D62AE037ED43E245
:10CB00005CE30F9421D79B01AC01C701B6010F94E0
:10CB100021D76B017C01C0929302D0929402E092E3
:10CB20009502F0929602FF90EF90DF90CF900895DB
:10CB3000C12CD12C80E8E82E8FE3F82ED1CF8F9234
:10CB40009F92AF92BF92CF92DF92EF92FF9281EFCE
:10CB50009FE00F94987B6B017C018DEE9FE00F941A
:10CB6000987B4B015C010F94A83F2CE330E040E040
:10CB700050E00F94C7DCBA01A901480D591D6A1D88
:10CB80007B1D8DEE9FE00F948ADC609165067091AD
:10CB90006606809167069091680628EE33E040E0D3
:10CBA00050E00F94C7DCBA01A9014C0D5D1D6E1D4C
:10CBB0007F1D81EF9FE00F948ADC0F9477431092E2
:10CBC00065061092660610926706109268068091BC
:10CBD000BA13813081F46091BE137091BF1390E05D
:10CBE00080E00F94807B1092BF131092BE131092BE
:10CBF000C1131092C013FF90EF90DF90CF90BF90C1
:10CC0000AF909F908F9008958091E7031F928F932C
:10CC100080916B031F928F93E9ECF3E04281538183
:10CC20002CE3249FC001259F900D11249F938F9387
:10CC300040815181249FC001259F900D11249F9315
:10CC40008F938EE795E69F938F930F9416DB8DB7A6
:10CC50009EB70A960FB6F8949EBF0FBE8DBF08957B
:10CC6000CF93C82F8FEF9FE00F9454DC813021F0D9
:10CC700080918C06813029F481E08C27CF910C942F
:10CC80000960CF91089586E893E00D94F42C20E09C
:10CC900030E040E752E40F947BDE08951092B70233
:10CCA0004091660350916703609168037091690336
:10CCB0004093B8025093B9026093BA027093BB02DA
:10CCC00090933A028093390286E893E00D94F42C15
:10CCD0001F93CF93DF93182F8091B8029091B902E0
:10CCE000A091BA02B091BB02809366039093670350
:10CCF000A0936803B0936903C0913902D0913A02BE
:10CD000084E690E090933A028093390286E893E0BB
:10CD10000F94F42C1093B702CE01DF91CF911F91A5
:10CD2000089540E050E0BA018DEE9FE00F948ADC58
:10CD300040E050E0BA0181EF9FE00F948ADC0E944E
:10CD4000A45B70E060E085E09FE00F9496DC70E00B
:10CD500060E083E09FE00F9496DC70E060E081E0AB
:10CD60009FE00F9496DC70E060E08FEF9EE00F9400
:10CD700096DC70E060E083ED9EE00F9496DC70E05E
:10CD800060E080ED9EE00F9496DC40E050E0BA0158
:10CD900088EA9CE00D948ADCF89488E198E00FB66C
:10CDA000F894A895809360000FBE90936000FFCF29
:10CDB000C82F9FB7F894E2E0F1E08081846080831F
:10CDC0009FBF6C2F83E09DE00F9478DC8C2F0E9436
:10CDD0009AEE0E94CC661F920F920FB60F9211240A
:10CDE00083E00E94D8661F920F920FB60F92112413
:10CDF00082E00E94D86685EA9FE00F9454DC91E0BF
:10CE0000811101C090E0892F08958091E403811180
:10CE100006C081E090919D03923009F080E0089572
:10CE20008091901481110AC080910E05811106C075
:10CE300081E090919D03913009F080E00895CF93B7
:10CE4000DF93C091A70DC1111FC08091A80D811162
:10CE50001CC00E940567811118C0D091B40DD43058
:10CE600061F48091B60D9091B70D892B91F480916A
:10CE7000720690917306892B61F40E941067C82F87
:10CE8000811103C0C1E0D111C0E08C2FDF91CF919F
:10CE90000895C1E0FACF0E941F67882389F020E03F
:10CEA00030E040E050E460919A0670919B068091DA
:10CEB0009C0690919D060F9471DE881F8827881F1D
:10CEC00008950E941067811118C00E9405678111A2
:10CED00014C08091A90D811110C08091B40D8111F1
:10CEE0000BC08091BB13811107C08091A70D8111E8
:10CEF00004C08091A80D089581E00895FC0120816F
:10CF0000211101C06695FC0162830895FC016183D3
:10CF100021E0603208F020E09081291781F08281C1
:10CF2000992351F090E095958795828370E07595EF
:10CF30006795618320830895880F8283FBCF211139
:10CF400004C070E0759567956183089520919212F1
:10CF500030919312BC01C90188559F4E0F945BDA42
:10CF60009C01909396038093950381E0232B09F411
:10CF700080E0089580E1E2E9F6E0A4E7B6E0019000
:10CF80000D928A95E1F708954F925F926F927F928A
:10CF90008F929F92AF92BF92CF92DF92EF92FF92C9
:10CFA0000F931F93CF93DF9300D000D01F921F9257
:10CFB000CDB7DEB72091A90D222309F473C12091CA
:10CFC000E603223009F46EC12091E603213011F40A
:10CFD0001092E6032B013C011092E7031091AE057D
:10CFE0006091EE047091EF048091F0049091F1044F
:10CFF0000F94F4DE611731F0812F90E09093730667
:10D00000809372060E9449648091AB058093E70388
:10D010009091E5038091640581958927887089271F
:10D020008093E503A301920160917F0270918002D9
:10D0300080918102909182020F947BDD6D837E83CB
:10D040008F839887CE0105960F94F9641092380269
:10D0500020E030E040E85FEB609173027091740271
:10D0600080917502909176020F9471DE811120C03B
:10D070008091920690919306A0919406B0919506A6
:10D080008093730290937402A0937502B09376021A
:10D090008091960690919706A0919806B091990676
:10D0A0008093770290937802A0937902B0937A02EA
:10D0B000A301920160917F027091800280918102B0
:10D0C000909182020F947BDD69837A838B839C83AA
:10D0D000E0909A06F0909B0600919C0610919D06A8
:10D0E00020917702309178024091790250917A0232
:10D0F0006091730270917402809175029091760232
:10D100001F921F921F921F92E2E68E2EE7E29E2E42
:10D11000E6E7AE2EE2E4BE2EFE0131966F010F94DB
:10D120002CB1A301920160917F02709180028091E5
:10D130008102909182020F947BDD69837A838B83D5
:10D140009C83E0907B02F0907C0200917D02109124
:10D150007E022091770230917802409179025091BD
:10D160007A026091730270917402809175029091BD
:10D1700076021F921F921F921F920F942CB1E09083
:10D180007B02F0907C0200917D0210917E02209142
:10D190007702309178024091790250917A02609141
:10D1A00073027091740280917502909176021F92C1
:10D1B0001F921F921F92812C912CF8EEAF2EF2E459
:10D1C000BF2EAFE7CA2EA2E0DA2E0F942CB10F9437
:10D1D000ED4311E01093380260915E0570915F0598
:10D1E00090E080E00F94E0D66093B8027093B902AB
:10D1F0008093BA029093BB02809171039091720365
:10D2000090933A028093390280E1E3E7F2E0A2E9E9
:10D21000B6E001900D928A95E1F70E94BA6780917D
:10D220006A020FB6F894DEBF0FBECDBF811151C0A8
:10D230006091600570916105809162059091630530
:10D240006093A4177093A5178093A6179093A717C0
:10D250000F94D7768091600590916105A091620549
:10D26000B09163058093820390938303A09384031A
:10D27000B09385031093901460E085EA9FE00F94CB
:10D2800078DC60E08FE79CE00F9478DC8FEC9FE621
:10D290000E943BF282E080936A021092A90D81E025
:10D2A0008093AC0D28960FB6F894DEBF0FBECDBFAD
:10D2B000DF91CF911F910F91FF90EF90DF90CF9072
:10D2C000BF90AF909F908F907F906F905F904F90A6
:10D2D0000895813089F68091600590916105A09153
:10D2E0006205B091630580937A0390937B03A093CA
:10D2F0007C03B0937D0310929F1010929E100E94A9
:10D300000D5BBACF3F924F925F926F927F928F9256
:10D310009F92AF92BF92CF92DF92EF92FF920F93C4
:10D320001F93CF93DF9330900F18332009F480C000
:10D330008B01EC0131FE54C088809980AA80BB80AB
:10D34000FB01C080D180E280F3802091E41730910E
:10D35000E5174091E6175091E717C501B4010F9406
:10D3600021D72B013C012091E8173091E91740911A
:10D37000EA175091EB17C701B6010F9421D79B0113
:10D38000AC01C301B2010F947CDD2B013C01209163
:10D39000DC173091DD174091DE175091DF17C50182
:10D3A000B4010F9421D74B015C012091E01730911B
:10D3B000E1174091E2175091E317C701B6010F94AE
:10D3C00021D79B01AC01C501B4010F947CDD6883BA
:10D3D00079838A839B83F8014082518262827382BF
:10D3E00030FE26C020910718309108184091091886
:10D3F00050910A18688179818A819B810F947CDD24
:10D40000688379838A839B8320910B1830910C1851
:10D4100040910D1850910E18F80160817181828140
:10D4200093810F947CDDF801608371838283938301
:10D43000DF91CF911F910F91FF90EF90DF90CF90F0
:10D44000BF90AF909F908F907F906F905F904F9024
:10D450003F9008952F923F924F925F926F927F92EA
:10D460008F929F92AF92BF92CF92DF92EF92FF92F4
:10D470000F931F93CF93DF9300D000D01F921F9282
:10D48000CDB7DEB78C011B01FC0180819181A281A7
:10D49000B38189839A83AB83BC83FB0180819181B3
:10D4A000A281B3818D839E83AF83B887BE016B5FFA
:10D4B0007F4FCE0101960E948269C980DA80EB809D
:10D4C000FC8020E030E0A901C701B6010F9471DEB5
:10D4D00087FF35C019821A821B821C82FF24F394B5
:10D4E0008D809E80AF80B88420E030E040E850EC32
:10D4F000C501B4010F9471DE87FF35C080E090E074
:10D50000A0E8B0EC8D839E83AF83B887CD80DE80AA
:10D51000EF80F88489809A80AB80BC8070900F186F
:10D5200071104CC0F80180829182A282B382F10115
:10D53000C082D182E282F382FF24F39425C020E0EE
:10D5400030E04FE753E4C701B6010F9405E0F12C3A
:10D55000181634F680E090E0AFE7B3E489839A834D
:10D56000AB83BC83BBCF20E030E844E553E4C50186
:10D57000B4010F9405E018162CF480E090E8A4E5BF
:10D58000B3E4C0CFF110C2CF8F2D28960FB6F89418
:10D59000DEBF0FBECDBFDF91CF911F910F91FF90E6
:10D5A000EF90DF90CF90BF90AF909F908F907F9043
:10D5B0006F905F904F903F902F90089570FE1CC029
:10D5C00020910718309108184091091850910A18B5
:10D5D000C501B4010F947BDD4B015C0120910B1858
:10D5E00030910C1840910D1850910E18C701B601DA
:10D5F0000F947BDD6B017C0171FE9ECF2091F717AC
:10D600003091F8174091F9175091FA17C501B401FC
:10D610000F9421D72B013C012091FB173091FC176F
:10D620004091FD175091FE17C701B6010F9421D705
:10D630009B01AC01C301B2010F947CDDF801608352
:10D640007183828393832091FF173091001840915A
:10D65000011850910218C501B4010F9421D74B0154
:10D660005C012091031830910418409105185091E5
:10D670000618C701B6010F9421D79B01AC01C50163
:10D68000B4010F947CDDF101608371838283938305
:10D6900053CFCF92DF92EF92FF92CF93DF93EC01C3
:10D6A000BC016C5F7F4F0E942A6AC0902902D09013
:10D6B0002A02E0902B02F0902C02A70196016885C7
:10D6C00079858A859B850F9471DE87FF04C0C886A3
:10D6D000D986EA86FB86C0901D02D0901E02E0909B
:10D6E0001F02F0902002A7019601688579858A853E
:10D6F0009B850F9405E0181624F4C886D986EA861F
:10D70000FB86DF91CF91FF90EF90DF90CF9008954F
:10D710002F923F924F925F926F927F928F929F9241
:10D72000AF92BF92CF92DF92EF92FF920F931F932F
:10D73000CF93DF93CDB7DEB7A2970FB6F894DEBFD5
:10D740000FBECDBF1C0184E796E00E94496B86E8BE
:10D7500093E00F94F42C40909206509093066090C2
:10D76000940670909506C0907406D0907506E0906F
:10D770007606F0907706A7019601C301B2010F94D7
:10D7800071DE81113FC02091780630917906409179
:10D790007A0650917B06609196067091970680916B
:10D7A0009806909199060F9471DE81112BC020E0AC
:10D7B00030E040E752E46091B8027091B902809184
:10D7C000BA029091BB020F947BDE0F944EC00E9470
:10D7D0007F5AA2960FB6F894DEBF0FBECDBFDF9181
:10D7E000CF911F910F91FF90EF90DF90CF90BF905E
:10D7F000AF909F908F907F906F905F904F903F90F1
:10D800002F9008956091390270913A02072E000C12
:10D81000880B990B0F94E2D62091B8023091B9028F
:10D820004091BA025091BB020F9421D72EE333EC02
:10D830004EE259E30F9421D76F83788789879A87BF
:10D840008091C213882309F40FC1A3019201C7017B
:10D85000B6010F947BDD2B013C012091960630919F
:10D8600097064091980650919906609178067091BC
:10D87000790680917A0690917B060F947BDD6B8709
:10D880007C878D879E87C301B2019F772B853C855E
:10D890004D855E855F770F947CDD6B017C0120E018
:10D8A00030E0A9010F9405E018160CF0DDC020E06F
:10D8B00030E040EF51E4C701B6010F947BDE0F94D6
:10D8C0005ADE0F94F4DE7E836D836230710508F4B6
:10D8D000CBC02114310409F4C7C020919A063091BD
:10D8E0009B0640919C0650919D0660917C0670912C
:10D8F0007D0680917E0690917F060F947BDD6F8779
:10D90000788B898B9A8B20919E0630919F0640914F
:10D91000A0065091A10660918006709181068091C9
:10D920008206909183060F947BDD6B8B7C8B8D8BB5
:10D930009E8BAD81BE81CD01B0E0A0E08F8F98A31A
:10D94000A9A3BAA32D813E812216330608F08CC00C
:10D95000B10190E080E00F94E0D66B017C016F8D07
:10D9600078A189A19AA10F94E0D69B01AC01C701CF
:10D97000B6010F947BDE6B017C01AC019B016B89CE
:10D980007C898D899E890F9421D79B01AC01609180
:10D990009E0670919F068091A0069091A1060F941B
:10D9A0007CDD69837A838B839C83A70196016F85D5
:10D9B000788989899A890F9421D720919A06309184
:10D9C0009B0640919C0650919D060F947CDD6F8BC9
:10D9D000788F898F9A8FA70196016B857C858D85BD
:10D9E0009E850F9421D720919606309197064091FD
:10D9F0009806509199060F947CDD6B8F7C8F8D8FEC
:10DA00009E8FA7019601C301B2010F9421D72091E7
:10DA100092063091930640919406509195060F948A
:10DA20007CDD3F922F92A2E9B6E0BF93AF938F8047
:10DA30009884A984BA84DE0111966D01EF88F88C70
:10DA4000098D1A8D2B8D3C8D4D8D5E8D0F942CB1D3
:10DA50000F900F900F900F908091AC0D8111B7CE69
:10DA6000BFEF2B1A3B0A6ECFE0907C06F0907D064C
:10DA700000917E0610917F062091780630917906FC
:10DA800040917A0650917B066091740670917506FC
:10DA900080917606909177061F921F92E2E9F6E058
:10DAA000FF93EF938F809884A984BA84E0E8CE2E08
:10DAB000E6E0DE2E0F942CB10F900F900F900F9098
:10DAC00086CECF92DF92EF92FF92CF939B01AC0173
:10DAD000C0909A06D0909B06E0909C06F0909D0620
:10DAE000C701B6010F947CDD60939A0670939B0684
:10DAF00080939C0690939D0683B19091910691111D
:10DB000002C084FF26C082E996E00E94496BE09142
:10DB10007102F091720260857185828593850F9400
:10DB200081C00F94ED43A701960160919A06709110
:10DB30009B0680919C0690919D060F947BDD6B0166
:10DB40007C01C701B601CF91FF90EF90DF90CF909D
:10DB5000089515980F94ED4381E00F94E74EC82F78
:10DB600084E00F94DD2665E575E585E591E40F9485
:10DB700081C00F94ED4382E00F94D943A701960131
:10DB80000F947BDD6B017C010F94F54E882391F09F
:10DB900080911D0290911E02A0911F02B09120025F
:10DBA00080939A0690939B06A0939C06B0939D0643
:10DBB0000F9441BF0F94AE268C2F0F94E74EC1CF28
:10DBC0008F929F92AF92BF92CF92DF92EF92FF928D
:10DBD0004B015C01C0909A06D0909B06E0909C0699
:10DBE000F0909D06AC019B01C701B6010F9405E0C2
:10DBF00087FF11C0A5019401C701B6010F947BDD19
:10DC00009F77FF90EF90DF90CF90BF90AF909F9065
:10DC10008F900C94616DFF90EF90DF90CF90BF904C
:10DC2000AF909F908F900895EEE5F3E09FE781918C
:10DC30008F3731F0DF01119787FF07C08F778C9303
:10DC400083E0E636F80799F708959C93F9CF909111
:10DC50006D02981710F480936D0280916E028823F4
:10DC600039F0E0911504F0911604309709F01994F9
:10DC70000895CF93DF93CDB7DEB7AE014A5F5F4F14
:10DC8000FA0161917191AF0183E094E00F949BDB05
:10DC9000DF91CF91089563E074E00D94ECDA63E0D6
:10DCA00074E0082E000C990B0D94BCDACF93C82FAA
:10DCB000C15020F080E20E944F6EFACFCF910895BC
:10DCC000CF93C82F862F643008F083E080935D03E4
:10DCD0000E94895A8C0F80935C0344E650E060E018
:10DCE0008068CF910C948763CF93DF93EA010E9401
:10DCF000606E63E074E0CE01DF91CF910D94ECDAB9
:10DD0000CF93C42F0E94606E63E074E08C2FCC0F21
:10DD1000990BCF910D94BCDA60E080E00E94606EB8
:10DD200010925C03089540E456E060E081E00E94B8
:10DD3000876310925D0310925C0348E050E06FE748
:10DD400070E08EE593E00D9486E290916E02981754
:10DD500009F180936E028823E9F010927106109207
:10DD600070061092D1058CED93E00F94F42C0F9473
:10DD7000512A61507109810991096093D803709308
:10DD8000D9038093DA039093DB030E94936E82E0C1
:10DD90000C94276E0895CF93C82F10925D031092B4
:10DDA0005C0348E050E06FE770E08EE593E00F948D
:10DDB00086E244E951E162E080E30E94876346E93C
:10DDC00050E062E080E30E94876346E950E062E051
:10DDD00080E30E94876346E950E062E080E20E94AF
:10DDE00087638091110444E650E060E080620E9405
:10DDF000876384E080935B0344E650E060E08CE05E
:10DE00000E948763C1110E94936E44E650E060E077
:10DE100086E0CF910C94876381E00C94CB6ECF9217
:10DE2000DF92FF920F931F93CF93DF9300D000D028
:10DE30001F921F92CDB7DEB78A30D9F480915D036F
:10DE4000843018F08FEF80935D0360915D036F5F06
:10DE500080E00E94606E28960FB6F894DEBF0FBE79
:10DE6000CDBFDF91CF911F910F91FF90DF90CF90A9
:10DE7000089590E8980F44E650E061E09A3408F580
:10DE8000482F4058550B9A0196E0929FA001939F0E
:10DE9000500D1124FA01E95FF648F490EEE5F3E045
:10DEA00030E020E09FEF6191782F76277F7789F42B
:10DEB000F901E25AFC4F8083F22E44E650E061E023
:10DEC0008F2D0E94876380915C038F5F80935C033A
:10DED000C2CF6F3709F03CC0F901E25AFC4F808392
:10DEE000922FF92EFA01EE5FF6488E010F5F1F4F59
:10DEF000D801959188E0182E10FE05900294802D8F
:10DF00009795881F8D931A94B9F7BF2DE8E0BE024C
:10DF1000C001112444E650E060E080640E94876301
:10DF20006E01F9E0CF0ED11C44E650E061E0D8016B
:10DF30008D918D010E948763C016D106A9F780914B
:10DF40005C0344E650E060E080680E948763B5CFE0
:10DF500067FF922F2F5F3F4F2830310509F0A3CF85
:10DF60009F3F09F0BECFA9CF8F929F92AF92BF92F1
:10DF7000EF92FF920F931F93CF93DF93CDB7DEB74E
:10DF8000A0970FB6F894DEBF0FBECDBF6115710527
:10DF90008105910599F480E3A0960FB6F894DEBF51
:10DFA0000FBECDBFDF91CF911F910F91FF90EF90EA
:10DFB000BF90AF909F908F900C940F6F00E0842ED5
:10DFC000912CB12CA12C9E012F5F3F4F7901A5010F
:10DFD00094010F94C7DCF701E00FF11D6083B901D4
:10DFE000CA010F5F611571058105910581F70E0D5D
:10DFF0001F2D111DE016F10659F0F80182918F01D5
:10E000008A3020F4805D0E940F6FF4CF895CFBCFD3
:10E01000A0960FB6F894DEBF0FBECDBFDF91CF91B3
:10E020001F910F91FF90EF90BF90AF909F908F90B6
:10E030000895CF92DF92EF92FF926B017C01F7FE81
:10E040000BC08DE20E940F6FF094E094D094C094C6
:10E05000C11CD11CE11CF11C4AE0C701B601FF90B4
:10E06000EF90DF90CF900C94B46F0F931F93CF93EA
:10E070008C01C62FCC2359F0F8012491222339F0CA
:10E080000F5F1F4F84910E940F6FC150F3CF8C2FF1
:10E090000E94566E8C2FCF911F910F9108950F9370
:10E0A0001F93CF938C01C62FCC2349F0F8018191A7
:10E0B0008F01882321F00E940F6FC150F5CF8C2F64
:10E0C0000E94566E8C2FCF911F910F910895CF9380
:10E0D000DF93EC018991882319F00E940F6FFACF2A
:10E0E000DF91CF9108950E940F6F90E080E0089536
:10E0F0001092A8031092D4050895CF938091A8039D
:10E10000C1E0811104C0C0E08C2FCF9108950E941E
:10E110007870FACFE0E0F1E085919591A591B49106
:10E12000853A9A45A44BBB4429F4EAE0F1E0859195
:10E13000949108958FE39FE308958EEF9FE00F94ED
:10E1400054DC8E3F39F091E020915A03281390E07F
:10E15000892F089580E0089510925A036EEF8EEF94
:10E160009FE00D9478DC853728E6920709F459C0C2
:10E17000F8F48E3625E6920709F459C050F4833737
:10E1800023E69207B1F185369446B1F18CEF94E61F
:10E190000895823726E6920791F1823728E69207A2
:10E1A00009F442C08337954689F783E595E60895DB
:10E1B0008C3620E7920731F170F48C362EE6920708
:10E1C00021F18F362EE6920731F184379946F1F628
:10E1D00081E495E608958B3623E79207F9F08637B8
:10E1E00023E79207A9F08F36924781F68FEF94E6E6
:10E1F000089583E695E608958BE595E608958AE40B
:10E2000095E608958AE395E608958FE295E60895E8
:10E2100087E295E6089581E295E6089586E195E620
:10E2200008958FE095E6089586E095E608958BE6DB
:10E2300095E60895CF92DF92EF92FF921F93CF93CE
:10E24000DF93CDB7DEB760970FB6F894DEBF0FBE91
:10E25000CDBF8823C1F1182F813081F40E948A70CC
:10E2600060960FB6F894DEBF0FBECDBFDF91CF91A1
:10E270001F91FF90EF90DF90CF9008958CE58CBDBB
:10E280001DBC1150C12CD12C760120E130E0AE0133
:10E290004F5F5F4FC701B6010E94C5ED89819A812A
:10E2A000AB81BC81853A9A45A44BBB4479F41150AB
:10E2B00019F48B859C85D4CF8D819E81C80ED91E83
:10E2C000E11CF11CE2CF8EE695E6CACF8FE39FE317
:10E2D000C7CFCF92DF92EF92FF921F93CF93DF933E
:10E2E000CDB7DEB760970FB6F894DEBF0FBECDBFD7
:10E2F000EEEFF8E785919591A591B49111E08F3FEC
:10E300009F4FAF4FBF4F09F18CE58CBD1DBCC12C99
:10E31000D12C760112E020E130E0AE014F5F5F4F7B
:10E32000C701B6010E94C5ED89819A81AB81BC818C
:10E33000853A9A45A44BBB4441F48D819E81C80E19
:10E34000D91EE11CF11C1F5FE6CF812F60960FB62E
:10E35000F894DEBF0FBECDBFDF91CF911F91FF902C
:10E36000EF90DF90CF9008950F931F93CF93C82F16
:10E37000811106C0109259031092580310925A034B
:10E380008C2F0E941A718C010E948A70081719073D
:10E3900019F0C13009F03EC0E0E0F1E085919591BF
:10E3A000A591B491853A9A45A44BBB4409F031C07C
:10E3B000E4E0F1E065917491E8E0F1E04591549179
:10E3C00030E020E090E080E06217730789F5841B5D
:10E3D000950B98278927982748175907D1F4ECE01F
:10E3E000F1E04591559165917491EEEFF8E78591D3
:10E3F0009591A591B491481759076A077B0749F48D
:10E4000080E091E0909359038093580381E08093DA
:10E410005A03C1E080915A038C131CC06C2F8EEFFD
:10E420009FE00F9478DC81E0CF911F910F910895C8
:10E43000F901E050FF4FE491F0E0A8E020FDA0E0FA
:10E4400002C0EE0FFF1FAA95E2F78E0F9F1F2F5FEE
:10E450003F4FBACF80E0E8CF20915A03211104C08A
:10E46000FC013296CF010895409158035091590311
:10E4700041155105A9F3FC01259134912F3F320735
:10E4800079F3F9013896EE0FFF1FE40FF51F259180
:10E490003491FA01E20FF31F2491222309F3E2CF12
:10E4A000CF93DF93EC0120E030E04CE852E4609140
:10E4B0009E0670919F068091A0069091A1060F94F0
:10E4C0007CDD60939E0670939F068093A0069093D8
:10E4D000A10660E070E080EA91E40F9481C00E94A0
:10E4E00013640E94936E85E79BE50E942C72AC0139
:10E4F00060E080E00E94746E8881882339F061E0DA
:10E5000080E00E94606ECE010E94677089E999E305
:10E510000E942C72AC0162E080E00E94746E83E481
:10E520009BE20F947421DF91CF910D94ED430F94F2
:10E53000F4758F3F11F180E00E94A56E0E94936EEA
:10E540008CE392E50E942C72AC0161E080E00E94B5
:10E55000746E80E20E940F6F0F94F475682F70E064
:10E560006F5F7F4F072E000C880B990B0E9419706C
:10E570000F9475AD81E00C94A56E08954F925F9253
:10E580006F927F928F929F92AF92BF92EF92FF9283
:10E590000F931F93CF93DF930E94936E82E39DE4CA
:10E5A0000E942C72AC0161E080E00E94746ED091F8
:10E5B000B70281E08093B702ECE8FBE7C49184E006
:10E5C0000F94DD2682E9E82E86E0F82EF70110860A
:10E5D0001186128613860F9441BF0E94BA67E6E83F
:10E5E000FBE785909590A590B49004E716E08C2FFA
:10E5F000992781950CF49095BC01072E000C880B8F
:10E60000990B0F94E2D62B013C012DEC3CEC4CE82D
:10E610005FE3C501B4010F9421D79B01AC01C30195
:10E62000B2010F9421D7F8012085318542855385A9
:10E630000F947CDDF801608771878287938780E083
:10E6400090E0A8E4B4E48093B8029093B902A09358
:10E65000BA02B093BB0265E575E585E591E40F94D8
:10E660004EC00F94ED430F94AE261092B702F701FF
:10E6700010861186128613860F9441BF0E94BA67D6
:10E68000F6EFCF02B0011124072E000C880B990B76
:10E690000F94E2D69B01AC01F801608571858285FB
:10E6A00093850F947CDDF80160877187828793875B
:10E6B00080E090E0A8ECB3E48093B8029093B902B4
:10E6C000A093BA02B093BB0265E575E585ED90E4D1
:10E6D0000F944EC00F94ED43D093B70280E090E0CA
:10E6E000A4E5B3E4F70180879187A287B3870F94ED
:10E6F00041BF81E0DF91CF911F910F91FF90EF908B
:10E70000BF90AF909F908F907F906F905F904F9051
:10E710000895CF93DF93EC0160FF03C028E52883C1
:10E72000219661FF03C029E52883219680E2899321
:10E7300080E096E30E942C72BC01CE01DF91CF9164
:10E740000D940BDA1F920F920FB60F9211240BB695
:10E750000F922F938F939F93EF93FF93E091530327
:10E76000E830E8F4F0E08827E754FC488F4F0D9438
:10E7700064DDC173DB73E673F4730A741374367467
:10E78000487480918D0681110AC080911D06880F02
:10E7900080935203882319F081E080935303FF9103
:10E7A000EF919F918F912F910F900BBE0F900FBE05
:10E7B0000F901F901895809151038F5F80935103A4
:10E7C00090915203981758F382E0E7CF83E080934B
:10E7D00053038FE0809350038FEF86BD81E085BDAA
:10E7E00084B58F7E84BDDBCF809150038295807F7E
:10E7F000819588BD80915003882321F081508093BA
:10E800005003CDCF84E0809353038FEF88BD8EEF0C
:10E8100086BDC5CF85E0809353038FEF88BD86BD4D
:10E8200082E085BDBCCF2FEF28BD80918D06811180
:10E83000B6CF809151038F5F809351039091520323
:10E84000891708F4ACCF80911D0690E08F379105B1
:10E850000CF0A5CF86E0809353038FE080935003A4
:10E8600026BD81E085BD84B58061BCCF8091500319
:10E870008295807F819588BD809150038111BECFA4
:10E8800087E08093530380E886BD8FEF88BD87CFF4
:10E890001092530380E886BD8FEF88BDC1CFCF9320
:10E8A000C82F682F87E69FE00F9478DCCC2319F0FF
:10E8B000CF910D94747C1092AA171092B617CF9135
:10E8C000089510926F060F94512A6093C0177093A9
:10E8D000C1178093C2179093C31708951F920F9288
:10E8E0000FB60F9211242F934F935F936F937F93E3
:10E8F0008F939F93AF93BF9380916F068823F1F01E
:10E900008091A6048B34D0F080916A0086FF24C0E9
:10E9100080913B0690913C06A0913D06B0913E0649
:10E920008093490390934A03A0934B03B0934C0305
:10E9300080916A0090E4892780936A00BF91AF912B
:10E940009F918F917F916F915F914F912F910F9038
:10E950000FBE0F901F90189580913B0690913C063A
:10E96000A0913D06B0913E064091490350914A0363
:10E9700060914B0370914C03841B950BA60BB70B56
:10E980002091E70344E050E060E070E0253620F09D
:10E9900043E050E060E070E084179507A607B707F2
:10E9A00038F28091E4059091E50502969093E50593
:10E9B0008093E405BDCF80934D0380FD1CC0109271
:10E9C0006B0320916B038FEF820F8E3FE8F08091F5
:10E9D000A000877F8093A0001092AD001092AC0041
:10E9E0009FB7222361F0F8948091020180628093A6
:10E9F00002019FBF08958FEF80936B03E2CFF894DD
:10EA0000809102018F7DF3CFEFB7F8948091A00041
:10EA100088608093A00030E0809172004FEF50E05A
:10EA200081FF04C04091A8005091A900249FC0011B
:10EA3000259F900D349F900D11246FEF70E00F947F
:10EA40001DDD7093AD006093AC00EFBF08951F9380
:10EA5000CF93DF93D0914D03D1FD1DC010911B05C5
:10EA6000C1E020E030E048E452E46091B00D7091E4
:10EA7000B10D8091B20D9091B30D0F9405E0181671
:10EA80000CF0C0E0DE7FCD2B81E0111101C080E0F1
:10EA9000C82BC0934D0380914D03DF91CF911F91FF
:10EAA0000C94DB74EF92FF920F931F93CF93DF933D
:10EAB000EC018B017A010E943B5B81110BC0A80124
:10EAC000BE01C701DF91CF911F910F91FF90EF9091
:10EAD0000D9468DCDF91CF911F910F91FF90EF9023
:10EAE00008950F931F93CF93DF938C01D62FC72FD9
:10EAF0000F9462DC8F3F980739F46D2F7C2FC8018B
:10EB00000F94B2DC8D2F9C2FDF91CF911F910F912D
:10EB100008950F931F93CF938C01C62F0F9454DC4D
:10EB20008F3F29F46C2FC8010F949CDC8C2FCF9160
:10EB30001F910F910895CF93DF93EC010F9462DC46
:10EB4000BC016F5F7F4FCE01DF91CF910D94B2DC9E
:10EB5000CF93DF93EC010F9454DC61E0680FCE019A
:10EB6000DF91CF910D949CDCCF93DF93EC010F9458
:10EB700054DC61E0811160E0CE01DF91CF910D9412
:10EB80009CDC2BE0829FC0011124805B924F0F948C
:10EB900062DC21E0019609F420E0822F0895CF93F2
:10EBA000DF93C82FD8E0CF5FC8300CF0C0E08C2FC7
:10EBB0000E94C175811103C0D150A9F7CFEF8C2FEE
:10EBC000DF91CF91089581EA9DE00F9454DC0E947B
:10EBD000CF7587FD05C0682F81EA9DE00D9478DC34
:10EBE00008950F931F93CF93C82F8B0162E678E7A8
:10EBF000823070F06BE578E7843050F063E578E7B9
:10EC0000843031F06BE478E7853011F064E478E724
:10EC1000C8010F940BDA8CEF8C0F823028F0C17092
:10EC2000CF5CF801C6831782CF911F910F91089591
:10EC300061E080EC9FE00F9478DC60E08FEB9FE078
:10EC40000F9478DC60E08EEB9FE00F9478DC60E05E
:10EC50008DEB9FE00F9478DC60E08CEB9FE00D94EF
:10EC600078DCCF93C82F82958F700E9455638C2FCC
:10EC70008F70CF910C9455638091A3109091A41044
:10EC8000181619060CF043C001979093A4108093B6
:10EC9000A310892BA1F480919E1090919F10892B35
:10ECA00021F41092A1101092A0108091A0109091C8
:10ECB000A110909393128093921281E00895809115
:10ECC0009212909193120396FC01EB55FF4E208116
:10ECD00001962111F9CFFC01EB55FF4E8D3E21E04D
:10ECE000920740F441919C012F5F3F4F4111E1CFCA
:10ECF000C901F4CFE5EAF0E18D3E21E09207C9F6C3
:10ED0000CF01855A904121912223D1F3D2CF80E0C7
:10ED100008958091990490919A0420919B043091D8
:10ED20009C04821B930B8F7799270895FC0120E0A8
:10ED30003EE2DB014D91BD01403249F0283011F433
:10ED400030833196DB0111974C91408331962F5FD0
:10ED50002B3079F71082089540E050E0BA010D940D
:10ED6000CD57FC01238121110D94AB590895909149
:10ED70003905911107C09091C00095FFFCCF809399
:10ED8000C6000895913031F49091C80095FFFCCFF2
:10ED90008093CE0008950E94B77690E080E00895B9
:10EDA000CF93DF93EC01FE018491882321F00E9430
:10EDB000B7762196F8CFDF91CF910895CF92DF9269
:10EDC000EF92FF92C090B00DD090B10DE090B20DD7
:10EDD000F090B30D89E79DE70E94D07642E0C7012D
:10EDE000B6010F94BFD581E79DE70E94D076609170
:10EDF000EE047091EF048091F0049091F10441E0F1
:10EE00000F94BFD5FF90EF90DF90CF900D9435D643
:10EE10004F925F926F927F928F929F92AF92BF922A
:10EE2000CF92DF92EF92FF920F931F93CF93DF93D6
:10EE3000CC24CA94DC2C76010EEA1FE093E2892EE2
:10EE4000912CA12CB12C412C512C3201D0E0C0E0EE
:10EE50008FEFC81609F45DC0C8010F9462DCEC01A5
:10EE6000BC01990F880B990B0F94E2D62091CA0D23
:10EE70003091CB0D4091CC0D5091CD0D0F947BDE98
:10EE80002B013C01C701B6010F94A3D58DEC9CE783
:10EE90000E94D076C501B4010F94A3D58DEC9CE7F8
:10EEA0000E94D076BE010D2E000C880B990B0F949A
:10EEB000A3D58DEC9CE70E94D07620E030E04AE7B5
:10EEC00054E4C301B2010F9421D70F94EF7585E08C
:10EED000880E911CA11CB11C0E5F1F4F8FEFC81A2A
:10EEE000D80AE80AF80A0A3B8FE0180709F0B0CF01
:10EEF000DF91CF911F910F91FF90EF90DF90CF9016
:10EF0000BF90AF909F908F907F906F905F904F9049
:10EF100008958AE897E40E94D076B8CF882371F1EB
:10EF200081EC9CE70E94D0766091491370E090E0FC
:10EF300080E00F94A3D5809149138430D8F01092CB
:10EF400049138CEB9CE70E94D0768091491390E0A6
:10EF50000F943076809149132091AC053091AD0526
:10EF60003093B70D2093B60D0F94B50F0E94136424
:10EF70000D94ED438F5F80934913E3CF8CE59BE3C2
:10EF80000E942C7270E060E00E94E1E4E5CFCF9334
:10EF9000DF9389EB9CE70E94D076C2E9D6E06881D6
:10EFA00079818A819B8142E00F94BFD585EB9CE7F4
:10EFB0000E94D0766C817D818E819F8142E00F948A
:10EFC000BFD581EB9CE70E94D076688579858A85DC
:10EFD0009B8542E00F94BFD58DEA9CE70E94D076D6
:10EFE0006C857D858E859F8542E00F94BFD583E734
:10EFF00095E60E94D07680E00F94CB430F94E2D642
:10F00000CEEBDDE02C813D814E815F810F947BDE74
:10F0100042E00F94BFD589EA9CE70E94D07681E058
:10F020000F94CB430F94E2D6288539854A855B85BA
:10F030000F947BDE42E00F94BFD585EA9CE70E94E7
:10F04000D07682E00F94CB430F94E2D62C853D8599
:10F050004E855F850F947BDE42E00F94BFD581EA39
:10F060009CE70E94D07683E00F94CB430F94E2D6C6
:10F07000288939894A895B890F947BDEDF91CF919A
:10F080000D94EF7580EB9BE70E94D0766091B00DF8
:10F090007091B10D8091B20D9091B30D41E00F943C
:10F0A000BFD58DEA9BE70E94D0766091B60D709136
:10F0B000B70D072E000C880B990B0F94E2D641E098
:10F0C0000F94BFD589EA9BE70E94D0766091EE0449
:10F0D0007091EF048091F0049091F10441E00F945D
:10F0E000BFD586EA9BE70E94D07660917206709148
:10F0F0007306072E000C880B990B0F94E2D641E0A3
:10F100000F94BFD581EA9BE70E94D0766091B00D45
:10F110007091B10D8091B20D9091B30D41E00F94BB
:10F12000BFD58EE99BE70E94D0766091B60D7091B5
:10F13000B70D072E000C880B990B0F94E2D641E017
:10F140000F94BFD58AE99BE70E94D076609116059F
:10F1500070E090E080E00F94A3D585E99BE70E94E2
:10F16000D07660911D0670E090E080E00F94A3D50A
:10F1700081E99BE70E94D0766091990370919A0390
:10F1800080919B0390919C0341E00F94BFD58DE843
:10F190009BE70E94D0766091560670915706809149
:10F1A00058069091590641E00F94BFD50D9435D67D
:10F1B0002091881430E0A8EEB3E00F94F4DCAB01AA
:10F1C000BC0189E894E10F94352B882399F0809154
:10F1D000871480FD0E9442788091871482FD0E94EE
:10F1E000C7778091871481FD0E94046689E894E1C5
:10F1F0000D94F42C08950E94D0760D9435D6CF93BB
:10F2000081EA9DE00F9454DCCBE08C9FC001112477
:10F21000805B924F0F9462DC8156904F803A9F4002
:10F22000C8F088E49DE70E94FB7881EA9DE00F9496
:10F2300054DC8C9FC001112470E060E0805B924F31
:10F240000F94B2DC8BE09DE70F94F62081E0CF9124
:10F250000C94A56ECF910895FF920F931F93CF93B7
:10F26000DF939091110591114FC0C82F81E08093D9
:10F270001105CC2311F10E9410678823F1F00E9440
:10F280000567811122C081EA96E30E942C7263E037
:10F290000E94FBF1F090AE050091AC051091AD0518
:10F2A000D091AB050F945D2AF092AE051093AD0599
:10F2B0000093AC05D093AB0508C061E080E00E94EC
:10F2C00078F58AE99AEACC2311F082EC9AEA0E9456
:10F2D000D0768CEE95E60E94FB7886E996E30E9454
:10F2E0002C720E943BF29FB7F894809102018460D7
:10F2F000809302019FBF0F94AB1FC11105C0809185
:10F30000D60381608093D603DF91CF911F910F9137
:10F31000FF900895EC01F8940F941D30179A109205
:10F320008F06169A10929006149A8AE99AEA0E9419
:10F33000D0768CEE9CE70E94FB78209779F0CE0186
:10F340000E94FB78BE0185E99CE00F94B2DC62E488
:10F3500084E99CE00F949CDC0E94CC66C4EEDCE760
:10F36000F1CF8091060186FD35C080E00E943066B5
:10F3700010929A0610929B0610929C0610929D067F
:10F380000F9441BF20E030E040EA50E460919A06DB
:10F3900070919B0680919C0690919D060F947CDD58
:10F3A00060939A0670939B0680939C0690939D06AB
:10F3B000E0917102F091720260857185828593857A
:10F3C0000F9481C00F94ED438FE893E60E942C7256
:10F3D0000E948A7908952F923F924F925F926F9286
:10F3E0007F928F929F92AF92BF92CF92DF92EF92D5
:10F3F000FF920F931F93CF93DF93CDB7DEB7609744
:10F400000FB6F894DEBF0FBECDBF282E6E875A8789
:10F4100049872091B7022D87772473947092B702A1
:10F4200042E0841709F4D4C1082F10E0F801E65730
:10F43000F4483490832D032C000C990B9C878B8708
:10F44000D801AA0FBB1FAA0FBB1FBA83A983FD0156
:10F45000E353FD4F80819181A281B3818B839C8393
:10F46000AD83BE838093B8029093B902A093BA0291
:10F47000B093BB02BC01CD010E9447666B017C01C9
:10F4800081E0022C01C0880F0A94EAF70F94DD2670
:10F49000A981BA81AE56B94FB887AF83FD011082FA
:10F4A0001182128213820F9441BF0E94BA67632DAA
:10F4B000032C000C770B880B990B0F94E2D64B01B1
:10F4C0005C0149815A814C58594F588B4F8720E035
:10F4D00030E040E450EC0F9421D7AF85B8896D93AC
:10F4E0007D938D939C931397C701B6010F944EC0E3
:10F4F0000F94ED430F94034F1092B702EF81F885FC
:10F5000010821182128213820F9441BFAF85B88995
:10F510008D929D92AD92BC921397C701B6010F9444
:10F520004EC00F94ED437092B702E981FA81E25820
:10F53000F44845905590659074902DEC3CEC4CE867
:10F540005FE3C501B4010F9421D7A30192010F9489
:10F5500021D7EF85F8896083718382839383C70104
:10F56000B6010F944EC00F94ED43712C612C4F8067
:10F5700058840F94034F1092B702D2011D921D922E
:10F580001D921C9213970F9441BF20E030E040E29F
:10F5900051ECC501B4010F9421D7EF85F889608340
:10F5A000718382839383C701B6010F944EC00F9479
:10F5B000ED430F94034FF1E0F093B70220E030E009
:10F5C00040E351E4C501B4010F9421D7AF85B88958
:10F5D0006D937D938D939C9313978B819C81AD81CB
:10F5E000BE818093B8029093B902A093BA02B093FF
:10F5F000BB02C701B6010F944EC00F94ED43822D9C
:10F600000F947A259C0144E0369527954A95E1F7B9
:10F61000A985BA85109721F0FD01E60DF71D20831D
:10F620009F938F933F932F937F926F92E6E6FBE732
:10F63000FF93EF930F9416DB4FEF641A740A0FB623
:10F64000F894DEBF0FBECDBF9E85691608F491CF3A
:10F650000F94034F1092B7028091F204882309F4AB
:10F66000B2C0F801ED50FB4F6081603408F0ABC0D0
:10F67000F801E65AFD4FA081AB83F801EB50FB4F38
:10F68000808140E051E002C0569547958A95E2F7A7
:10F69000822D0F94DB8BBB81BB2339F0432D419529
:10F6A0006B2F70E0822D0F94AC8B0F94AE26822DC1
:10F6B0000E942A5AF801E157F94F81E080836B8557
:10F6C0007C85719561957109072E000C880B990B4B
:10F6D0000F94E2D62AE037ED43E25CE30F9421D7A2
:10F6E0004B015C01F801E85AFD4F608170E090E049
:10F6F00080E00F94E2D69B01AC01C501B4010F94E8
:10F7000021D74B015C01E981FA81EE56F94FFC8368
:10F71000EB83AC019B0160817181828193810F94A5
:10F720007BDDAB81BC816D937D938D939C9313970F
:10F730000F9441BFEB81FC81208131814281538153
:10F74000C501B4010F947CDDAB81BC816D937D93C9
:10F750008D939C931397E981FA81EC58F94F60835C
:10F7600071838283938320E030E040E05FE3C70150
:10F77000B6010F9421D70F944EC00F94ED43109211
:10F78000B8021092B9021092BA021092BB02FD8523
:10F79000F093B70260960FB6F894DEBF0FBECDBFF0
:10F7A000DF91CF911F910F91FF90EF90DF90CF905D
:10F7B000BF90AF909F908F907F906F905F904F9091
:10F7C0003F902F900895432D419568E070E06ACFF7
:10F7D00081E00E943066ECE8FBE7B491B9831092B7
:10F7E0009A0610929B0610929C0610929D060F940A
:10F7F00041BFE6E8FBE785909590A590B490E9813C
:10F800006E2FEE0F770B880B990B0F94E2D66B01DE
:10F810007C0120E030E040EC5FE3C501B4010F94CF
:10F8200021D7A70196010F9421D760937C0670938E
:10F830007D0680937E0690937F0680E090E0A8E4AA
:10F84000B4E48093B8029093B902A093BA02B09343
:10F85000BB02BC01CD010E9447664B015C010F94C5
:10F860004EC00F94ED430E94B17910929A06109207
:10F870009B0610929C0610929D060F9441BFE2E6F3
:10F88000FBE765917591859194919058A701960138
:10F890000F9421D760937C0670937D0680937E063B
:10F8A00090937F06C501B4010F944EC00F94ED43B1
:10F8B000E2E6FBE765917591859194919B01AC011E
:10F8C0000F947CDDA70196010F9421D760937C06ED
:10F8D00070937D0680937E0690937F0680E090E093
:10F8E000A8ECB3E48093B8029093B902A093BA0253
:10F8F000B093BB02BC01CD010E9447660F944EC07D
:10F900000F94ED430E94B17982E00E942A5A8091BF
:10F910009A0690919B06A0919C06B0919D068093BB
:10F920007C0690937D06A0937E06B0937F0610928E
:10F93000B8021092B9021092BA021092BB020F9450
:10F94000034F7092910680E00E94306620CF2F9284
:10F950003F924F925F926F927F928F929F92AF925F
:10F96000BF92CF92DF92EF92FF920F931F93CF93AC
:10F97000DF9300D01F921F92CDB7DEB7D82E2A0199
:10F980003B01322EE982FA820B831C830F94ED43F4
:10F9900081E08093A70DFC2CE32CD31010C0ED2C3C
:10F9A000DC100DC060E070E080EA90E40E94E06D41
:10F9B000FF24F394EE24E3942224239401C02D2CFD
:10F9C0000F946ECE8091C2138D831092C21382E089
:10F9D0000F94D94360939A0670939B0680939C067C
:10F9E00090939D06F1100F9413CA81E00E946866FF
:10F9F0008C010E94BA671092B8021092B90210925C
:10FA0000BA021092BB02222009F477C19B8D91119A
:10FA10006AC150E040E061E080E00E94EB79EE20B6
:10FA200031F050E040E061E081E00E94EB79DD20C0
:10FA3000E9F04114510461047104C1F0C301B20141
:10FA40000F94E2D69B01AC016091160E7091170ED7
:10FA50008091180E9091190E0F947CDD60939206A0
:10FA6000709393068093940690939506332001F14A
:10FA700089819A81AB81BC810097A105B105C1F054
:10FA8000BC01CD010F94E2D69B01AC0160911A0E2E
:10FA900070911B0E80911C0E90911D0E0F947CDDB9
:10FAA00060939606709397068093980690939906B4
:10FAB000FF2009F4A2C060E070E080EA90E40E94B8
:10FAC000E06D80918F06811105C050E040E061E05B
:10FAD0000E94EB7980919006811106C050E040E0D1
:10FAE00061E081E00E94EB790F94D3CEE3EFF4EA7A
:10FAF00085919591A591B491EFEEF4EA45915591D8
:10FB000065917491409374065093750660937606E0
:10FB1000709377068093780690937906A0937A067F
:10FB2000B0937B0668E776E084E796E00E948269FE
:10FB30000F9435CE20E030E040E850EC609178063C
:10FB40007091790680917A0690917B060F9471DE10
:10FB500087FF0CC080E090E0A0E8B0EC80937806CE
:10FB600090937906A0937A06B0937B0680E090E0AC
:10FB7000A6E1B3E48093B8029093B902A093BA02CD
:10FB8000B093BB021092B7020F9441BF6091B802CC
:10FB90007091B9028091BA029091BB020F944EC04D
:10FBA0000F94ED438091740690917506A0917606AE
:10FBB000B09177068093920690939306A093940653
:10FBC000B09395068091780690917906A0917A0677
:10FBD000B0917B068093960690939706A093980623
:10FBE000B093990681E08093B7020F94034F50E0E1
:10FBF00040E061E082E00E94EB79CC20E9F08114E2
:10FC00009104A104B104C1F0C501B4010F94E2D67E
:10FC10009B01AC0160911E0E70911F0E8091200E11
:10FC20009091210E0F947CDD60939A0670939B0651
:10FC300080939C0690939D060F9441BFC8010E943B
:10FC40004E660F94034F0F94D3CE0F9471CCD11006
:10FC500007C0311005C08C8D811102C0CC2039F154
:10FC6000F11025C09D81992311F181E08093C21389
:10FC70000F94D9436B017C0180E00F94D943A70115
:10FC800096010F94E9A19B01AC0160919A067091D5
:10FC90009B0680919C0690919D060F947BDD60935E
:10FCA0009A0670939B0680939C0690939D060F94F2
:10FCB000ED431092A70D0F900F900F900F900F90A3
:10FCC000DF91CF911F910F91FF90EF90DF90CF9038
:10FCD000BF90AF909F908F907F906F905F904F906C
:10FCE0003F902F90089580E00F94A023EE2009F418
:10FCF0009ECE81E00F94A0239ACEEE2009F497CEF9
:10FD0000AB8DAA2309F48DCEF4CF8F929F92AF9240
:10FD1000BF92CF92EF92FF920F931F93262F91E005
:10FD20009F931F92812C912C5401C42EE12CF12C15
:10FD3000870140E050E0BA010E94A77C0F900F902D
:10FD40001F910F91FF90EF90CF90BF90AF909F9039
:10FD50008F90089586E893E00F94F42C8091A3107F
:10FD60009091A410892B79F0E0919212F091931266
:10FD7000EB55FF4E8081813011F0863021F487E110
:10FD80009DE60C94FB7808958091A3109091A410A7
:10FD9000892B29F00E94AA7E0E943C76F5CF109212
:10FDA0009312109292121092A1101092A01081E062
:10FDB0008093A2100895EF92FF920F931F93CF9319
:10FDC000DF938091C213882389F186E79CE70E9424
:10FDD000FB7880E69CE70E94FB788FE49CE70E941A
:10FDE000FB78C7E0DCE1C15058F1CD9F70011124D0
:10FDF00001E010E08CE49CE70E94D076F801EE0F61
:10FE0000FF1FEE0FFF1FEE0DFF1DE154FC4E608142
:10FE100071818281938145E00F94BFD50F5F1F4FA1
:10FE20000830110539F70F9435D6DDCF83E89CE70C
:10FE3000DF91CF911F910F91FF90EF900C94FB7881
:10FE4000DF91CF911F910F91FF90EF9008958F92C6
:10FE50009F92AF92BF92CF92DF92EF92FF920F9458
:10FE6000512A6B017C0120912F02222309F140913C
:10FE7000BE024130E9F08091100290911102A091F0
:10FE80001202B091130246015701881A990AAA0A70
:10FE9000BB0A30E0A8EEB3E00F94F4DC86169706B8
:10FEA000A806B9066CF0443031F19CF44230D4F429
:10FEB000C0921002D0921102E0921202F09213024C
:10FEC000FF90EF90DF90CF90BF90AF909F908F907A
:10FED0000895453069F782EC9AEA0E94D07688EF5F
:10FEE0009AE706C082EC9AEA0E94D07685E29BE708
:10FEF0000E94FB78DDCF82EC9AEA0E94D0768FE0F8
:10FF00009BE7F6CFCF92DF92EF92FF920F931F9372
:10FF1000CF93DF931F921F92CDB7DEB70F94512A74
:10FF20000091C0171091C1172091C2173091C317CB
:10FF3000601B710B820B930B69387341810591052E
:10FF4000D0F080916F06811116C00F94512A6093F2
:10FF5000C0177093C1178093C2179093C3178091F5
:10FF6000A604809314028B3418F08FEF8093A604BC
:10FF700081E080936F060F94512A0091C017109171
:10FF8000C1172091C2173091C317601B710B820BF0
:10FF9000930B653671058105910508F457C1809171
:10FFA0006F06882309F452C16091E2057091E30560
:10FFB000072E000C880B990B0F94E2D66B017C0185
:10FFC0000F94512A0091C0171091C1172091C217A8
:10FFD0003091C317601B710B820B930B0F94E0D60B
:10FFE0009B01AC0160E070E08AE793E40F947BDE54
:10FFF000A70196010F9421D70F94EDDE7093CA03E9
:020000021000EC
:100000006093C9036091E4057091E505072E000C2B
:10001000880B990B0F94E2D66B017C010F94512A47
:100020000091C0171091C1172091C2173091C317CA
:10003000601B710B820B930B0F94E0D69B01AC01FC
:1000400060E070E08AE793E40F947BDEA7019601FD
:100050000F9421D70F94EDDE8B017093CC03609346
:10006000CB031092E3051092E2051092E505109281
:10007000E40583E08A8382E08983809138028823C3
:1000800051F087E89FE00F9454DC91E0811101C0AA
:1000900090E0909338028091C9039091CA034497ED
:1000A0000CF09DC020E030E048E452E46091B00DD7
:1000B0007091B10D8091B20D9091B30D0F9405E048
:1000C00018160CF08CC080914E038F5F80934E0306
:1000D000053011050CF089C09091A50D8091A60DF9
:1000E000981709F47FC0E091A60D8EE6E89FF00115
:1000F0001124E55FF84F80818C3408F476C080913C
:100100004F038F5F80934F0380914E0381110BC08B
:1001100080914F03811107C08091E603823019F46A
:1001200081E08093E6038091E603813061F40E94D0
:100130006167811108C01092E6031092D5038FEC1D
:100140009FE60E943BF280913802882309F46EC03A
:100150008091E603823009F469C08EE4E82E83E0E2
:10016000F82EFE0131966F0110E002E0F701919147
:100170007F01F60181916F01891768F5F7013197C9
:1001800010828091E603823031F10093E6030E94F1
:100190001067882381F10E940567811106C0809154
:1001A0000E05882329F10F949E15113059F189E627
:1001B00098E70E94FB788091D50381110CC041E043
:1001C00070E060E088EC90E00F94815262E08AE396
:1001D0009AE60E94FBF1113049F111E0C7CF10926D
:1001E0004E0376CF8091E70387CF10924F038CCFD9
:1001F0000F945D2ADACF1092B70D1092B60D1092BF
:10020000E303D3CF81E998E70E94FB788091D5037F
:1002100081110CC041E070E060E088EC90E00F9448
:10022000815262E086E29AE60E94FBF1809114021C
:100230008093A6040F94512A6093C0177093C1173E
:100240008093C2179093C31710926F060F900F9070
:10025000DF91CF911F910F91FF90EF90DF90CF90A2
:100260000C942775CF92DF92EF92FF926B017C0185
:10027000C0925403D0925503E0925603F092570374
:10028000809170038230B1F420E030E040E950E426
:10029000C7010F9471DE87FF14C08091EE0D90911D
:1002A000EF0DA091F00DB091F10D803D9740A105AB
:1002B000B10520F5C701B601FF90EF90DF90CF9018
:1002C00008952AE939E949E95EE3C701B6010F94C7
:1002D00071DE87FF0AC020E030E048E351E4C70147
:1002E000B6010F9421D76B017C0185EE98E70E943F
:1002F000D076C701B6010F94EF75DCCF2AE939E952
:1003000049E95EE3C701B6010F9471DE87FDE3CFD3
:1003100020E030E040E85EE3C701B6010F9421D74A
:1003200020E030E048E550E40F947CDDDCCFCF9254
:10033000DF92EF92FF92CF93909170039817B9F1EB
:10034000C82FC0905403D0905503E0905603F0900E
:10035000570320E030E0A901C701B6010F9471DE18
:10036000882341F0C092120ED092130EE092140E28
:10037000F092150E88EC98E70E94D076C13011F10A
:10038000E0F0C23011F1C09370036091120E7091D1
:10039000130E8091140E9091150E0E94328160937D
:1003A000120E7093130E8093140E9093150ECF912E
:1003B000FF90EF90DF90CF90089580EC98E70E9437
:1003C000FB78E1CF8CEB98E7FACF88EB98E7F7CF93
:1003D0000F94ED43179AEFE8F6E01082169A118217
:1003E000149A80E00E9497818FEF9FEF9093B20262
:1003F0008093B1022FEF2093AE029093B6028093C8
:10040000B5022093AD029093B0028093AF02909317
:10041000B4028093B302089541ED50E063E777E7BB
:100420008EEB9DE00F94EED90F949A640F94D83B15
:100430000F94AD320E94396582EC9AEA0E94D07620
:1004400081E597E70C94FB78CF93DF9363E777E739
:100450008EEB9DE00F940BDA41ED50E064E170E02B
:100460008EEB9DE00F9468DC60911D0582E09DE0BD
:100470000F9478DCC0EBD2E14AA55BA56CA57DA505
:100480008EEF9CE00F948ADC4EA55FA568A979A940
:1004900082EA9CE00F948ADC4AA95BA96CA97DA939
:1004A0008EE99CE00F948ADC4EA95FA968AD79AD16
:1004B0008AEF9CE00F948ADC4AAD5BAD6CAD7DADFC
:1004C0008AE99CE00F948ADC6EAD7FAD88E99CE000
:1004D0000F9496DC40E450E06AEB7CE080EF92E120
:1004E0000F9468DC409130135091311360913213B6
:1004F0007091331386EB9CE00F948ADC40913413A7
:1005000050913513609136137091371382EB9CE054
:100510000F948ADC409138135091391360913A134B
:1005200070913B138EEA9CE00F948ADC82EC9AEA8D
:100530000E94D0768DEF96E7DF91CF910C94FB78F7
:100540002F923F924F925F926F927F928F929F92E3
:10055000AF92BF92CF92DF92EF92FF920F931F93D1
:10056000CF93DF93CDB7DEB7A2970FB6F894DEBF77
:100570000FBECDBF8FE590E00E94C25B882309F4D7
:1005800091C00E9489768F37910561F480919B0418
:1005900090919C0490939A04809399048EEE96E730
:1005A0000E94FB781E012FE1220E311CDD24D39422
:1005B0000E948976181619060CF068C08091A90D62
:1005C000882329F00E940567882309F45FC0809181
:1005D000A60381115BC00F943CD697FDE9CF282F6D
:1005E0008F3F09F07BC080914003882309F473C0DA
:1005F000D0923F03109240031F8E18A2C090430375
:10060000CC20B1F2809141038F8F91E09C1518F4BA
:100610008091420388A3109243033AA229A289A1A0
:1006200082198C1528F6E9A1FAA11191FAA3E9A380
:1006300086E493E00F94B22A17FDF1CF80919E10CB
:1006400090919F101A3009F44AC11D3009F447C136
:100650008F3591050CF048C11B3311F4D09245033E
:10066000209145032111DBCF9C012F5F3F4F309339
:100670009F1020939E102091A0103091A1102B5517
:100680003F4E820F931FFC011383C9CF80919E10B0
:1006900090919F10181619060CF456C28091901470
:1006A000811166C2A2960FB6F894DEBF0FBECDBF11
:1006B000DF91CF911F910F91FF90EF90DF90CF903E
:1006C000BF90AF909F908F907F906F905F904F9072
:1006D0003F902F900895D09240038ECF30913F03EA
:1006E000332309F457C0893F09F43FC080F5863FA2
:1006F00009F448C080913E038260273F79F189EB7D
:1007000096E70E94D07684EB96E70E94D07610910F
:100710003E0380EB96E710FD02C08BEA96E70E944D
:10072000D076012F027086EA96E711FD02C081EAB9
:1007300096E70E94D07680EA96E70E94FB78002335
:1007400029F145E440930B0210923F0355CF8A3FB5
:1007500041F080913E0381602B3F89F680933E03F8
:10076000CECF80913E038E7FF9CF1092430310923B
:100770003F0310923E0310923D03109240031092EB
:100780003C03BDCF80913E038D7FE8CF50E2509374
:100790000B02DACF2091400340913E03222331F136
:1007A000E091430340FF49C030913C03332309F4F7
:1007B00040C021E02E0F20934303AE2FB0E0AF5B8B
:1007C000BC4FFFEFFC9350913D03552351F0EE5F7A
:1007D000E0934303E22FF0E0EF5BFC4F5083109275
:1007E0003D03315030933C0310924003E0914303AA
:1007F00040FF6CC020913C03222349F191E09E0F01
:1008000090934303AE2FB0E0AF5BBC4F8C938091CD
:100810003D03882351F0EE5FE0934303E92FF0E0BE
:10082000EF5BFC4F808310923D03215020933C03EB
:10083000E3CE22E020933C03D7CF21E02E0F20937C
:100840004303F0E0EF5BFC4F5FEF5083CDCFA82F69
:10085000AF7040E031E0AF3029F0B0E0A050BE4FC3
:100860004C9130E0582F507F503F59F4326030FFA8
:1008700013C0D0923C0331FF0CC082E080933C0354
:10088000BBCE82958F70A82FB0E0A050BE4F2C91A8
:10089000EECF20933D03B0CE81E08E0F80934303D3
:1008A000AE2FB0E0AF5BBC4F4C934A3009F4A4CEFE
:1008B00031FF03C0D0923C039FCEEE5FE093430331
:1008C000E82FF0E0EF5BFC4F208396CE91E09E0F87
:1008D00090934303F0E0EF5BFC4F80838DCE009755
:1008E00019F410924503DECE0091A0101091A110D2
:1008F00008551F4E800F911FFC0110821A83098337
:1009000080914503811103C1F80180818E3409F083
:100910008AC04AE050E0BE016F5F7F4FC801019678
:100920000F94DFD72B013C01E980FA80F701808129
:10093000803231F4FFEFEF1AFF0AFA82E982F4CF36
:1009400080907A0390907B03A0907C03B0907D030D
:10095000D501C4010196A11DB11D84159505A605FB
:10096000B70549F044E050E069EE76E7C7010F941F
:1009700033DA892BA1F46AE270E0C7010F94ABE28D
:100980009093960380939503009709F445C0F8016E
:10099000F12CE817F90771F02191F226FACF8AE9D4
:1009A0009AEA0E94D07688E894E60E94D076C50143
:1009B000B40115C00E94F55AF8161906D9F08AE953
:1009C0009AEA0E94D07689E694E60E94D0766091F9
:1009D0007A0370917B0380917C0390917D030F9447
:1009E000A3D50F9435D60E940D5B10929F101092E4
:1009F0009E1058CEE0919503F09196031082E98005
:100A0000FA8064EE76E7C7010F9402DA892B39F594
:100A100083EA97E60E948A798AE99AEA0E94D07668
:100A20008FE394E6C2CF89819A81FC012081203234
:100A300021F401969A838983F6CF6AE270E00F94DD
:100A4000ABE2892B39F08AE99AEA0E94D07685E1F7
:100A500094E6BBCF44244A94542C3201D0CF44E0D6
:100A600050E06FED76E7C7010F9433DA5C01F701D0
:100A70008081873481F48091B80D853061F08EE0FB
:100A800095E00F94B22AF6E0F093B80D60E085EAA5
:100A90009FE00F9478DCAB2821F080911105811143
:100AA000A4CF26E077FC21E08091A0109091A110C6
:100AB000FC01EB55FF4E208349815A81F801DA0190
:100AC00040175107A1F501900020E9F79F01201B75
:100AD000310B0396280F391F2D3EF1E03F0779F1C6
:100AE0003093A1102093A0108091A3109091A41096
:100AF00001969093A4108093A31077FC08C04092B5
:100B00007A0350927B0360927C0370927D03109273
:100B10009F1010929E100E948976892B09F4C2CDF5
:100B20008FE590E00E94C25B811179CDBBCD6D91C4
:100B300061939D01241B350B6111F9CFCACF10922F
:100B4000A1101092A010D0CF60ED77E086E493E082
:100B50000F94832A882309F4A1CD109245031092A3
:100B60009F1010929E1084ED96E70E94FB789ACD1C
:100B700080912317882309F495CD80919E10909140
:100B80009F10892B09F08ECD8091A3109091A41015
:100B9000892B11F4109244032DE9E22E20E1F22E6C
:100BA00032E0D32ECC24C3944091A4175091A517C2
:100BB0006091A6177091A71780919D1790919E172D
:100BC000A0919F17B091A017481759076A077B0794
:100BD00008F02FC18091440381112BC10F94BE7B7B
:100BE000882349F120913B1730913C1789019BEFF5
:100BF000B92EF80180818B3351F5F80161916A308B
:100C0000E9F78F01CF018D599E4081309240D4F099
:100C1000C801821B930B01970F94AF7B80E297E191
:100C20000F945457882339F00F94BE7B2DE93EE092
:100C300089018111E2CFF0923C17E0923B170FEF50
:100C40001FEF37C0BA94B110D5C001501109C801C7
:100C5000821B930B01960F94AF7BC8010196F8019C
:100C6000008110E08090281790902917A0902A17F3
:100C7000B0902B1740913117509132176091331774
:100C80007091341784169506A606B706A0F69C0147
:100C90002D593E402115324044F080E297E10F94F7
:100CA0005457882341F28DE99EE090933C1780933E
:100CB0003B17409128175091291760912A1770917E
:100CC0002B174093A4175093A5176093A617709302
:100CD000A71780919E1090919F100A3061F00D30FF
:100CE00051F0033209F48CC08F3591053CF40F3F6D
:100CF000100709F08CC0009709F4D4CC2091231779
:100D0000211103C040E050E0BA01209182033091EC
:100D10008303421B530BA091A010B091A110FD01C1
:100D2000EB55FF4ED0824183528313968B559F4ED5
:100D3000FC01EA0FFB1F1082AB55BF4EFD01019075
:100D40000020E9F73197EA1BFB0BF8948091A31080
:100D50009091A41001969093A4108093A310EC5F3F
:100D60008091A0109091A110E80FF92FF11DF09340
:100D7000A110E093A01080912317882309F443C0A9
:100D80008091A4179091A517A091A617B091A717CD
:100D90008093820390938303A0938403B09385038D
:100DA000ED3EF14021F41092A1101092A010789421
:100DB0001092450310929F1010929E104091A4171C
:100DC0005091A5176091A6177091A71780919D1754
:100DD00090919E17A0919F17B091A017481759079F
:100DE0006A077B0730F58FE590E00E94C25B8111B6
:100DF000DBCE58CCF80180818B3309F4FACE25CFB5
:100E0000C092440378CF80E090E0DC01C1CF9C0128
:100E10002F5F3F4F30939F1020939E102091A01082
:100E20003091A1102B553F4E820F931FFC0103837D
:100E3000BBCE4091A4175091A5176091A617709151
:100E4000A71780919D1790919E17A0919F17B09121
:100E5000A017481759076A077B0708F423CC0E949C
:100E6000935A892B09F01ECC80E297E10F947659B2
:100E700080E297E10F94AB5910928E1410928F1468
:100E800082E094E60E94FB780F94A83F6B017C01FE
:100E90000E949F658CE3882E912CA12CB12CC70158
:100EA000B601A50194010F94C7DCCA01B901A501DF
:100EB00094010F94C7DC7F936F93C701B60120E1C3
:100EC0003EE040E050E00F94C7DC3F932F9380EC6E
:100ED00096E79F938F938E010F5F1F4F1F930F9382
:100EE0000F946BDB82EC9AEA0E94D076C8010F94D3
:100EF00038D6C8010E9467F50F94BE81109269022E
:100F00000FB6F894DEBF0FBECDBF80919114882339
:100F100019F00F94F276C6CB81E00F94FD81809199
:100F200091148111F6CFBECBCF93DF93EC01899161
:100F3000882319F00E94B776FACFDF91CF910895F8
:100F4000FF920F931F93CF93DF93EC01F62E66234E
:100F500009F44BC00F9412DA8C01C8010E94C25BE5
:100F6000882309F453C08091A0109091A110FC0136
:100F7000EB55FF4E23E0208388559F4EBE01FF2096
:100F8000E9F10F940BDA82EC9AEA0E94D07687EFAF
:100F900093E60E94D0768091A0109091A110885580
:100FA0009F4E0E9494878EE996E70E94FB7880917D
:100FB000A0109091A1100496080F191F0D3E81E01A
:100FC0001807F9F01093A1100093A0108091A310BE
:100FD0009091A41001969093A4108093A310DF9198
:100FE000CF911F910F91FF900895FC010190002077
:100FF000E9F731978F01081B190BAFCF0F94BFE2B0
:10100000C2CF1092A1101092A010E0CF8AE99AEA04
:101010000E94D07687EF93E60E94D076CE01FF2023
:1010200059F00E94D07683E89AEADF91CF911F9120
:101030000F91FF900C94FB780E949487F4CF0F934C
:101040001F93CF93DF93D62F8C01C0E0F8018591D9
:1010500094912BE68733920721F42091BA13213023
:1010600019F461E00E94A087CF5F0E5F1F4FDC1371
:10107000EDCFDF91CF911F910F910895CF93DF9323
:10108000CDB7DEB76E970FB6F894DEBF0FBECDBFFB
:101090009E012C5D3F4FF901419151919F016EE1FD
:1010A00070E0CE0101960F94AADB60E0CE010196BC
:1010B0000E94A0876E960FB6F894DEBF0FBECDBF1C
:1010C000DF91CF910895EF92FF920F931F93CF93EB
:1010D000DF93CDB7DEB76B970FB6F894DEBF0FBEC8
:1010E000CDBF8AE59FE00F9454DCE82E0AE01FE0B4
:1010F000F12C48E050E0FE1479F0B801CE010E96D4
:101100000F9444DC1E8A60E0CE010E960F944F7F50
:10111000F394085F1F4FEDCF65E97FE08E010F5F0D
:101120001F4FC8010F9444DC19868EE28F8B43E079
:1011300050E061E97CE0CE0148960F9444DC1B8EC0
:10114000BE01695E7F4FC8010F94A0E21F930F9309
:1011500080E590E79F938F930E943E880F900F90B9
:101160000F900F906B960FB6F894DEBF0FBECDBFF9
:10117000DF91CF911F910F91FF90EF900895BF9253
:10118000CF92DF92EF92FF920F931F93CF93DF9353
:10119000E091A90DE111B1C0052F142FE9016B01F8
:1011A0007C01F8940E94BA64B090A80DB11002C0FE
:1011B000B090A70D0E9470640F94FBC180E1E2E93A
:1011C000F6E0A3E7B2E001900D928A95E1F7BB202B
:1011D00061F080E090E0A0E8BFEB80937302909311
:1011E0007402A0937502B0937602809139029091B7
:1011F0003A0290937203809371038091B60D90919F
:10120000B70D9093AD058093AC05809172068093E5
:10121000AE058091E50383FB882780F98093640500
:101220008091E7038093AB050E94C47E10929014D6
:1012300081E08093A90D0F944744789420E030E03A
:10124000A901C701B6010F9471DE20E030E0A901C9
:10125000F8016C2F7D2F81115AC08F2F902F0F9482
:1012600071DE882309F449C080916405811105C0AD
:1012700061E08CE39BE60E94A0870F931F93DF93AE
:10128000CF9386EB9DE69F938F930E943E880F90AD
:101290000F900F900F900F900F9020E030E0A90179
:1012A000C701B6010F9471DE882321F184E48F9386
:1012B00088E48F931F921F9220917B0230917C02D1
:1012C00040917D0250917E02C701B6010F947CDDF2
:1012D0009F938F937F936F938CE79DE79F938F935B
:1012E0000E943E888DB79EB70A960FB6F8949EBFAF
:1012F0000FBE8DBF81E08093A210DF91CF911F912F
:101300000F91FF90EF90DF90CF90BF9008958F2FB7
:10131000902F0F9471DE882349F2A6CF80910204AA
:10132000882321F180914F028230E9F4A0914D028F
:10133000B0914E0228EE33E00F9474DDAB01BC0196
:1013400087E393E00F94352B882331F060910004FC
:1013500070E085E00C94F4E980913703882331F044
:1013600060910104F5CF8111FBCFF0CF089560911A
:10137000010484E39DE00F9478DC6091000483E332
:101380009DE00F9478DC60914F0282E39DE00F9422
:1013900078DC60914D0270914E0280E39DE00D94E7
:1013A00096DC882361F081E080934F0280910104F4
:1013B0008E3118F48EE1809301040C948E8982E3BF
:1013C0009DE00F9454DC80934F0284E39DE00F94E2
:1013D00054DCF1CF80910204882331F087E393E05D
:1013E0000F94F42C0C948E890895FF920F931F9301
:1013F000CF93DF9390910204992399F1882351F1BF
:1014000000914F02C82FD0E0CC0FDD1F10E0FF2469
:10141000F394212F30E0809137038F25023009F0BB
:1014200080E08C0F9D2F911D281739078CF481E0E7
:1014300090914F02911180E080934F020E948E891B
:1014400069E170E080E090E00F9458281F5FE1CFE1
:1014500000934F02DF91CF911F910F91FF900C9459
:10146000EA89DF91CF911F910F91FF9008950F931B
:101470001F93CF93DF93C82F8091AA17813009F46F
:1014800041C0823009F457C00E9461678111F9C0E0
:101490008091B60D9091B70D009739F420917206A6
:1014A00030917306232B09F4ECC040913002509127
:1014B000310260913202709133024115510561058C
:1014C000710509F4DEC0892B31F480917206909188
:1014D0007306892B29F08091DA05882309F439C134
:1014E0008AED95E00F94352B882309F4CCC00F9436
:1014F0001D3082E796E30E942C720F94F6200F9421
:10150000AB1FC1C00F94237D882309F4BDCF81E0B8
:101510009091B717911101C080E08093AD17809131
:101520008F0E9091900E9093BA178093B91782E026
:101530008093AA17A9CF0F94237D1092AE178091A4
:10154000AA17823009F0A0CF8091AF17811140C057
:10155000D091B71781E0D11101C080E09091AD1713
:10156000891709F491CF8093AD178FEA97E10F9413
:10157000B22ADD23B1F18091AB17882311F180915C
:10158000A70381111EC08091BA138130D1F08091E0
:10159000A50D9091A60D891B8F7099F40E9410677C
:1015A00081110FC08091B40D843059F08FE59FE018
:1015B0000F9454DC811105C061E08CE09AE30F9434
:1015C0003BD381E08093AE1781E080936D025CCFC6
:1015D00064E670E08FEA97E10F94832A8111B8CF17
:1015E00053CF8091AC17882379F38091A7038111A1
:1015F000EBCF8091A50D9091A60D891B8F7021F4E2
:101600000E941067882301F38091A90D8111DCCF1E
:101610008091BA138130C1F28091B40D8430A1F26F
:101620008FE59FE00F9454DC8111CECF82ED95E6DB
:101630009F938F9388EB95E69F938F930F9416DB80
:101640001092AC171092AB1720E030E0A901CA014C
:10165000B9010E94BF8860E070E0CB010E94C467BE
:1016600085E69FE00E94A87581E09FE00E949B753F
:1016700087E490E70F9438760F900F900F900F90BB
:10168000A3CF1092DA058091A3109091A410039734
:1016900014F40E94A0829091A50D8091A60D981738
:1016A00081F08091B80D863061F468E873E18EE0D6
:1016B00095E00F94832A882321F08EE095E00F9423
:1016C000B22A40917E0350917F0360918003709114
:1016D0008103411551056105710509F03FC0409135
:1016E00034025091350260913602709137024115F3
:1016F000510561057105A9F086E893E00F94352B3B
:10170000882379F09091A50D8091A60D981309C0BA
:10171000C11107C0179A10928F06169A1092900660
:10172000149AC091E7039091A60D8091A50D98178A
:1017300001F18091A60D9EE6899FF0011124E55FDD
:10174000F84FC0819091A50D981799F08F5F8F7019
:10175000F9CF8AED95E00F94F42C95CF86E893E0CD
:101760000F94352B882309F4BACF80ED9CE70E94B3
:101770008A79CC2309F49FC080916C0390916D030A
:10178000A0916E03B0916F03892B8A2B8B2B81F470
:101790000F94512A605E7C4F8F4F9F4F60936C0374
:1017A00070936D0380936E0390936F03CFEF0FC020
:1017B0000F94512A00916C0310916D0320916E03D8
:1017C00030916F03601771078207930778F3809158
:1017D0006F06882309F478C0C093140280910C0529
:1017E000811107C081E080930C050F943AA71092F5
:1017F0000C058091D3058823E1F11092D30580E098
:101800000E94F5894FB7F8948091D105282F082EB2
:10181000000C330B37FF03C031952195310924307B
:1018200031050CF454C0982F87FF02C093E0980F45
:10183000959595952091700630917106290F311D6F
:1018400097FD3A953093710620937006837887FF51
:1018500003C081508C6F8F5F8093D1054FBF86E0AE
:101860000F940C4F80916D02811103C081E0809331
:101870006D020E948E898091D405882361F00E94B8
:101880007870E0911704F0911804309721F080915E
:101890006E02811119950E94D8780E94277F40E33B
:1018A00055E760E070E08EE993E0DF91CF911F9102
:1018B0000F910D94352B10926C0310926D031092C2
:1018C0006E0310926F0383CFC093A60487CF10924C
:1018D000D1054FBF80E0C4CFCF93DF93EC010F94CD
:1018E000613981E00E94378A80E00E94276E20974C
:1018F00099F0C233D10540F062E370E080E090E0FF
:101900000F945828E297EBCFBE0190E080E00F944F
:101910005828D0E0C0E0E3CFDF91CF910895CF9376
:10192000DF93C82FDFEF0F94613981E00E94378A7F
:101930008091B8138F3FD9F480914D13843021F4F6
:10194000809150138111EFCF80918B1390918C1364
:10195000019749F78091B2139091B313893290485F
:1019600011F360E089E290E80F942984DCCFD093F2
:10197000B813853039F4CF3FF9F261E08C2F0F9422
:10198000D0ADD1CF8430C1F6DF91CF9108951F92B1
:101990000F920FB60F9211240BB60F922F933F9315
:1019A0004F935F936F937F938F939F93AF93BF9367
:1019B000EF93FF932091780030917900E091360306
:1019C000F0E0EE0FFF1FEA5DFC4F80819181820FF6
:1019D000931F91838083809125038F5F80932503DC
:1019E000803109F056C0809136038F5F80933603B3
:1019F000883009F046C08091260390912703909388
:101A00000C0680930B0680912A0390912B039093F0
:101A10000A068093090680912C0390912D039093E0
:101A200008068093070680913003909131039093CC
:101A300016068093150680912E0390912F039093A4
:101A40005D0680935C0680913403909135039093FA
:101A50005B0680935A0681E080931C05FF91EF910D
:101A6000BF91AF919F918F917F916F915F914F91B6
:101A70003F912F910F900BBE0F900FBE0F901F90B4
:101A80001895809124034FE553E08F5F41F4109245
:101A9000240380917A00806480937A00DFCF9A01DA
:101AA000082E02C0359527950A94E2F720FFEDCF66
:101AB000809324030E94D35A10922503EACFCF9338
:101AC000DF93CAE7D0E088818F7B8883109225035B
:101AD000109236031092240380E00E94D35AE6E26B
:101AE000F3E080E1DF011D928A95E9F78881806447
:101AF0008883DF91CF9108952F923F924F925F920A
:101B00006F927F928F929F92AF92BF92CF92DF920D
:101B1000EF92FF920F931F93CF93DF93CDB7DEB772
:101B2000A4970FB6F894DEBF0FBECDBF0F94ED4360
:101B30008091AC0D811117C081E08093A80D809138
:101B40008F06882349F080919006882329F0209100
:101B500091062F83211120C081E08093A21080E4A0
:101B60009BE60F943876A4960FB6F894DEBF0FBEAE
:101B7000CDBFDF91CF911F910F91FF90EF90DF903C
:101B8000CF90BF90AF909F908F907F906F905F901D
:101B90004F903F902F9008958BEA9DE00F9454DC76
:101BA000182F8EE40E94565B082F0E94E85A8E83FD
:101BB000002329F0873009F4C9C0833029F013309D
:101BC00009F0C3C063E06E8380E090E0A0E8BFE36B
:101BD0008A839B83AC83BD838AEA9DE00F9454DCA7
:101BE000888F83E40E94565B182F0E94E85A1123C5
:101BF00029F0882319F08B3008F4888F88E50E943B
:101C0000565B882309F4ABC00E941D6020E030E0E1
:101C100048E052E40F947BDD20E030E048EB51E4F3
:101C20000F947BDD6A877B878C879D8789E50E947F
:101C3000565B882309F49CC00E941D6020E030E0C0
:101C400048E052E40F947BDD20E030E040EA50E4CD
:101C50000F947BDD6C8B7D8B8E8B9F8B87E50E9439
:101C6000565B882309F489C00E941D602A853B8544
:101C70004C855D850F947CDD20E030E048E852E43F
:101C80000F947CDD698F7A8F8B8F9C8F88E40E9404
:101C9000565B882309F47AC00E941D602C893D8917
:101CA0004E895F890F947CDD20E030E048E852E403
:101CB0000F947CDD6D8F7E8F8F8F98A30F94858C12
:101CC0008091290290912A02A0912B02B0912C02BE
:101CD0008093C3139093C413A093C513B093C613FA
:101CE0000F9413CA05EC1FE0C8010F9462DC019643
:101CF00009F051C00E5F1F4F053D8FE01807A1F797
:101D0000212CA2ECB3E1BAA3A9A3B987A887512CCF
:101D1000412C312C042D842D63E00F9403DD988B2E
:101D20006884798410E0F889F11137C0812F63E06D
:101D30000F9403DD911131C021103FC17E817330BA
:101D400009F470C08F818E8737C01E836AE979E9F4
:101D500089E19FE36A837B838C839D833DCF80E011
:101D600090E0A0E8BFEF8A879B87AC87BD875ECFF6
:101D700060E070E080E89FEF6DCF80E090E0A0E849
:101D8000BFE7898F9A8FAB8FBC8F80CF60E070E008
:101D900080E89FE78FCF2F80B4CF60E070E080ECC9
:101DA0009FE7D30111966D937D938D939C93149728
:101DB000BE81B330C1F11E86812F0F946DCA4B01D5
:101DC0005C01802F0F946DCA6B017C01A501940109
:101DD0006A857B858C859D850F9405E018160CF42B
:101DE0001CC1298D3A8D4B8D5C8DC501B4010F94BA
:101DF00005E018160CF411C1A70196016C897D89C4
:101E00008E899F890F9405E018160CF406C12D8D5C
:101E10003E8D4F8D58A1C701B6010F9405E01816ED
:101E20000CF4FBC033941F5F24E0620E711C17306A
:101E300009F079CF6FEF461A560A888599854C9636
:101E40009987888797E04916510409F063CF0F946A
:101E50002EA3A091C406AF83B091F703B88781E0A9
:101E60008093C4068AE0830D8093F70381E00E948B
:101E7000276E80E090E0A0EAB0E480939A06909309
:101E80009B06A0939C06B0939D0665E575E585E5E8
:101E900091E40F9481C080E00E9468669CA38BA3AC
:101EA000312C832D67E00F9403DDF82E092F682F66
:101EB00070E07F876E8780FF03C076E0791B072F75
:101EC000802F63E00F9403DD911105C08F2D0F94D7
:101ED00003DD11E0911110E0802F0F946DCA688B23
:101EE000798B8A8B9B8B8F2D0F946DCA4B015C0174
:101EF0008E81833009F099C01111C8C027E0AE85EA
:101F0000BF852A9FF0012B9FF00D1124E00FF11DDA
:101F1000EE0FFF1FEE0FFF1FEE53FC4E60E070E070
:101F200080EC9FE761837283838394833394E1E33E
:101F30003E12B7CF80E090E0A0EAB0E480939A062A
:101F400090939B06A0939C06B0939D0665E575E56E
:101F500085E591E40F9481C00F94ED43B1E33B1606
:101F600009F433C280916A0391E0980F90936A0359
:101F7000882309F4D3C160E080E00E9478F586E40C
:101F800096E30E942C720F94F62080E00F94BB0D14
:101F900081E08093BE028FEC9FE60E943BF22F818E
:101FA0002093C40668856093F70382E00E94276E41
:101FB0000F94ED431092A80DD6CD011103C011234B
:101FC00009F4BCCE812F63E00F940FDD840D952DB5
:101FD000911D880F991F8D53904F0F9462DCBC01A7
:101FE000990F880B990B0F94E2D62AE037ED43E264
:101FF0005CE30F9421D79B01AC016091C3137091F6
:10200000C4138091C5139091C6130F947CDDF30126
:10201000618372838383948391CEFE85FF2309F4C9
:1020200002CF222009F4FECEFECE288939894A89C2
:102030005B896A857B858C859D850F9405E01816E4
:1020400004F1288939894A895B89698D7A8D8B8D5C
:102050009C8D0F9471DE87FD14C0A50194016C89DD
:102060007D898E899F890F9405E0181654F0A5018B
:1020700094016D8D7E8D8F8D98A10F9471DE87FFF9
:1020800005C0112309F452CF211050CF10E0A7E072
:102090008E859F85A89FF001A99FF00D1124E00F68
:1020A000F11FEE0FFF1FEE0FFF1FEE53FC4E41809E
:1020B000528063807480C12CD12CE0EAEE2EE0E4E3
:1020C000FE2E222051F023E333E343EB5EE3C30112
:1020D000B2010F947CDD6B017C01A7019601609138
:1020E0009A0670919B0680919C0690919D060F9494
:1020F00071DE87FF10C0C0929A06D0929B06E092D4
:102100009C06F0929D0665E575E585E591E40F94E2
:1021100081C00F94ED43688979898A899B8960938E
:1021200092067093930680939406909395068092FE
:10213000960690929706A0929806B092990666E944
:1021400076E082E996E00E942A6A60E070E086E12B
:1021500093E40F9481C00F94ED438091AC0D8823DC
:1021600039F07F817093C40688858093F703FBCC98
:10217000812C912C70E2A72E71ECB72E222051F009
:102180002A813B814C815D81C301B2010F947BDDCB
:102190004B015C01488DC501B4010F948F8C8111F6
:1021A0000BC08FE893E60E942C729F938F930F943D
:1021B00016DB0F900F90BECE20919A0630919B06B1
:1021C00040919C0650919D06C701B6010F947BDD9E
:1021D00020E030E0A9010F9471DE87FF36C060E097
:1021E00070E080EA90E460939A0670939B06809377
:1021F0009C0690939D0665E575E585E591E40F9451
:1022000081C00F94ED43488DC501B4010F948F8CAC
:10221000882339F220919A0630919B0640919C06C2
:1022200050919D0660E070E080EA90E40F947BDDC1
:102230002DEC3CEC4CEC5DE30F9471DE87FF05C0A8
:102240008DE19CE70F943DDB75CEC0909A06D0904F
:102250009B06E0909C06F0909D062220A1F0A7012D
:102260009601C301B2010F947BDD9B01AC015F7746
:102270006A817B818C819D810F9471DE87FF03C011
:1022800084EE9BE7DFCF8FEA9FE00F9454DC882336
:1022900009F440C086EA9FE00F9454DC8823D1F112
:1022A0006091990370919A0380919B0390919C0394
:1022B0000E940A5C2091CA0D3091CB0D4091CC0D4B
:1022C0005091CD0D0F947BDE9B01AC01E7E0AE8514
:1022D000BF85EA9FC001EB9F900D1124080F191FC5
:1022E000000F111F000F111F0E531C4EC701B60126
:1022F0000F947BDDD80111966D937D938D939C9304
:1023000014978091F70381508093F70381E00E9436
:10231000276E0CCE20E030E0A901D8CF85E00F94E5
:102320000C4FC12CD12C90EAE92E90E4F92E82E1D9
:1023300096E30E942C720F94E9208EE190E00F94B6
:10234000343B0E94BE7280E00F94E74E182F60E08D
:1023500070E080E89FEB0E94616D81E00F94E74E92
:1023600084E00F94DD26C0929A06D0929B06E092FC
:102370009C06F0929D0665E575E585E591E40F9470
:1023800081C00F94ED430F94AE26812F0F94E74E3A
:1023900082E00F94D94320E030E040EA50E40F940B
:1023A00005E0181624F2EF81E093C406F885F09357
:1023B000F70381E00E94A56E41E061E081E00E94A8
:1023C000857E81E08093A210CECB10926A038BA110
:1023D0009CA10E944E660F94BDC960918A067091BF
:1023E0008B06072E000C880B990B0F94E2D69058A1
:1023F0002091CA0D3091CB0D4091CC0D5091CD0D57
:102400000F947BDE0F94D9C980EC9FE00F9454DCCD
:1024100091E0813009F090E099834FEB5FE06CE44C
:10242000CE0101960E946B5BF82E4EEB5FE062E5F9
:10243000CE0101960E946B5B082F4DEB5FE066E4D6
:10244000CE0101960E946B5B182F4CEB5FE062E4BB
:10245000CE0101960E946B5B212F110F330B082ECA
:10246000000C990B5C01A21AB30A8F2DFF0C990B7B
:10247000280F391F46E0429F6001439FD00C112472
:10248000F12CE12C002E000C110B081B190BB701CD
:102490006D537C4E3B01460177E07A83D3012D904A
:1024A0003D904D905D903D01FD013497FB87EA879B
:1024B000B401092C000C880B990B0F94E2D62FE382
:1024C00033EC4EE259E30F9421D7A20191010F940E
:1024D0007CDDAA85BB856D937D938D939C9313972B
:1024E000BA81B150BA83800E911EB111D7CFCA0CF8
:1024F000DB1CECE1EE0EF11CF4ECEF16F10439F606
:102500000F942EA38DE40E94565B882309F484C0A7
:102510000E94E85A2E81273009F094C0882309F4DC
:1025200091C0BB24B394AA24AA94AB0C09A11AA10C
:10253000612C8EEF882E8B0C6A2D862D0F9488C906
:1025400099249394960C81116EC06B2D862D0F9457
:1025500088C9C12CD12C7601712C882381F020E010
:1025600030E0A901D8015D966D917D918D919C918E
:1025700090970F947CDD6B017C0177247394682D18
:10258000862D0F9488C9882369F0F8017B972081F4
:10259000318142815381C701B6010F947CDD6B010B
:1025A0007C0173946A2D892D0F9488C9882361F06A
:1025B000F8012581368147815085C701B6010F9406
:1025C0007CDD6B017C0173946A2D8FEF860D0F9477
:1025D00088C9882331F1F801339720813181428104
:1025E0005381C701B6010F947CDD6B017C017394AC
:1025F000672D70E090E080E00F94E2D69B01AC0183
:10260000C701B6010F947BDED80111966D937D93BF
:102610008D939C93149707C08CEA9DE00F9454DC33
:1026200079CF7110E5CF692C0C5F1F4FB7E09B127B
:1026300083CFB394E9A1FAA17C96FAA3E9A3F8E0C9
:10264000BF1271CF81E08093C2138FE40E94565B6A
:10265000811103C00F942ECA9BCC0E94E85A8111AD
:10266000F9CF0E94436694CC4F925F926F927F9213
:102670008F929F92AF92BF92EF92FF920F931F9310
:10268000CF93DF931F92CDB7DEB744E050E064E113
:1026900070E08EEB9DE00F9444DC43E050E063E794
:1026A00077E78EEB9DE00F9433DA892B09F0A0C118
:1026B000E7E3F8E7459155916591749188ED90E0D5
:1026C0000E94A763EBE3F8E74591559165917491FA
:1026D0008CED90E00E94A763EFE3F8E7649180EE51
:1026E00090E00E948975E0E4F8E76591749181EECD
:1026F00090E00E947175E2E4F8E76591749183EED1
:1027000090E00E947175E3E3F8E74591559165917A
:10271000749184ED90E00E94A7634FE058E760E178
:1027200070E080EB90E00E9452754FE158E760E165
:1027300070E080EC90E00E9452754FE258E764E050
:1027400070E080ED90E00E94527541ED50E064E150
:1027500070E08EEB9DE00F9444DC0E9439650EEB37
:102760001DE08AE5E82E8EE0F82E94EC892E99E0A3
:10277000992EA12CB12C20EC422E23E0522E612C5C
:10278000712C20E030E048E453E4F8016489758955
:10279000868997890F9405E018164CF480E090E044
:1027A000A8E4B3E4F801848B958BA68BB78BF70173
:1027B00061917191819191917F0120E030E048EC2D
:1027C00052E40F9405E0181654F480E090E0A8EC71
:1027D000B2E4F701349780839183A283B383F80135
:1027E00084A195A1A6A1B7A1853C9940A105B105F9
:1027F00028F0F80184A295A2A6A2B7A2F7018485C9
:102800009585A685B785813C9340A105B10528F043
:10281000F70144865586668677860C5F1F4FFDE07C
:10282000063C1F0709F0ADCF60917A0E70E080E0A2
:102830000F94FF2560917B0E70E081E00F94FF25DF
:1028400060917C0E70E082E00F94FF2560917D0E18
:1028500070E083E00F94FF250F949A640F94D83BA7
:10286000CE0101960F949F3244E350E867EB7AEB78
:1028700082EA9CE00E94A76346E656E666E87FE3AC
:102880008EE99CE00E94A7634AE959E969E17EE389
:102890008AE99CE00E94A7636EE071E088E99CE011
:1028A0000E94717561E087E99CE00E94897582E071
:1028B0009DE00F9454DC91E0811101C090E0909371
:1028C0001D058EEF9CE00F945CDC6093DA12709330
:1028D000DB128093DC129093DD1282EA9CE00F946D
:1028E0005CDC6093DE127093DF128093E0129093B1
:1028F000E1128EE99CE00F945CDC6093E21270932D
:10290000E3128093E4129093E5128AEF9CE00F9417
:102910005CDC6093E6127093E7128093E812909368
:10292000E9128AE99CE00F945CDC6093EA127093F0
:10293000EB128093EC129093ED1288E99CE00F94D7
:1029400062DC0F94872F40E450E06AEB7CE080EF7C
:1029500092E10F9444DC86EB9CE00F945CDC609386
:10296000301370933113809332139093331382EBAF
:102970009CE00F945CDC6093341370933513809368
:102980003613909337138EEA9CE00F945CDC6093CF
:1029900038137093391380933A1390933B130F9429
:1029A000A62F811106C08DE097E70E94FB780F9457
:1029B000AD320F940E30CE0101960F94923282EC1C
:1029C0009AEA0E94D07687E397E70E94FB7881E03D
:1029D0000F90DF91CF911F910F91FF90EF90BF90DB
:1029E000AF909F908F907F906F905F904F900895E1
:1029F0000E940C8264E070E084E190E00E943B5B06
:102A000091E08927E5CF2F923F924F925F926F928C
:102A10007F928F929F92AF92BF92CF92DF92EF926E
:102A2000FF920F931F93CF93DF93CDB7DEB7CF58AD
:102A3000D1090FB6F894DEBF0FBECDBF82E0809300
:102A4000BE02A0909212B0909312850108551F4EBD
:102A500046E050E06FE078E8C8010F9433DA892B44
:102A600009F0B8C080E098E80E94A667882309F4BE
:102A700091C088E50E94565B182F89E50E94565B3D
:102A8000811112600F94ED431A821982FE01339670
:102A900083E1DF011D928A95E9F748EC5FEA60E087
:102AA00070E085E793E00F94352B81111092740349
:102AB000009174030F5F0093740385E793E00F9414
:102AC000F42C80917303812B8093730310FF08C053
:102AD00086E69FE00E94A87585E09FE00E949B75B6
:102AE00011FF08C088E69FE00E94A87583E09FE080
:102AF0000E949B7581E00E94A56E82E00E94276E75
:102B0000612FCE0101960E948973CE0101960E9429
:102B100067F540E061E081E00E94857E61E084E944
:102B200094E8033060F11092B70D1092B60D80E07A
:102B30000E94A56E0E94936E60917303CE01019670
:102B40000E94897310927303CE0101960E946770F0
:102B500084EA96E40E942C72AC0161E080E00E945D
:102B6000746E8FE30E944F6E40E060E090E080E082
:102B70000F946E5061E081110AC086E894E80E94CB
:102B8000A08781E08093BE020E94AA7E5EC389E78F
:102B900094E8F5CF82EF97E80E94A667882369F052
:102BA0000E940567811106C060E070E080E89FE345
:102BB0000E94C4670F945A27E4CF85EE97E80E94DD
:102BC000A6678823F1F20F945A2760E080E00E9404
:102BD00078F5D7CF44E050E060EE77E8C8010F9475
:102BE00033DA892B09F0FCC0850104551F4E49E0FA
:102BF00050E066ED77E8C8010F9433DA892BC9F409
:102C0000F501EB54FF4E1081153489F0185514303E
:102C100008F0B7CF4AE050E070E060E0C5018A54A8
:102C20009F4E0F94DFD7812F0F94C488AACF13E053
:102C3000F1CF49E050E06CEC77E8C8010F9433DA4B
:102C4000892B51F5F501EB54FF4E1081153411F12C
:102C50001855143008F095CF4AE050E070E060E07D
:102C6000C5018A549F4E0F94DFD7E12FF0E0EB505F
:102C7000FB4F808140E051E002C0569547958A9510
:102C8000E2F7842F880F880F81506823812F0F94DB
:102C9000DB8B77CF13E0E0CF49E050E062EC77E8E0
:102CA000C8010F9433DA892B09F06BCFF501EB548F
:102CB000FF4E8081853409F490C098EAC92EC80E71
:102CC000B3E0BC1508F45DCFEC2CF12C4701880C67
:102CD000991CF401EB55FD4F0081202F2F70102F10
:102CE00012951770001F0027001F61816770660F23
:102CF000062BF401EA55FD4FD080D694D694D69495
:102D0000ED2DE370DE2E1A821982C5018A549F4E82
:102D1000DC013C91B22E3323E1F14AE050E0BE01E8
:102D20006F5F7F4F0F94DFD76F70B62E89819A81C6
:102D3000009779F1FC012081222359F14AE050E00B
:102D4000BE016F5F7F4F0F94DFD7162F17708981F9
:102D50009A810097F1F0DC012C912223D1F04AE016
:102D600050E0BE016F5F7F4F0F94DFD7062F0F70CB
:102D700089819A81009769F0FC012081222349F022
:102D80004AE050E0BE016F5F7F4F0F94DFD7637062
:102D9000D62EF401EB55FD4F17701295107F602F62
:102DA0006795662767951B29162B1083602F6695FC
:102DB0000181007E2D2D2370D22EDD0CDD0CDD0C6B
:102DC000062BD02AD182F701EB50FB4F50E040E0B8
:102DD00060818C2D0F949425D4CE03E0C02E74CF47
:102DE00045E050E06CEB77E8C8010F9433DA892BAB
:102DF00009F064C182EB97E80E94A667882309F472
:102E00003CC010926F0614E6C12CD12C76016F9A4B
:102E1000779864E170E080E090E00F9458280F9478
:102E200032284B015C01F8946F98679BFECF789431
:102E30000F943228DC01CB0188199909AA09BB0932
:102E4000C816D906EA06FB0610F46C017D01115084
:102E5000F1F68EE694E80E94D0768AE694E835EFA3
:102E6000C31631E0D306E104F10410F487E694E8D8
:102E70000E94FB786F98779A84CE8EEA97E80E943A
:102E8000A667882321F14091CB035091CC032CE31A
:102E9000249FC001259F900D11249F938F934091F3
:102EA000C9035091CA03249FC001259F900D11248E
:102EB0009F938F9384E899E69F938F930F9416DBEB
:102EC0000F900F900F900F900F900F905ACE89EAAD
:102ED00097E80E94A667882311F18CE89FE00F9481
:102EE00054DC811110C061E08CE490E70E94A0875F
:102EF00060E085EA9FE00F9478DC60E08FE79CE07B
:102F00000F9478DC3ECE813009F03BCE0F94924393
:102F10008EE095E00F94B22A0F945D2A32CE82EAB9
:102F200097E80E94A667882321F080E00F94811023
:102F300028CE8CE997E80E94A667882351F010926A
:102F4000FC1F1092FD1F1092FE1F1092FF1F0E9487
:102F5000CC6689E997E80E94A6678823A9F044E136
:102F600050E065E17DE0CE0101960F9444DC8C8950
:102F7000882329F08EE897E80F943DDB02CECE013E
:102F800001960F94E3E2FDCD8AE897E80E94A667D8
:102F9000882329F08EE797E80E94FB78F2CD8AE734
:102FA00097E80E94A667882319F08DE597E8F4CF8B
:102FB00088E597E80E94A667882319F00E94AC7004
:102FC000E0CD85E597E80E94A667882379F081EA3D
:102FD0009DE00F9454DC4BE0849FC001112470E00D
:102FE00060E0805B924F0F9496DCCBCD82E597E852
:102FF0000E94A667882351F00E94936E40E070E023
:1030000060E084E690E00F948152D8CF8EE497E898
:103010000E94A6678823E1F086E50E94565B88231C
:1030200009F4AFCD0E94F55A11E0892B09F410E0A4
:103030000F94ED438091C21390E01817190609F41C
:10304000A0CD1093C2138AE996E00F942C6599CD18
:1030500087E497E80E94A667882309F492CD84E468
:103060000E94565B8823A1F00E941D6020E030E0A2
:103070004AE754E40F9421D720E030E040E05FE3DA
:103080000F947CDD0F94F4DECB010E940EF679CD17
:1030900083E497E80E94A66785EA9DE00F9462DCCE
:1030A000BC0190E080E00F94E0D620E030E04AE7F9
:1030B00054E40F947BDE0F94EF7563CDD8018C91AF
:1030C000873411F00C94F9A31093960300939503A1
:1030D0000E94F55A90939403809393038E31910547
:1030E00009F4DAC60CF045C18430910509F47EC6B6
:1030F0000CF0C5C097FDCBC002970CF0FCC10E943C
:10310000F3598C010E9444616091650670916606D6
:1031100080916706909168060F94E0D66B017C0160
:1031200040909E0650909F066090A0067090A10669
:103130008090800690908106A0908206B0908306D1
:10314000A5019401C301B2010F947BDD20E030E0C2
:1031500048EC52E40F9421D79B01AC01C701B601A2
:103160000F9405E01816D4F4A3019201C501B4012F
:103170000F947BDD20E030E048EC52E40F9421D73F
:10318000A70196010F947CDD0F94F4DE6093650631
:103190007093660680936706909368068091400E50
:1031A000882309F4A4C188E50E94565B81119FC160
:1031B00089E50E94565B81119AC18AE50E94565B9F
:1031C000811195C185E40E94565B882309F48FC163
:1031D00020919E0630919F064091A0065091A10635
:1031E000609180067091810680918206909183069D
:1031F0000F947BDD6B017C012DEC3CEC4CEC5DEB2A
:103200000F9471DE87FF65C180918E0681110C9449
:103210000DCD0F94ED438091800690918106A09191
:103220008206B091830680939E0690939F06A0939A
:10323000A006B093A1068EE996E00F94F9649091F0
:103240008E0681E089270F94608AC157DF4F0FB641
:10325000F894DEBF0FBECDBFDF91CF911F910F91CC
:10326000FF90EF90DF90CF90BF90AF909F908F90A6
:103270007F906F905F904F903F902F9008958B308C
:10328000910509F400C6DCF40A9709F4F8C58091A9
:1032900092129091931288559F4E9F938F931F92F5
:1032A00087E48F9386EA98E69F938F930F9416DBBB
:1032B0000F900F900F900F900F900F90A5C0853139
:1032C000910509F4A1C04C9711F788E50E94565B5F
:1032D000382E412C512C3201882321F00E94025BB0
:1032E0002B013C0189E50E94565B282E882309F4B6
:1032F000CCC50E94025B6E966CAF7DAF8EAF9FAF68
:103300006E978AE50E94565BD82E812C912C540131
:10331000882321F00E94025B4B015C0187E50E943B
:10332000565B67968FAF679783E40E94565B6796FC
:10333000FFAD6797FF938F93CD2C6E96ECACFDACF1
:103340000EAD1FAD6E97222DB301A201832D0E94F9
:10335000A77C0F900F90311057C0211055C0679671
:103360002FAD6797211150C0D1104EC00E947C8DA7
:103370004BC08635910511F40C94A8A3B4F58C3498
:10338000910509F4DFC53CF508E210E0F6E5EF2E03
:10339000F9E6FF2E8B34910509F079CF602F70E0AC
:1033A00090E080E00F94E0D60E940A5C9F938F9398
:1033B0007F936F931F930F93FF92EF920F9416DBFF
:1033C0000F5F1F4F0FB6F894DEBF0FBECDBF0F3695
:1033D000110521F719C08035910541F2813591051C
:1033E00009F055CF0E94DB7E0FC08A35910511F49C
:1033F0000C94B2A374F48735910511F40C94ADA329
:103400008835910509F043CF1092940310929303ED
:10341000B8CB8B35910511F40C94B9A38C3591057B
:1034200009F035CFBDEDCB2EB2E0DB2E8E010F5B68
:103430001F4F9E012F5F3F4F790181EE882E82E062
:10344000982E58013901D6018D916D010E94565B6D
:10345000F50181935F01882341F00E941D60D7012F
:103460006D937D938D939C931397B4E0EB0EF11CB9
:103470008C149D0441F7F801D380DD2011F40C94E5
:10348000BDA320E030E0A9016D857E858F859889F8
:103490000F9471DE81110C94BDA3D8018C91811120
:1034A0000C94BDA311968C91119781110C94BDA31E
:1034B00012968C9181110C94BDA310929E061092CD
:1034C0009F061092A0061092A10681E08093B80496
:1034D0009BCF2DEC3CEC4CEC5DE3C701B6010F94A7
:1034E00005E0181624F480918E06811192CEC80151
:1034F0000E94886B89CF0E94F359E0969FAF8EAFF0
:10350000E0970E94446189E40E94565B882309F495
:1035100000C40E941D6060938B0370938C038093A2
:103520008D0390938E038AE40E94565BC12CD12CAC
:103530007601882321F00E941D606B017C01C092FE
:103540008F03D0929003E0929103F0929203E09166
:103550009303F0919403C257DF4FF983E883CE5869
:10356000D04080908B0390908C03A0908D03B090FE
:103570008E03A7019601C501B4010F9418E0AE9621
:103580006CAF7DAF8EAF9FAFAE97609139027091F7
:103590003A02072E000C880B990B0F94E2D620916B
:1035A000B8023091B9024091BA025091BB020F9417
:1035B00021D72EE333EC4EE259E30F9421D7AA969C
:1035C0006CAF7DAF8EAF9FAFAA9780E1E2E9F6E0E6
:1035D000DE01119601900D928A95E1F7A501940103
:1035E00050586A962CAF3DAF4EAF5FAF6A97D70188
:1035F000C601B0586E968CAF9DAFAEAFBFAF6E97A1
:1036000029813A814B815C81E6962CAF3DAF4EAF6C
:103610005FAFE697C501B4010F947CDDEA966CAF0D
:103620007DAF8EAF9FAFEA978D819E81AF81B885C8
:10363000EE968CAF9DAFAEAFBFAFEE979C01AD01E4
:10364000C701B6010F947CDDCE57DF4F68837983C5
:103650008A839B83C258D04029853A854B855C85F7
:1036600060917C0670917D0680917E0690917F0628
:103670000F947BDDC258DF4F688379838A839B83F5
:10368000CE57D04020917406309175064091760651
:1036900050917706CA57DF4F288339834A835B836B
:1036A000C658D040EA962CAD3DAD4EAD5FADEA9721
:1036B000CA57DF4F688179818A819B81C658D04083
:1036C0000F947BDD6B017C018091780690917906E7
:1036D000A0917A06B0917B06C657DF4F8883998305
:1036E000AA83BB83CA58D040CE57DF4F2881398187
:1036F0004A815B81C258D040BC01CD010F947BDD73
:103700004B015C013090820E2090830E9091840ECC
:103710006F969FAF6F97A091850EA396AFAFA397BB
:10372000A70196016A966CAD7DAD8EAD9FAD6A978F
:103730000F9421D72B013C01A50194016E966CAD2D
:103740007DAD8EAD9FAD6E970F9421D79B01AC01DF
:10375000C301B2010F947CDD2B013C01A501940152
:103760006A966CAD7DAD8EAD9FAD6A970F9421D7F3
:103770004B015C01A70196016E966CAD7DAD8EADDF
:103780009FAD6E970F9421D79B01AC01C501B40189
:103790000F947BDDA30192010F94FBDD6B017C0193
:1037A00020E030E0A9010F9471DE87FF0AC02BED05
:1037B0003FE049EC50E4C701B6010F947CDD6B019A
:1037C0007C0160918B0E70918C0E6115710509F46E
:1037D000A4C290E080E00F94E0D69B01AC016BEDB9
:1037E0007FE089EC90E40F947BDEAE962CAD3DAD8E
:1037F0004EAD5FADAE970F9421D75B018C01609108
:103800008D0E70918E0E61157105F1F090E080E0E3
:103810000F94E0D620E030E040E752E40F9421D747
:103820009B01AC01AA966CAD7DAD8EAD9FADAA9704
:103830000F947BDE3B014C019501A8010F9471DED2
:1038400087FF02C0530184014090860E5090870E7E
:103850006090880E7090890E9501A801B201C30195
:103860000F9405E01816C4F09501A801632D722D80
:103870006F968FAD6F97A3969FADA3970F9471DE50
:103880002501380187FF08C0432C522C6F966FAC7E
:103890006F97A3967FACA397C257DF4FE881F9815A
:1038A000CE58D040329751F42BED3FE049EC50E434
:1038B000C701B6010F947BDD6B017C01CA57DF4F56
:1038C000288139814A815B81C658D040E6966CAD2B
:1038D0007DAD8EAD9FADE6970F9471DE811125C051
:1038E000C657DF4F288139814A815B81CA58D04051
:1038F000EE966CAD7DAD8EAD9FADEE970F9471DE03
:10390000811113C020E030E0A901C701B6010F9476
:1039100071DE81110AC02BED3FE049EC50E4C70194
:10392000B6010F947CDD6B017C01A7019601AE9678
:103930006CAD7DAD8EAD9FADAE970F9421D7C258C3
:10394000DF4F288139814A815B81CE57D0400F9467
:1039500018E04B015C012FE632E143E85AE30F9493
:1039600071DE87FDCFC19201A301C501B4010F949F
:103970007BDE0F945ADE0F94F4DEA4967FAF6EAF19
:10398000A4976230710508F48BC1E0964EAD5FAD2F
:10399000E097452B09F484C150918A0E6F965FAF72
:1039A0006F9790E080E00F94E0D64B015C01AC0192
:1039B0009B01C701B6010F947BDE2B013C01A501E1
:1039C0009401C258DF4F688179818A819B81CE57EB
:1039D000D0400F947BDEEE966CAF7DAF8EAF9FAF85
:1039E000EE972D853E854F855889609180067091B0
:1039F000810680918206909183060F947BDDA5015C
:103A000094010F947BDEC258DF4F688379838A83E9
:103A10009B83CE57D040A3019201C301B2010F9402
:103A200021D76B017C01AC019B01C301B2010F9452
:103A300021D720E030E040EC50E40F947BDE9B0186
:103A4000AC01C301B2010F947BDDAE966CAF7DAFCC
:103A50008EAF9FAFAE9720E030E040E05FE3C7015C
:103A6000B6010F9421D79B01AC0160E070E080E8C3
:103A70009FE30F947BDDE6966CAF7DAF8EAF9FAF7B
:103A8000E69722242394312C6F968FAD6F97811186
:103A90004DC1B10190E080E00F94E0D6A301920106
:103AA0000F9421D76B017C010F9476DE6E966CAF7C
:103AB0007DAF8EAF9FAF6E97C701B6010F943CE10B
:103AC0004B015C01C0908B03D0908C03E0908D0380
:103AD000F0908E03F7FAF094F7F8F09420918F03AA
:103AE000309190034091910350919203A2962CAF94
:103AF0003DAF4EAF5FAFA297A70196016E966CAD3A
:103B00007DAD8EAD9FAD6E970F9421D76A966CAF49
:103B10007DAF8EAF9FAF6A97A2962CAD3DAD4EADF7
:103B20005FADA297C501B4010F9421D79B01AC01F1
:103B30006A966CAD7DAD8EAD9FAD6A970F947CDDBE
:103B40006A966CAF7DAF8EAF9FAF6A97A701960163
:103B5000C501B4010F9421D76B017C01A2962CAD55
:103B60003DAD4EAD5FADA2976E966CAD7DAD8EADA9
:103B70009FAD6E970F9421D79B01AC01C701B60191
:103B80000F947BDD6E966CAF7DAF8EAF9FAF6E975F
:103B900030918A0E6F963FAF6F976A962CAD3DAD10
:103BA0004EAD5FAD6A97EA966CAD7DAD8EAD9FADC3
:103BB000EA970F947CDD69837A838B839C836E966E
:103BC0002CAD3DAD4EAD5FAD6E97CE57DF4F6881EA
:103BD00079818A819B81C258D0400F947CDD6D83AE
:103BE0007E838F839887EE962CAD3DAD4EAD5FAD55
:103BF000EE9769857A858B859C850F947CDD698736
:103C00007A878B879C87C258DF4F288139814A8108
:103C10005B81CE57D0406D857E858F8598890F94C6
:103C20007CDD6D877E878F87988BCE0101960E9401
:103C3000496BE0968EAD9FADE0972816390608F1E6
:103C4000E984FA840B851C852D813E814F8158853E
:103C500069817A818B819C813F922F92A2E9B6E0A3
:103C6000BF93AF93AA968CAC9DACAEACBFACAA97F9
:103C7000DE011D966D010F942CB10F900F900F90E7
:103C80000F908091AC0D81113DC0BFEF2B1A3B0A04
:103C9000A496EEADFFADA497E215F30509F0F4CEBE
:103CA00084E796E00E94496BE0907C06F0907D06E8
:103CB00000917E0610917F0620917806309179065A
:103CC00040917A0650917B0660917406709175065A
:103CD00080917606909177061F921F92E2E9F6E0B6
:103CE000FF93EF93AA968CAC9DACAEACBFACAA97F9
:103CF000A0E8CA2EA6E0DA2E0F942CB10F900F90F8
:103D00000F900F900E947F5A86E893E00F94F42C56
:103D10007BCB60E070E0CB01FECBA32CB22C6F9686
:103D20000FAD6F97A3961FADA39769CD6F964FAD5B
:103D30006F9741506F964FAF6F97AE962CAD3DADDC
:103D40004EAD5FADAE976A966CAD7DAD8EAD9FAD5D
:103D50006A970F9421D76B017C01E6962CAD3DAD9F
:103D60004EAD5FADE6976E966CAD7DAD8EAD9FAD01
:103D70006E970F9421D79B01AC01C701B6010F9438
:103D80007CDD7B018C01E6962CAD3DAD4EAD5FAD8B
:103D9000E6976A966CAD7DAD8EAD9FAD6A970F9438
:103DA00021D74B015C01AE962CAD3DAD4EAD5FAD64
:103DB000AE976E966CAD7DAD8EAD9FAD6E970F9448
:103DC00021D79B01AC01C501B4010F947BDD6A963C
:103DD0006CAF7DAF8EAF9FAF6A97C701D8016E966B
:103DE0008CAF9DAFAEAFBFAF6E97D7CE80E50E94D0
:103DF000565BC12CD12C7601882331F00E941D60C6
:103E00000F94F4DE6B017C0183E50E94565B8823EE
:103E100061F00E941D6020E030E04AE754E40F9416
:103E200021D70F94F4DE6B017C01C114D104E104AD
:103E3000F10441F08091C406873021F08BE799E6C8
:103E40000E943BF20F94ED430F94512AC60ED71EE9
:103E5000E81EF91E86E893E00F94F42C0F94512A83
:103E60006C157D058E059F0508F0CECA0F9461394B
:103E700080E00E94378A80E00E94276EEFCF81E0C9
:103E80000F94608AC1CA80E0FBCF6E961CAE1DAE57
:103E90001EAE1FAE6E9735CA0F94ED4381E080933E
:103EA000A70D0E9468668C0180E090E0A8E4B4E46D
:103EB0008093B8029093B902A093BA02B093BB0268
:103EC00043E060E070E080E291EC0F948F8C7090A2
:103ED0009A0660909B0650909C0640909D06B0907C
:103EE0009606A09097069090980680909906F0907C
:103EF0009206E0909306D0909406C090950689E9CA
:103F000093E40E942C724F925F926F927F928F92F5
:103F10009F92AF92BF92CF92DF92EF92FF929F93C8
:103F20008F938FE599E69F938F930F9416DBC801CB
:103F30000E944E661092A70D0FB6F894DEBF0FBE1A
:103F4000CDBF62CA20E030E040E251E460919903C5
:103F500070919A0380919B0390919C030F9405E0CC
:103F600087FF05C08FE297E80E94FB784DCA82E088
:103F70000E947DEF811107C08EE09AE30E942C72AF
:103F80000F94F62041CA80918F06882341F08091DA
:103F90009006882321F010919106111108C081E04C
:103FA0008093A21080E49BE60F9438762DCA85ECAE
:103FB00099E30E942C720F94F62083E69EE30E9400
:103FC0002C7241E060E00F946E50811161C080E07E
:103FD00090E0A0EAB0E480939A0690939B06A093A9
:103FE0009C06B0939D0660E070E088E492E40F9434
:103FF00081C080E090E0A8E4B2E480939A069093B8
:104000009B06A0939C06B0939D0680E090E0A4E3FD
:10401000B3E48093960690939706A0939806B09386
:10402000990660E070E088E492E40F9481C00F94F8
:10403000ED4389E39EE30E942C720F94F620E3EF98
:10404000F4EA85919591A591B49180939606909309
:104050009706A0939806B0939906EFEEF4EA85913F
:104060009591A591B4918093920690939306A09315
:104070009406B093950660E070E088E492E40F94B3
:1040800081C00F94ED4341E060E080E00E94857EB6
:1040900020E030E04CE052E46091990370919A0383
:1040A00080919B0390919C030F9405E018160CF0EF
:1040B00073C080E090E0A8ECB2E480939A069093FD
:1040C0009B06A0939C06B0939D0660E070E088E498
:1040D00092E40F9481C00F941D3019821A821B82C2
:1040E0001C821D82CE0101960F94F42C03E2EFE5B1
:1040F000EE2EE4E8FE2E20E030E04CE052E4609149
:10410000990370919A0380919B0390919C030F9463
:1041100005E01816C4F587E799E30E942C720F9406
:10412000E92042E864E080E00E94806E1F920F93D5
:104130006091990370919A0380919B0390919C03E5
:104140000F94EDDE7F936F93FF92EF920E94396E92
:1041500081E80E944F6E88EE93E00E946C8C0E9472
:10416000DE7640E053E567E070E0CE0101960F9403
:10417000352B0F900F900F900F900F900F9088237A
:1041800009F4B9CF10E081E00E94A56E111104C0BE
:1041900080E00F94412138C90F94ED4381E0809372
:1041A000A70D0E94A56E81E197E80E94FB788090A0
:1041B000990390909A03A0909B03B0909C0320E0F9
:1041C00030E040EA50E4C501B4010F947BDE0F9467
:1041D000EDDE25E0269FA001279F500D1124BA0196
:1041E000550F880B990B0F94E2D61B017C0120E040
:1041F00030E04CE052E40F9471DE87FF06C0212CC2
:10420000312C6CE0E62E72E4F72E222D332D4E2D4C
:104210005F2DC501B4010F9405E0181664F420E089
:1042200030E040EA50E4622D732D8E2D9F2D0F94C7
:104230007CDD1B017C01FF92EF923F922F928DE378
:1042400099E69F938F930F9416DB20E030E040EFC8
:1042500051E4622D732D8E2D9F2D0F947BDD20E078
:1042600030E04CE852E40F947CDD0F94EDDE709367
:1042700073066093720684E08093C40681E08093A5
:10428000F70385EB94E40E942C720E943BF280E0DD
:1042900090E0A0EAB0E480939A0690939B06A093E6
:1042A0009C06B0939D0660E070E088E492E40F9471
:1042B00081C080E090E0A0EAB1E480939206909300
:1042C0009306A0939406B093950680E090E0A0E753
:1042D000B2E48093960690939706A0939806B093C5
:1042E000990660E070E088E492E40F9481C08AE966
:1042F00099E9A9E1BEE380939A0690939B06A09367
:104300009C06B0939D0660E070E088E492E40F9410
:1043100081C00F94ED430F900F900F900F900F906E
:104320000F902091990330919A0340919B035091F3
:104330009C03622D732D8E2D9F2D0F9405E0181672
:104340003CF488EE93E00E946C8C0E94DE76E9CF0C
:1043500060E086EA9FE00F9478DC80E090E0A0EADD
:10436000B0E480939A0690939B06A0939C06B0932A
:104370009D0660E070E088E492E40F9481C0EFEE67
:10438000F4EA85919591A591B491809392069093CA
:104390009306A0939406B0939506E3EFF4EA859113
:1043A0009591A591B4918093960690939706A093CA
:1043B0009806B093990660E070E088E492E40F9468
:1043C00081C00F94ED4343E060E070E080E89FEB34
:1043D0000F948F8C811106C00F9441211092A70D6C
:1043E0000C94049A90919A0667969FAF6797A09154
:1043F0009B066B96AFAF6B97B0919C066F96BFAF65
:104400006F97E0919D06A796EFAFA797EF93BF93A5
:10441000AF939F9380E399E69F938F930F9416DB5E
:104420000F900F900F900F900F900F904EEA842EE8
:104430004FE0942E53E2C52ED12C0FEF1FEFB601A3
:104440000D2C000C880B990B0F94E2D62B013C012C
:10445000DF92CF92C80102969F938F9324EF38E6A4
:104460003F932F930F9416DB58015FEFA51AB50AFF
:104470000F900F900F900F900F900F9011F40C94DD
:104480001BCD70E060E0C4010F9496DCA3019201A3
:10449000622D732D8E2D9F2D0F9471DE181644F40E
:1044A00085E0A816B10411F00C9427CD05E010E0CA
:1044B000580197E2A91A98EFB90AAA0CBB1C85E02B
:1044C000809F1001819F300C11240D5F1F4F2AE93E
:1044D000422E29E9522E29E1622E2EE3722E3BEB69
:1044E000832E38E6932EC801029705970CF0D4C0AE
:1044F000B101635D7F4F072E000C880B990B0F9461
:10450000E2D66B017C011F930F93A7EEB8E6BF9331
:10451000AF930F9416DB0093F70320E030E040EFF9
:1045200051E4C701B6010F947BDD20E030E040E2AA
:1045300051E40F9421D720E030E040EA50E40F949A
:104540007BDE20E030E048E452E40F947CDD0F9401
:10455000EDDE709373066093720680E090E0A0EA4F
:10456000B0E480939A0690939B06A0939C06B09328
:104570009D0660E070E088E492E40F9481C020E042
:1045800030E040EA51E42093920630939306409342
:1045900094065093950680E090E0A0E7B2E4809303
:1045A000960690939706A0939806B093990660E0BC
:1045B00070E088E492E40F9481C040929A06509291
:1045C0009B0660929C0670929D0660E070E088E415
:1045D00092E40F9481C00F94ED430F900F900F90D1
:1045E0000F902091990330919A0340919B03509131
:1045F0009C03C701B6010F9405E018163CF488EE41
:1046000093E00E946C8C0E94DE76EBCF80E090E01D
:10461000A0EAB0E480939A0690939B06A0939C0630
:10462000B0939D0660E070E088E492E40F9481C04E
:10463000EFEEF4EA85919591A591B491809392065D
:1046400090939306A0939406B0939506E3EFF4EA53
:1046500085919591A591B491809396069093970634
:10466000A0939806B093990660E070E088E492E425
:104670000F9481C00F94ED4343E060E070E080E868
:104680009FEB0F948F8C95E0290E311C0F5F1F4F0D
:10469000811104C00F94412181E09ECE67967FADC9
:1046A00067976B966FAD6B976F969FAD6F97A79659
:1046B0008FADA797272F362F492F582F60919A0635
:1046C00070919B0680919C0690919D060F947BDDD6
:1046D000F62EE72ED82EC92E2091CA0D3091CB0D83
:1046E0004091CC0D5091CD0DD701F6016B2F7A2F53
:1046F0008F2F9E2F0F9421D70F94EDDEA6966CAFCF
:104700007DAF8EAF9FAFA697CF92DF92EF92FF92D1
:1047100080919C038F9380919B038F9380919A0348
:104720008F93809199038F939F928F920F9416DBB2
:10473000A4966EAD7FADA497C5010F9496DCA2E060
:10474000AA0EB11C0FB6F894DEBF0FBECDBFCBCE04
:1047500080E10E941BEF0C94049A80E10E9470EFAC
:104760000C94049A8091E503887F8093E5030C9470
:10477000049A8091E5038760F8CF0F94ED43F12C04
:10478000E12CF80181918F018823D1F097012E56F9
:10479000394F5901F301EE0DFF1D20813181428116
:1047A0005381F701EA5EF14F6081718182819381CB
:1047B0000F947CDDD5016D937D938D939C9313971E
:1047C000B4E0EB0EF11CECE0EE16F104D1F6DD20C6
:1047D00061F08D859E85AF85B88980939E06909304
:1047E0009F06A093A006B093A1060F9441BF0C941E
:1047F000049A8D3411F00C948CCB10939603009393
:104800009503F801319681918032E9F38930D9F32B
:1048100080538A3070F01F930F938DEF96E89F932B
:104820008F930F9416DB0F900F900F900F900C94B6
:10483000C1950E94F55A9093AB0D8093AA0D893CC7
:10484000910511F40C9445B80CF040C38E349105D9
:1048500011F40C94A7B30CF035C28C31910511F40E
:104860000C9406B20CF000C18531910511F40C9442
:104870001FB10CF05EC08131910511F40C9414B19C
:10488000ECF4029710F40C9488B0809192129091FD
:10489000931288559F4E9F938F931F928DE48F9311
:1048A00086EA98E69F938F930F9416DB0F900F90F4
:1048B0000F900F900F900F900C946CB08231910577
:1048C00011F40C945EB5449701F781E08093BE0229
:1048D00086E998E60E94FB7884E50E94565B182FD3
:1048E0008CE40E94565B00E080FB00F910FB01F9AC
:1048F00086E195E10E94AC7683E2E6E1F5E1DE0136
:10490000119601900D928A95E1F720E050E040E089
:10491000BE016F5F7F4F88EF92E00F944A78CE011F
:1049200001960E94B17688E898E60E94FB780C9484
:104930006CB08831910511F40C9430B194F4863147
:10494000910511F40C9423B1479709F09ECF809103
:1049500095039091960361E004960F9486800C94E1
:104960006CB08A31910511F40C9476B114F00C946A
:1049700098B10DED12E0FFE3AF2EF2E0BF2EA1E201
:10498000CA2EA2E0DA2EB5E1EB2EB2E0FB2E80EECD
:10499000882E82E0982EF80181918F010E94565B4B
:1049A000882321F10E941D60D6014D905D906D908D
:1049B0007C90A30192010F9471DE87FD11C00E94CB
:1049C0001D60F7014080518062807380A3019201D5
:1049D0000F9405E0181624F00E941D602B013C0185
:1049E000D5014D925D926D927C921397B4E0AB0E1F
:1049F000B11CE4E0CE0ED11CF4E0EF0EF11C8016E9
:104A0000910649F683E50E94565B882311F40C94C5
:104A10000AC40E94E85A81110C946CB080E090E0C6
:104A2000A8E4B2E480933F0290934002A093410235
:104A3000B093420280E090E0AEE3B3E4809343029F
:104A400090934402A0934502B093460280E090E028
:104A5000A0EAB1E48093470290934802A0934902F0
:104A6000B0934A020C946CB08D32910511F40C9401
:104A7000ABB20CF0F0C08F31910511F40C9438B248
:104A80000CF06AC08D31910511F40C946CB04E9706
:104A900009F0FBCE80919114882311F40C946CB032
:104AA00080E297E10F94765980E297E10F94AB5939
:104AB00010928E1410928F1400919503109196030A
:104AC0000C5F1F4F80919114882311F40C946CB0EB
:104AD00080E297E10F94AB591092901423961FAF88
:104AE0000EAF2397CE018F5B9F4F0F9401808823D9
:104AF00011F40C946CB023964EAD5FAD239760918A
:104B0000391570913A1519821C8222E0CE01019666
:104B10000F94536581110C940EB210E0CE010196F2
:104B20000E94B176112311F40C9428B285E294E826
:104B30000E94D07623968EAD9FAD23970F9438D6E2
:104B40001092A4171092A5171092A6171092A717EB
:104B50000F94CD7D0C946CB08A32910511F40C94B5
:104B60005FB28C32910511F40C9492B2809709F0E7
:104B70008CCE8091901481110F94ED430091950398
:104B8000109196030C5F1F4F61E270E0C8010F9413
:104B9000ABE2009719F08C010F5F1F4F80E50E9478
:104BA000565BF82E8091950390919603081719078C
:104BB00008F4F12C80919114882311F40C946CB0BA
:104BC00061E06F25C8010F94868083E50E94565BE3
:104BD000882399F08091950390919603801791070F
:104BE00060F40E94025B6093A4177093A5178093F2
:104BF000A6179093A7170F94D776809191148823C6
:104C000031F081E08093901485E08093B80DF1102D
:104C10000C946CB080912317882361F08091A417C5
:104C20009091A517A091A617B091A717892B8A2B51
:104C30008B2B69F40E94A45B109282031092830371
:104C4000109284031092850380E00E9497810F9454
:104C500092430C946CB08934910511F40C94EFB22A
:104C6000F4F48E32910511F40C94B1B288349105AC
:104C700009F00BCE83E50E94565B882311F40C9457
:104C8000E0B20E94E85A882311F40C94DDB281301E
:104C900011F00C946CB08093B80D0C946CB08C3403
:104CA000910511F40C948FB314F00C94A2B38B34CF
:104CB000910509F0EACD0E94E0F5882311F40C94E7
:104CC0006CB0C5CF8E36910511F40C9455B60CF02E
:104CD00086C08635910511F40C94AEB5D4F58335B4
:104CE000910511F40C9458B584F48F34910511F4A6
:104CF0000C9412B48235910509F0C7CD8091E5037B
:104D0000877F8093E5030C946CB08435910511F492
:104D10000C945EB58535910509F0B7CD83E50E9409
:104D2000565B882311F40C946CB00E941D6020E047
:104D300030E04AE754E40F9421D70F94F4DE6093F7
:104D40007E0370937F0380938003909381030C9480
:104D50006CB08936910511F40C946EB4D4F48C3592
:104D6000910511F40C94CBB58836910509F08DCDE1
:104D700083E50E94565B882311F40C946CB00E946A
:104D80001D600F94EDDE7093B70D6093B60D0C941B
:104D90006CB08B36910511F40C9455B514F40C9449
:104DA00047B58D36910509F070CD8BE69DE40E94E4
:104DB0002C720E943BF281E08093E30383E50E9422
:104DC000565B882311F40C9482B40E941D600F94EA
:104DD000EDDE7093B70D6093B60D0C9488B48737F1
:104DE000910511F40C949AB7ACF58237910511F442
:104DF0000C944FB7B4F48037910511F40C945BB464
:104E00008137910509F041CD83E50E94565B8823E7
:104E100011F40C9466B60E94E85A80932F020C9409
:104E20006CB08537910511F40C9452B714F00C94C2
:104E300062B78337910509F028CD86E50E94565B5D
:104E4000882311F40C947BB686E094E80E94FB78EA
:104E50000C946CB08C38910511F40C945FB454F43C
:104E60008B37910511F40C94FFB78D37910509F438
:104E700080CD0BCD8E3B910511F40C94B8B4883CD9
:104E8000910511F40C9402B88B39910509F0FDCC11
:104E900083E50E94565B882361F00E94E85A809364
:104EA0008814882311F40C947AB489E894E10F945F
:104EB000F42C83E40E94565B882311F40C947EB496
:104EC0000E94E85A809387140C946CB0853FF1E0FF
:104ED0009F0711F40C94ECBF0CF060C4811531E015
:104EE000930711F40C946EBB0CF024C1803D910526
:104EF00011F40C94B1B90CF077C08D3C910511F40C
:104F00000C941BB9ACF58B3C910511F40C9492B840
:104F10008C3C910509F0B9CC83E50E94565B88234F
:104F200011F40C94EAB80E941D6060937E0E709399
:104F30007F0E8093800E9093810E6093F20D70939C
:104F4000F30D8093F40D9093F50D84E50E94565B6C
:104F5000882311F40C946CB00E941D606093F60DD0
:104F60007093F70D8093F80D9093F90D0C946CB03D
:104F70008E3C910511F40C9494B98F3C910509F085
:104F800084CC83E50E94565B882351F00E941D600B
:104F90006093410E7093420E8093430E9093440EA3
:104FA00086E40E94565B882361F00E941D600E9487
:104FB00047666093450E7093460E8093470E90931C
:104FC000480E8AE50E94565B882311F40C946CB05D
:104FD0000E941D606093490E70934A0E80934B0EA1
:104FE00090934C0E0C946CB08C3D910511F40C9484
:104FF00018BA0CF082C0813D910511F40C94D5B91A
:10500000863D910509F041CC80E50E94565B8823DE
:1050100011F40C9404BA0E941D602B013C0183E53D
:105020000E94565B882311F40C940EBA0E941D60F6
:105030004B015C018EE40E94565BD0908A0E88235F
:1050400029F00E941D600F94F4DED62E82E50E94A6
:10505000565BE0908B0EF0908C0E882329F00E9416
:105060001D600F94F4DE7B0186E40E94565B009184
:105070008D0E10918E0E882329F00E941D600F94D2
:10508000F4DE8B0120E030E0A901C301B2010F94EE
:1050900071DE181614F00C946CB020E030E0A90119
:1050A000C501B4010F9471DE87FF02C00C946CB08F
:1050B000A5019401C301B2010F9471DE87FF02C004
